:020000040800F2
:1000000000060020F505000821300008A12F000897
:10001000F92F0008A12F0008CD2F0008F7050008D0
:10002000F7050008F7050008F7050008BD410008BE
:10003000F7050008F7050008F7050008F7050008B0
:10004000F7050008F7050008F7050008F7050008A0
:10005000F7050008F7050008056E0008316E000876
:100060005D6E0008896E0008B56E0008F70500088F
:10007000F7050008F7050008F7050008F705000870
:10008000F7050008F7050008F7050008812B0008B0
:10009000F7050008912B0008F7050008E16E00083D
:1000A000F7050008F7050008F7050008F705000840
:1000B000F7050008F7050008F7050008F705000830
:1000C000F7050008F7050008F7050008F705000820
:1000D000F7050008F7050008F7050008F705000810
:1000E000456F0008F7050008F7050008F705000848
:1000F000F7050008F7050008F7050008F7050008F0
:10010000F7050008F7050008B96F0008F7050008B3
:10011000F7050008F7050008F7050008F7050008CF
:10012000F7050008F7050008F7050008F7050008BF
:10013000F7050008F7050008F7050008F7050008AF
:10014000F7050008F7050008F7050008F70500089F
:10015000F7050008F7050008F7050008F70500088F
:10016000F7050008F7050008F7050008F70500087F
:10017000F705000899610008F7050008F705000871
:10018000F7050008F7050008F7050008F70500085F
:10019000F7050008F7050008F7050008F70500084F
:1001A000F7050008F7050008F7050008F70500083F
:1001B000F7050008F7050008F7050008F70500082F
:1001C000F7050008F7050008F7050008F70500081F
:1001D000F7050008F7050008F7050008F70500080F
:1001E000F7050008F7050008F7050008F7050008FF
:1001F000F7050008F7050008F7050008F7050008EF
:10020000F7050008F7050008F7050008F7050008DE
:10021000F7050008F7050008F7050008F7050008CE
:10022000F7050008F7050008F7050008F7050008BE
:10023000F7050008F7050008F7050008F7050008AE
:10024000F7050008F7050008F7050008F70500089E
:10025000F7050008F7050008F7050008F70500088E
:10026000F7050008F7050008F7050008F70500087E
:10027000F7050008F7050008F7050008F70500086E
:10028000F7050008F7050008F7050008F70500085E
:10029000F7050008F7050008F7050008F70500084E
:1002A000F7050008F7050008F7050008F70500083E
:1002B000F7050008F7050008F7050008F70500082E
:1002C000F7050008F7050008F7050008F70500081E
:1002D000F7050008F7050008F7050008F70500080E
:1002E00069180008A12B0008292C00080000000054
:1002F00053B94AB9002908BF00281CBF4FF0FF318D
:100300004FF0FF3000F074B9ADF1080C6DE904CE88
:1003100000F006F8DDF804E0DDE9022304B07047E0
:100320002DE9F047089D04468E46002B4DD18A42A8
:10033000944669D9B2FA82F252B101FA02F3C2F1DB
:10034000200120FA01F10CFA02FC41EA030E94406C
:100350004FEA1C48210CBEFBF8F61FFA8CF708FB8D
:1003600016E341EA034306FB07F199420AD91CEB65
:10037000030306F1FF3080F01F81994240F21C8197
:10038000023E63445B1AA4B2B3FBF8F008FB1033DF
:1003900044EA034400FB07F7A7420AD91CEB040414
:1003A00000F1FF3380F00A81A74240F207816444E4
:1003B000023840EA0640E41B00261DB1D440002369
:1003C000C5E900433146BDE8F0878B4209D9002DCD
:1003D00000F0EF800026C5E9000130463146BDE857
:1003E000F087B3FA83F6002E4AD18B4202D38242C1
:1003F00000F2F980841A61EB030301209E46002D70
:10040000E0D0C5E9004EDDE702B9FFDEB2FA82F2C4
:10041000002A40F09280A1EB0C014FEA1C471FFA22
:100420008CFE0126200CB1FBF7F307FB131140EA09
:1004300001410EFB03F0884208D91CEB010103F1D6
:10044000FF3802D2884200F2CB804346091AA4B298
:10045000B1FBF7F007FB101144EA01440EFB00FE6C
:10046000A64508D91CEB040400F1FF3102D2A645D1
:1004700000F2BB800846A4EB0E0440EA03409CE770
:10048000C6F12007B34022FA07FC4CEA030C20FA1D
:1004900007F401FA06F31C43F9404FEA1C4900FA3D
:1004A00006F3B1FBF9F8200C1FFA8CFE09FB1811BA
:1004B00040EA014108FB0EF0884202FA06F20BD92D
:1004C0001CEB010108F1FF3A80F08880884240F27D
:1004D0008580A8F102086144091AA4B2B1FBF9F0C1
:1004E00009FB101144EA014100FB0EFE8E4508D9BC
:1004F0001CEB010100F1FF346CD28E456AD9023841
:10050000614440EA0840A0FB0294A1EB0E01A14225
:10051000C846A64656D353D05DB1B3EB080261EB93
:100520000E0101FA07F722FA06F3F1401F43C5E96D
:10053000007100263146BDE8F087C2F12003D840A3
:100540000CFA02FC21FA03F3914001434FEA1C47E5
:100550001FFA8CFEB3FBF7F007FB10360B0C43EAD7
:10056000064300FB0EF69E4204FA02F408D91CEB87
:10057000030300F1FF382FD29E422DD90238634485
:100580009B1B89B2B3FBF7F607FB163341EA034125
:1005900006FB0EF38B4208D91CEB010106F1FF3874
:1005A00016D28B4214D9023E6144C91A46EA00466B
:1005B00038E72E46284605E70646E3E61846F8E6FD
:1005C0004B45A9D2B9EB020864EB0C0E0138A3E746
:1005D0004646EAE7204694E74046D1E7D0467BE727
:1005E000023B614432E7304609E76444023842E79F
:1005F000704700BF02E000F000F8FEE772B638482E
:1006000080F30888374880F30988374837490860FD
:1006100040F20000CCF200004EF63471CEF2000140
:100620000860BFF34F8FBFF36F8F40F20000C0F23E
:10063000F0004EF68851CEF200010860BFF34F8FF4
:10064000BFF36F8F4FF00000E1EE100A4EF63C71E1
:10065000CEF200010860062080F31488BFF36F8F8C
:1006600005F048FA05F0EAF906F0A6F94FF0553022
:100670001F491B4A91423CBF41F8040BFAE71D4950
:10068000184A91423CBF41F8040BFAE71A491B4A49
:100690001B4B9A423EBF51F8040B42F8040BF8E79B
:1006A00000201849184A91423CBF41F8040BFAE770
:1006B00005F002FA06F002FA144C154DAC4203DACA
:1006C00054F8041B8847F9E700F042F8114C124D2A
:1006D000AC4203DA54F8041B8847F9E705F0EAB99D
:1006E00000060020002200200000000808ED00E0C5
:1006F0000000002000060020E07500080022002015
:10070000C8220020C8220020806B0020E0020008E0
:10071000EC020008EC020008EC0200082DE9F04FA2
:100720002DED108AC1F80CD0D0F80CD0BDEC108A99
:10073000BDE8F08F002383F311882846A0470020EE
:1007400004F02CFCFEE704F041FB00DFFEE70000B4
:10075000F8B505F047F930B1274B00220C211A7289
:100760005A729972DA7205F0FDF8074605F05CF9E5
:100770000546B8BB214B9F4234D001339F4234D051
:1007800027F0FF021E4B9A4232D12E4642F21074DD
:10079000F8B200F0B9FE00F0BDFE08B10024264614
:1007A00002F05AFD20B10024032000F07DF8264617
:1007B00035B1144B9F4203D0002405F02DF9264695
:1007C000002005F0D9F80EB100F084F801F0FCF932
:1007D00000F0C4FE01F0AEF8204600F02BF900F066
:1007E00079F8F9E72E460024D5E704460126D2E73A
:1007F000064641F28834CEE700220020010007B00F
:10080000000008B0263A09B008B501F065F8A0F17B
:1008100020035842584108BD07B541F21203022196
:1008200001A8ADF8043001F075F803B05DF804FBE1
:1008300038B5302383F31188174803680BB104F0EF
:10084000B5FC0023154A4FF47A71134804F0A4FC58
:10085000002383F31188124C236813B12368013BF2
:100860002360636813B16368013B63600D4D2B78AF
:1008700033B963687BB9022001F028F93223636041
:100880002B78032B07D163682BB9022001F01EF9E6
:100890004FF47A73636038BDC82200203108000825
:1008A000E8230020E0220020084B187003280CD811
:1008B000DFE800F008050208022001F005B9022077
:1008C00001F000B9024B00225A607047E02200207C
:1008D000E8230020F8B502F0BFFC30B14C4B0322F6
:1008E0001A7000224B4B5A60F8BD4B4B4B4A1C46CA
:1008F00019680131F8D004339342F9D16268484B4A
:100900009A42F1D9474B9B6803F1006303F58023BA
:100910009A42E9D205F068F8002001F031F802208F
:10092000FFF7C2FF404B00219A6C99641A6F196758
:100930001A6FDA6CD9645A6F59675A6F1A6D196554
:100940009A6F99679B6F394BD3F8802042F0006211
:10095000C3F88020D3F8802022F00062C3F8802002
:10096000D3F88020D3F8802042F00072C3F88020B2
:10097000D3F8802022F00072C3F88020D3F88030B2
:1009800072B64FF0E023C3F8084DD4E90004BFF37A
:100990004F8FBFF36F8F264AC2F88410BFF34F8F7B
:1009A000536923F480335361BFF34F8FD2F8803003
:1009B00043F6E076C3F3C905C3F34E335B0103EAA4
:1009C000060C29464CEA81770139C2F87472F9D2D3
:1009D000203B13F1200FF2D1BFF34F8FBFF36F8F86
:1009E000BFF34F8FBFF36F8F536923F4003353610D
:1009F0000023C2F85032BFF34F8FBFF36F8F302305
:100A000083F31188854680F3088820476CE700BF90
:100A1000E0220020E8230020000004082000040851
:100A2000FFFF03080022002000450258004402583E
:100A300000ED00E02DE9F04F93B0B74B2022FF21ED
:100A400000900AA89D6801F069F8B44A1378A3B928
:100A50000121B34811700360302383F311880368C8
:100A60000BB104F0A3FB0023AE4A4FF47A71AC48FB
:100A700004F092FB002383F31188009B13B1AA4B6F
:100A8000009A1A60A94A1378032B03D0002313702D
:100A9000A54A53604FF0000A009CD3465646D14603
:100AA000012001F011F824B19F4B1B68002B00F0CE
:100AB0002C82002000F010FF0390039B002B01DA32
:100AC00000F094FD039B002BEDDB012000F0FAFF0A
:100AD000039B213B1F2BE3D801A252F823F000BF58
:100AE000610B0008890B00081D0C0008A10A000812
:100AF000A10A0008A10A0008AF0C00087F0E000838
:100B0000990D0008FB0D0008230E0008490E00088F
:100B1000A10A00085B0E0008A10A0008CD0E00081B
:100B2000010C0008A10A0008110F00086D0B000855
:100B3000010C0008A10A0008FB0D0008A10A00082A
:100B4000A10A0008A10A0008A10A0008A10A0008D9
:100B5000A10A0008A10A0008A10A00081D0C00084B
:100B60000220FFF751FE002840F0F981009B02218E
:100B700005A8BAF1000F08BF1C4641F21233ADF8C8
:100B8000143000F0C7FE8BE74FF47A7000F0A4FE3B
:100B9000071EEBDB0220FFF737FE0028E6D0013FFF
:100BA000052F00F2DE81DFE807F0030A0D1013368F
:100BB0000523042105A8059300F0ACFE17E00421ED
:100BC0005548F9E704215A48F6E704215948F3E764
:100BD0004FF01C08404608F1040800F0D3FE042141
:100BE000059005A800F096FEB8F12C0FF2D1012077
:100BF0004FF0000900FA07F747EA0B0B5FFA8BFB8F
:100C000000F0D8FF26B10BF00B030B2B08BF00241C
:100C1000FFF702FE44E704214748CDE7002EA5D0A8
:100C20000BF00B030B2BA1D10220FFF7EDFD0746C4
:100C300000289BD00120002600F0A2FE0220FFF732
:100C400033FE5FFA86F8404600F0AAFE0446B0B1D3
:100C5000039940460136A1F140025142514100F052
:100C6000AFFE0028EDD1BA46044641F2121302212C
:100C700005A83E46ADF8143000F04CFE10E72546BE
:100C80000120FFF711FE244B9B68AB4207D9284691
:100C900000F078FE013040F067810435F3E700256D
:100CA000224BBA463E461D701F4B5D60A8E7002EE2
:100CB0003FF45CAF0BF00B030B2B7FF457AF02201C
:100CC000FFF7F2FD322000F007FEB0F10008FFF65A
:100CD0004DAF18F003077FF449AF0F4A08EB050347
:100CE000926893423FF642AFB8F5807F3FF73EAF40
:100CF000124BB845019323DD4FF47A7000F0ECFD00
:100D00000390039A002AFFF631AF039A0137019B43
:100D100003F8012BEDE700BF00220020E4230020B0
:100D2000C822002031080008E8230020E02200202B
:100D300004220020082200200C220020E4220020AF
:100D4000C820FFF761FD074600283FF40FAF1F2DB5
:100D500011D8C5F120020AAB25F0030084494245B1
:100D6000184428BF4246019200F0B2FE019AFF21CA
:100D70007F4800F0D3FE4FEAA803C8F387027C49FE
:100D80002846019300F0D2FE064600283FF46DAFDE
:100D9000019B05EB830533E70220FFF735FD0028B3
:100DA0003FF4E4AE00F02AFE00283FF4DFAE002757
:100DB000B846704B9B68BB4218D91F2F11D80A9BAD
:100DC00001330ED027F0030312AA134453F8203C3A
:100DD00005934046042205A9043702F027FA80460D
:100DE000E7E7384600F0CEFD0590F2E7CDF8148035
:100DF000042105A800F08EFD02E70023642104A869
:100E0000049300F07DFD00287FF4B0AE0220FFF7D0
:100E1000FBFC00283FF4AAAE049800F0E5FD059025
:100E2000E6E70023642104A8049300F069FD00288C
:100E30007FF49CAE0220FFF7E7FC00283FF496AE5B
:100E4000049800F0D3FDEAE70220FFF7DDFC00285C
:100E50003FF48CAE00F0E2FDE1E70220FFF7D4FCA6
:100E600000283FF483AE05A9142000F0DDFD0746FD
:100E70000421049004A800F04DFD3946B9E7322062
:100E800000F02AFD071EFFF671AEBB077FF46EAEC1
:100E9000384A07EB0903926893423FF667AE022097
:100EA000FFF7B2FC00283FF461AE27F003074F4480
:100EB000B9453FF4A5AE484609F1040900F062FDCA
:100EC0000421059005A800F025FDF1E74FF47A70A4
:100ED000FFF79AFC00283FF449AE00F08FFD002890
:100EE00044D00A9B01330BD008220AA9002000F04D
:100EF0001DFE00283AD02022FF210AA800F00EFE95
:100F0000FFF78AFC1C4804F04FF813B0BDE8F08FDF
:100F1000002E3FF42BAE0BF00B030B2B7FF426AE11
:100F20000023642105A8059300F0EAFC0746002889
:100F30007FF41CAE0220FFF767FC804600283FF4D8
:100F400015AEFFF769FC41F2883004F02DF80598E2
:100F500000F064FE46463C4600F02CFEA0E5064646
:100F60004EE64FF0000901E6BA467EE637467CE6DB
:100F7000E422002000220020A0860100094A49F254
:100F80006900136899B21B0C00FB013344F25061F5
:100F90001360054B186882B2000C01FB0200186058
:100FA00080B270471422002010220020002110225D
:100FB00010B5044600F0B2FD034B03CB2060616026
:100FC0001868A06010BD00BF00E8F11F2DE9F041D6
:100FD000ADF54E7D0D46002140F275126CAC074612
:100FE0000EA80D9100F09AFD4FF4C4720021204626
:100FF00000F094FD0DF1340802F01AF84FF47A7203
:10100000264BB0FBF2F0186093E80700012384E858
:1010100007000DF5E9702382FFF7C8FF40F604537F
:101020001F4907A8238406F0B1F815230DF2E32227
:101030000DF12C0C84F8323107AB1E46083203CE7A
:10104000664542F8080C42F8041C3346F5D1306876
:1010500041461060204633791371012201F0EEFF02
:10106000002380B2E97E0393AB7E029305F119035E
:1010700001930123009307A3D3E90023CDE9048062
:10108000384602F041FC0DF54E7DBDE8F08100BF11
:10109000AFF300809E6AC421818A46EEF0230020CF
:1010A000BC7100082DE9F043224DBBB001F0C0FF38
:1010B00040F2ED22AB68C31A934232D906AF2B46F9
:1010C00028220021A860384602F006FE05F10E0035
:1010D00000F01CFD002604465FFA80F905F10E08B9
:1010E000F3B2F100994501F1280107D908EB060395
:1010F00008223846013602F0EFFDF1E7082301220D
:101100000534297B0C48A4B2CDE902320B4B019384
:101110003023CDE90474009304A3D3E9002302F043
:10112000F3FB3BB0BDE8F083AFF3008078F6339F6C
:1011300093CACD8DE048002008340020ED480020FF
:10114000F0B58B8AC9B006460C46013B9BB2C92B51
:1011500047D8274D2F7B27BB05F10C0308223946C2
:1011600000933B46204602F07BFC7B1CFAB2D90080
:101170001F46A38A013B9A4205DA0E3200232A4415
:1011800000920822EEE700230022C5E90023002395
:10119000AB6085F8D730C5F8D8302B7B0BB9E37E30
:1011A0002B7306AD8122002127A800F0B7FC012295
:1011B000294627A802F00EF8002380B2E17E0393AF
:1011C000A37E029304F1190301932823CDE904506F
:1011D0000093304604A3D3E9002302F095FBFFF708
:1011E00061FF49B0F0BD00BF26417272DF25D7B75D
:1011F000E048002070B50D4614461E4602F01AFB6A
:1012000050B9022E10D1012C0ED112A3D3E9002324
:101210000120C5E9002307E0282C10D005D8012CB7
:1012200009D0052C0FD0002070BD302CFBD10BA3B2
:10123000D3E90023ECE70BA3D3E90023E8E70BA3F2
:10124000D3E90023E4E70BA3D3E90023E0E700BFE1
:10125000AFF30080401DA12026812A0B78F6339F32
:1012600093CACD8D9E6AC421818A46EE2641727250
:10127000DF25D7B7F017304A39059E562DE9F04FD4
:101280008DB080460D4602AF02F0D4FA0446002825
:101290005BD12B7E022B1BD1EB8A012B18D101F0E5
:1012A000C7FE0646FFF76AFE03464FF4C87006F510
:1012B0001676DFF81892B3FBF0F202FB103316FA41
:1012C00083F3C9F80030EB7E33B97B4B00221A70F0
:1012D0002C37BD46BDE8F08FAB8AE6B20134013B46
:1012E000B3420CD907F10803E100082228461E4446
:1012F00001F0F8010023009602F0B2FBECE707F1E1
:101300001800FFF753FE324607F1180107F10800F5
:1013100005F0BEFE0028D8D10F2E08D8664B1E70EF
:10132000D9F80030A3F51673C9F80030D0E7FB1DDB
:10133000F8710146072200930346284602F090FB0D
:10134000F979404602F06EFAC2E7EB8A282B26D0E4
:1013500010D8012B1ED0052BBAD1BFF34F8F5749A0
:10136000574BCA6802F4E0621343CB60BFF34F8F60
:1013700000BFFDE7302BABD16B7EE946514C01330A
:10138000627BDBB2934203D1EA7E237B9A420BD08D
:10139000CD469DE729464046FFF718FE98E72946C7
:1013A0004046FFF7CDFE93E74FF0000807F1180322
:1013B00010222846A7F8188041460093012302F026
:1013C0004FFBAE8A023EB6B2F31C9B109B00073364
:1013D000DB08A9EBC3039D460DF1080A1FFA88F349
:1013E0004FEAC8019E4201F110010AD90AEB080335
:1013F0000822284608F101080093002302F030FB80
:10140000ECE794F8D70000F0CBFAD4F8D8100546F2
:1014100019B994F8D70000F0D3FAD4F8D83033448F
:101420009D4205D294F8D7000021013000F0C8FA9F
:101430004FEA960B4FF000081FFA88F18B45D4E96C
:10144000003209D90AEB8801012203EB880008F178
:10145000010800F06BFBEFE7F31894F8D70042F1B6
:101460000002C4E90032D4F8D83006EB0308C4F80F
:10147000D88000F095FA804509D394F8D730D4F895
:10148000D8000133401B84F8D730C4F8D800FF2EB1
:101490000D4D09D80023237300F0B0FA01F0DCFEF3
:1014A000288108B9FFF716FA23689B0A01332B81BC
:1014B0000023A3606CE700BF0134002000ED00E0D2
:1014C0000400FA05E0480020F02300200434002046
:1014D0000A4B0B4A10B51A6003F5805393F8482065
:1014E0003AB95C6C2CB1204601F01EFC204605F098
:1014F000B7FD0448BDE8104001F016BC30340020B0
:101500003072000860440020014B1870704700BF23
:10151000FC23002010B54FF040540C4B22689A4237
:1015200012D1627D0A4B0B481A70C922237D0E30FE
:10153000094900F8023C00F0CBFAE02200212046E5
:1015400000F0ECFA012010BD0020FCE79AAD44C584
:10155000FC230020E04800201600003037B501F0E1
:101560007BFE194D02230022184928816B7101234B
:10157000174800F011FF002316494FF480520193E1
:10158000154B16480093164B02F026F9154B1978A7
:1015900011B1124802F046F901F04AFD0446FFF786
:1015A000EDFC4FF4C873B0FBF3F202FB130304F538
:1015B000167010FA83F00C4B186004F035FA08B17D
:1015C0000F232B8103B030BDF023002040420F00D9
:1015D0003034002000240020F511000808340020D9
:1015E0007D120008FC230020043400202DE9F04F78
:1015F000924C2DED028B8BA7D7E9006795B00FF2C7
:101600002C29D9E90089DFF84CA2DFF84CB220463A
:1016100002F0DEF9034650B300251095ADF84C50AA
:10162000CDE91155027B8DF84C2011AA99684068CC
:1016300003C21B6843F00043109301F0FBFC10EB66
:101640000A020095584641F1000310A900F04AFB38
:10165000A8427B4A05DD204602F0BEF9784A1570A3
:10166000D5E71378072B00F2B980013313700023FC
:101670000DADDFF8E4B10C93ADF83C300D936B6029
:101680009FED6C8B00234FF0010A0DF1250209A993
:1016900058468DF825308DF824A08DED008B01F093
:1016A00015FA9DF824200023002A40F09B80204654
:1016B00002F0C0F80546002847D1DFF8A0B101F0DC
:1016C000B7FCDBF8003098423FD301F0B1FC079043
:1016D000FFF754FC4FF4C873079AB0FBF3F102F51F
:1016E000167201FB130310A812FA83F3CBF8003033
:1016F000DFF86CB19BF80010002914BF2B4653464D
:1017000007918DF83030FFF751FC079910AB0DF1C0
:101710003100C1F110021944D2B2062A28BF0622B4
:10172000079200F0D5F9079A0CAB204603930132DB
:101730001823D2B20293434B04923246CDE900A360
:101740003B4602F079F88BF8005001F071FC3E4AFC
:101750003E4D1368C31AB3F57A7F32D3106001F09F
:1017600069FC02460B46204602F040F9204602F092
:1017700061F830B32B7B0DF1400BDFF8E8A0002BB4
:1017800014BF032302238AF8053001F051FC4FF403
:101790007A7301225946B0FBF3F0CAF800005046B4
:1017A00001F0F0FC182380B242460293284B0193CB
:1017B00040F25513CDE903B0009320464B4602F0AA
:1017C0003BF82B7B2BB1FFF76DFC2B7B002B7FF4C1
:1017D0001AAF15B0BDEC028BBDE8F08F204602F0C9
:1017E000FBF844E71946102210A800F097F90DF114
:1017F00026030AAA0CA9584600F07CFC11AB95E818
:10180000030083E803009DF83C3010A920468DF8C2
:101810004C300C9B1093DDE90A2302F0A5FA31E766
:10182000AFF30080401DA12026812A0BF1C6A7C17D
:10183000D068080F000000000000000008340020FD
:10184000C549002000340020C0490020E0480020A5
:10185000C449002040420F003034002004340020EE
:1018600001340020F023002008B5054800F0E8FC12
:10187000044A05490020BDE8084005F0EBBB00BF65
:10188000303400202C4C0020D11400080F4B70B5D0
:101890001B780C460133DBB2012B11D80C4D4FF4F1
:1018A0007A732968A2FB033222460E6A0146284653
:1018B000B047844204D1074B002201201A7070BD4A
:1018C0004FF4FA7003F070FB0020F8E718220020B4
:1018D000EC4E0020F4490020002307B50246012108
:1018E0000DF107008DF80730FFF7D0FF20B19DF80C
:1018F000070003B05DF804FB4FF0FF30F9E700008C
:101900000A46042108B5FFF7C1FF80F00100C0B20C
:10191000404208BD30B4054C0A46014623682046C3
:10192000DD69034BAC4630BC604700BFEC4E002085
:10193000A086010070B5104C0025104E03F08CFEFF
:1019400020803068238883420CD800252088013805
:1019500003F07EFE23880544013BB5F5802F2380EC
:10196000F4D370BD03F074FE336805440133B5F55C
:10197000802F3360E5D3E8E7F6490020C84900200E
:1019800003F048BF00F1006000F580200068704758
:1019900000F10060920000F5802003F0BFBE00005F
:1019A000054B1A68054B1B889B1A834202D91044C9
:1019B00003F04EBE00207047C8490020F6490020C1
:1019C00038B50446074D29B128682044BDE83840A1
:1019D00003F056BE2868204403F040FE0028F3D0F0
:1019E00038BD00BFC84900200020704700F1FF50FB
:1019F00000F58F10D0F8000870470000064991F8F4
:101A0000243033B100230822086A81F82430FFF71C
:101A1000BFBF0120704700BFCC490020014B1868B0
:101A2000704700BF0010005C244BF0B51A680446F4
:101A3000234BC2F30B06120C1F885868BE4293F961
:101A4000085028D09F89BE4206D101200C2505FBF5
:101A50000033586893F9085041F201039A421CD0B0
:101A600041F203039A421AD042F201039A4218D07B
:101A700042F203039A4208BF5625621E0B46441EDB
:101A80000A4493420FD214F9016F581C6EB10346F9
:101A900000F8016CF5E70020D8E75A25EDE7592555
:101AA000EBE75825E9E7184605E02C2482421C7034
:101AB00001D9981C5D70401AF0BD00BF0010005C99
:101AC0001C22002070470000704700007047000093
:101AD000002310B5934203D0CC5CC4540133F9E722
:101AE00010BD0000013810B510F9013F3BB191F96C
:101AF00000409C4203D11AB10131013AF4E71AB116
:101B000091F90020981A10BD1046FCE703460246E2
:101B1000D01A12F9011B0029FAD17047024403467A
:101B2000934202D003F8011BFAE770472DE9F8430E
:101B30001F4D14460746884695F8242052BBDFF80F
:101B400070909CB395F824302BB92022FF21484691
:101B50002F62FFF7E3FF95F824004146C0F1080229
:101B600005EB8000A24228BF2246D6B29200FFF7C2
:101B7000AFFF95F82430A41B17441E449044E4B2F0
:101B8000F6B2082E85F82460DBD1FFF737FF002876
:101B9000D7D108E02B6A03EB82038342CFD0FFF753
:101BA0002DFF0028CBD10020BDE8F8830120FBE702
:101BB000CC490020024B1A78024B1A70704700BFC4
:101BC000F44900201822002010B5104C104802F0F3
:101BD000E1FB21460E4802F009FC24680D48D4F8C8
:101BE0009020D2F8043843F00203C2F8043803F01E
:101BF000DBF90949204602F007FDD4F89020D2F81D
:101C0000043823F00203C2F8043810BD4C730008F6
:101C1000EC4E002040420F00547300087047000053
:101C2000302383F3118862B670470000002383F3EA
:101C3000118862B6704700007047000010B4134668
:101C4000026814680022A4465DF8044B6047000057
:101C500000F5805090F859047047000000F580505E
:101C600090F852047047000000F5805090F9580435
:101C7000704700004E20704700F5805208B5FFF70E
:101C8000CFFFD2F89834D2F894041844D2F89034A4
:101C90001844D2F878341844D2F888341844D2F86A
:101CA00084341844FFF7C2FF08BD000010B5044695
:101CB000FFF7B6FF084604F58054C4F854140B68C7
:101CC00007491B689847D4F8540494F85824012114
:101CD000036891405B689847FFF7A8FF10BD00BFFD
:101CE000044A00202DE9F74F0C4600F580511F46AD
:101CF000054691F852349046BDF830909BB1D1F82A
:101D000074340133C1F8743423689A0006D4237BF9
:101D1000082B0BD9627B0AB10F2B07D9D1F8783485
:101D20000133C1F878344FF0FF300FE0FFF778FF50
:101D3000EB6AD3F8C42012F4001A0AD0D1F87C342C
:101D400000200133C1F87C34FFF770FF03B0BDE819
:101D5000F08F22684FF0480BD3F8C460002A6B6AFA
:101D6000C6F30446B4BF42F0804292041BFB063B1C
:101D7000CBF8002023685B004FEA066344BF42F0C3
:101D80000052CBF80020227B43EA02437201CBF8D9
:101D90000430607B18B343F44013CBF80430D1F81F
:101DA000A4340133C1F8A434AB1803F58353197B71
:101DB00041F020011973207B019200F099FF03305C
:101DC000019A80105FFA8AF30AF1010A83420DDA60
:101DD00004EB83010BEB830349689960F2E7AB18CE
:101DE00003F58353197B60F34511E3E70121EB6AA7
:101DF00004F10C00B140C3F8D010AB18214603F534
:101E00008253C3E9048705EB461303F58253183365
:101E100051F804CB814243F804CBF9D109882A4414
:101E20002846198041F26803D65002F5805209F025
:101E3000030392F86C1043F0100321F01F010B43D1
:101E4000214682F86C304246FFF7F0FE3B46CDF863
:101E5000309003B0BDE8F04F00F010BF2DE9F0471F
:101E600000F58056044696F85254002D40F001814A
:101E7000037C032B40F092802B4628462F465FFAC6
:101E800083FC944510DA01EBCC0E51F83CC0BCF158
:101E9000000F04DBDEF804C0BCF1000F02DB0137E9
:101EA0000133ECE70130FBE7FFF7BAFEE36AF0B974
:101EB000D3F8800040F00200C3F880004E23E06AAF
:101EC000002F6ED1D0F8803043F00103C0F880308D
:101ED000694B6A4A1B6803F1805303F52C539B003E
:101EE0009342A36240F2AF80654801F09BF84D2811
:101EF00042D8DFF884814FEA004EDFF88891D8F8A5
:101F000000C04EEA8C0EC3F884E00CF1805303F558
:101F10002C539B00636100EB0C03D4F82CC0C8F871
:101F20000030C0F14E03DCF8800040F03000CCF807
:101F300080004FF0000CD4F81480E6465FFA8CF075
:101F40008242BCDD01EBC00A51F83000002810DBF2
:101F5000DAF804A0BAF1000F0BDA09EA00400AF03F
:101F60007F0A40EA0A0040F0084048F82E000EF1CF
:101F7000010E0CF1010CE1E79A6922F001029A616D
:101F800001F056F80646E36A9B69D90704D501F0CB
:101F90004FF8831BFA2BF6D9FFF748FE2846BDE819
:101FA000F087B7EB530F3DD2DFF8CCE04FEA074C98
:101FB000DEF800304CEA830CC0F888C003F1805092
:101FC00003EB4703002700F52C50CEF80030BC4649
:101FD0008000A061E06AD0F8803043F00C03C0F8C4
:101FE0008030D4F818E0FBB29A427FF771AF51F815
:101FF000330001EBC3080028D8F8043001DB002BC4
:102000000EDB20F0604023F0604340F0005043F0CE
:1020100000434EF83C000EEBCC000CF1010C436089
:102020000137E0E7836923F00103836101F000F8E1
:102030000646E36A9B69DA07AED500F0F9FF831B19
:10204000FA2BF6D9A8E7E26A936923F001039361BA
:1020500000F0EEFF0746E36A9B69DB0705D500F059
:10206000E7FFC31BFA2BF6D996E7012586F85254F1
:1020700092E7002592E700BF004A0020FCB500402F
:10208000F07100080000FF0713B500F580540191BE
:10209000606C00F07FFE1F280AD920220199606C35
:1020A00000F0EEFEA0F120035842584102B010BDEE
:1020B0000020FBE700F5805008B5FFF7B1FD406C4C
:1020C00000F03CFEBDE80840FFF7B0BD0022026012
:1020D00082814260826070470022002310B5C0E90F
:1020E0000023002304460C3020F8043CFFF7EEFFE9
:1020F000204610BD2DE9F047074688B09A4688462D
:1021000007F5805468469146FFF78AFDFFF7E4FF24
:10211000606C00F025FE1F282DD920226946606CD6
:1021200000F032FF202826D194F852341BB303ADBF
:10213000444605AB2E46083403CE9E4244F8080CB4
:1021400044F8041C3546F5D13068414620603846D5
:10215000B388A380DDE90023C9E90023BDF8083076
:102160004A46AAF80030FFF761FD534608B0BDE8C3
:10217000F04700F071BD0020FFF758FD08B0BDE842
:10218000F08700002DE9F84F0023064600F5815442
:10219000054688461034C0E90133264B46F8303BEB
:1021A000374638462037FFF797FFA742F9D105F5A4
:1021B00080544FF4805305F5A3594FF0000A26636D
:1021C0000026676405F5835709F110094FF0000BED
:1021D0001037E663C4E90D36012384F8403084F8F3
:1021E0004830A7F11800203747E910ABFFF76EFF22
:1021F00047F8286C4F45F4D184F85884A4F85A6401
:10220000A4F85C64A4F85E6484F86064A4F8626472
:10221000A4F86464A4F8666484F86864B8F1000FF4
:1022200002D0054800F0FEFE044B2846EB62BDE8F4
:10223000F88F00BF307200081472000800A0004040
:10224000044B10B5197804464A1C1A70FFF79AFF20
:10225000204610BDFD4900202DE9F04700295FD040
:10226000304F3148B7FBF1F581428CBF0A20112075
:10227000431EB5FBF0FC00FB1C50DCB220B1022B6E
:102280001846F5D8002037E00CF1FF35B5F5806F22
:1022900032D2C4EBC4094FF47A7009F103034FEA58
:1022A000E308C3F3C70308F1010AA4EB030E08FB1C
:1022B00000085FFA8EF65AFA8EFEB8FBFEFEBEF5F7
:1022C000617F1BDC1FFA8EF4581C56FA80F00CFB61
:1022D00000FCB7FBFCFC6145D4D1013BDBB20F2B0A
:1022E000D0D8711E0020C9B2072905D8107101206D
:1022F0001480558053719171BDE8F08709F1FF3367
:102300004FEAE30EC3F3C7030EF10108E41A0EFB14
:102310000000E6B258FA84F4B0FBF4F4A4B2D3E7B8
:102320000846E9E700B4C4043F420F0038B540F264
:102330007772C36A154CC3F8BC200722C36AC3F87E
:10234000C8202268C16A930043F4C023C1F8A030BA
:1023500002F1805302F16C01C56A03F52C53EA3295
:1023600089009B00226041F0E061094AC361C5F821
:10237000C01003F5D87103F56A734162934283621A
:1023800002D9044800F04EFE38BD00BF004A0020CC
:10239000FCB50040F07100082DE9F04F00F58055C4
:1023A000994689B0044695F858348A469046012BE0
:1023B00004D90027384609B0BDE8F08F974A52F893
:1023C000231009B942F823009549C4F80CA00B78F2
:1023D00084F81090C3B9FFF723FC924BD3F8EC209C
:1023E00042F48072C3F8EC20D3F8942042F4807257
:1023F000C3F89420D3F8942022F48072C3F8942078
:1024000001230B70FFF712FC95F8513473B90321C7
:102410001320FFF705FC01F033FF0321152001F025
:102420002FFF012385F85134FFF700FCFFF7F8FB7D
:10243000E26A936923F01003936100F0F9FD074607
:10244000E36A9E6916F0080607D000F0F1FDC31B91
:10245000FA2BF5D9FFF7EAFBABE79A6942F00102E4
:102460009A6100F0E5FD0746E36A9A69D00705D452
:1024700000F0DEFDC31BFA2BF6D9EBE79A690027C3
:1024800004F5825B42F002020BF1100B9A61E36AE1
:102490005F65FFF7CBFB686C00F050FC2022002149
:1024A0006846FFF73BFB02A8FFF710FE6A460BEBFE
:1024B00006030DF1180E069794460833BCE8030096
:1024C000F44543F8080C43F8041C6246F4D1DCF8E8
:1024D000000020361860B6F5806F9CF804201A7151
:1024E000DCD1002304F5A252514620461A3285F869
:1024F000503485F85334FFF7AFFE074690B9E26ACF
:10250000936923F00103936100F092FD0546E36AAD
:102510009B69D9077FF54DAF00F08AFD431BFA2B6D
:10252000F5D946E795F85F6495F85E243602C5F85C
:102530006CA4E36A46EA426695F860241643B5F84F
:102540005C2446EA0246DE61B8F1000F29D004F5AA
:10255000A352414620460232FFF77EFE90B9E26A5E
:10256000936923F00103936100F062FD0546E36A7D
:102570009B69DA077FF51DAF00F05AFD431BFA2B6C
:10258000F5D916E795F8683495F867141B01C5F876
:102590007084E26A43EA0123B5F8641443EA014314
:1025A000D360E36A00262046C3F8BC60FFF7BEFE96
:1025B00085F859646FF04042E36AB9F1030F1A6578
:1025C000194AE36A5A654FF00222E36A9A654FF0AE
:1025D000FF32E36AC3F8E0204FF00302E36ADA65F2
:1025E000E26A936943F4407393613FF4E3AEE26AB5
:1025F000936923F00103936100F01AFD0646E36A34
:102600009B69DB0705D500F013FD831BFA2BF6D978
:10261000CFE6012385F85234CCE600BFF84900200C
:10262000FC49002000440258550200022DE9F04FF9
:10263000054689B090469946002700F58056DFF898
:10264000C4A0EB6AD3F8D830FB40D80753D505EBCC
:1026500047124FEA471B02F58352137B08321907D2
:1026600049D4D6F880340133C6F8803413799A06F9
:1026700042BFD6F8A8340133C6F8A83405EB0B03E3
:1026800003F583531A7B42F008021A73D30723D54C
:1026900096F8533403B305F582546846FFF71CFDE2
:1026A00003AB18345C4404F1080C2068083454F877
:1026B000041C1A46644503C21346F6D120686946D5
:1026C00010602846A2889A800123ADF808302B6854
:1026D000CDE90089DB6B9847D6F854345BB1D6F866
:1026E0009C34012150460133C6F89C3496F8583486
:1026F000994000F08DFA0137202FA2D109B0BDE832
:10270000F08F00BF044A00202DE9F04F0F468DB036
:10271000044600F08FFC82468946002F5BD1E36AB5
:10272000D3F8A02012F4FE0F03D100200DB0BDE8B5
:10273000F08FD3F8A420920141BF04F58051D1F865
:1027400094240132C1F89424D3F8A4205606ECD086
:10275000D3F8A450E669C5F305254823E8464FF0B1
:10276000000B03FB05664046FFF7B0FC32685100E2
:102770004ABF22F06043C2F38A4343F00043920011
:1027800048BF43F080430093736813F400131BBFEA
:10279000012304F580528DF80D308DF80D301EBFE9
:1027A000D2F8AC340133C2F8AC34F38803F00F0331
:1027B0008DF80C309DF80C0000F09AFA5FFA8BF35C
:1027C000984225D9F2180CA90BF1010B127A0B448F
:1027D00003F82C2CEEE7012FA7D1E36AD3F8B02041
:1027E00012F4FE0FA1D0D3F8B420950141BF04F537
:1027F0008051D1F894240132C1F89424D3F8B42044
:10280000500692D0D3F8B450266AC5F30525A4E744
:10281000EFB9E36AC3F8A85004A807ADFFF75CFC62
:1028200098E80F0007C52B800023204604A9ADF8C7
:102830001830236804F58054DB6BCDE904A9984770
:1028400058B1D4F88C340133C4F88C346EE7012FBE
:10285000E2D1E36AC3F8B850DEE7D4F8903401203F
:102860000133C4F8903461E7F8B505460F4600F52A
:102870008054012639462846FFF746FF10B184F8F8
:102880005364F7E7D4F854346BB1D4F89C34012185
:1028900005480133C4F89C3494F858349940BDE895
:1028A000F84000F0B5B9F8BD044A0020C36AF0B59D
:1028B0001A6C12F47F0F2BD01B6C00F5805441F280
:1028C00068054FF0010CC4F8A0340023471900EB51
:1028D00043125E012A44117911F0020F15D0490705
:1028E00013D4B959C66A0CFA01F1D6F8CCE011EA52
:1028F0000E0F0AD0C6F8D410117941F004011171FD
:10290000D4F888240132C4F888240133202BDED186
:10291000F0BD000010B5264C264B22680AB340B328
:102920001A6D92050FD54FF400721A6500F082FB04
:1029300050EA01020B4602D0013861F10003024661
:102940002068FFF773FE1B4A136D9B012AD523688D
:102950004FF0007103F580531165012283F859246B
:1029600020E001221A6510221A654FF480521A6580
:1029700010BD196DC80702D4196D490705D5052189
:10298000104619650021FFF76FFF0A4B1A6DD0063C
:1029900002D41A6D510605D5502201211A6520680E
:1029A000FFF762FF2068BDE81040FFF77FBF00BF60
:1029B000F849002000A0004008B5FFF731F9FFF703
:1029C00075FFBDE80840FFF731B90000C36AD3F8CE
:1029D000C00010F07C5005D0D3F8C40080F4001083
:1029E000C0F340507047000000F5805008B5FFF775
:1029F00017F9406C00F0B4F9FFF718F943090CBF60
:102A00000120002008BD000000F5805393F85924F0
:102A100062B1C16A8A6922F001028A61D3F89824FE
:102A20000132C3F89824002283F85924704700002B
:102A30002DE9F74300F5825198460025FFF7F0F89D
:102A4000103141F2680E4FF0010900F5805C00EB97
:102A50004514744423795E071CD4DB061AD58E69AD
:102A6000C36A09FA06F6D3F8CC703E4212D04F681A
:102A700001970F689742019F77EB08070AD2C3F8C6
:102A8000D460237943F004032371DCF884340133E8
:102A9000CCF8843401352031202DD8D103B0BDE8E5
:102AA000F043FFF7C3B80000F8B51E4600230F46F9
:102AB000054613701446FFF797FF80F00100387049
:102AC0001EB12846FFF782FF2070F8BD2DE9F04FB8
:102AD000994685B00B780E468046174601931378C9
:102AE000DDE90EBA029300F0A5FA337804460D46EC
:102AF00013B93B78002B41D022462B464046FFF7C6
:102B000097FFFFF759FFFFF77FFF4B463A463146E5
:102B1000FFF7CAFF33782BB1019B1BB1012005B031
:102B2000BDE8F08F3B7813B1029B002BF6D108F57E
:102B3000805303935C4575EB0A031FD2039BD3F8C4
:102B40005404D8B1BBEB04020368D9686AEB0503EF
:102B500088474B463A4631464046FFF7A5FF337853
:102B600013B1019B002BD9D13B7813B1029B002BF1
:102B7000D4D100F05FFA04460D46DBE70020CEE733
:102B800008B50020FFF7C6FEBDE8084001F04EBBC7
:102B900008B50120FFF7BEFEBDE8084001F046BBC6
:102BA000034A0449134643F8041B5360704700BFAF
:102BB000044A002078720008F0B587B005461F4629
:102BC00016460C98043503681B6998474FF0FF338D
:102BD0000246044601A9284601F0F4FF56EA07031D
:102BE0000DD10021204602F047F8044601A92846ED
:102BF00001F0FCFFB4FA84F0400907B0F0BD0A2EE2
:102C0000314638BF0A21EDE7043002F029B8000050
:102C100008B5302383F31188043002F00DF8002347
:102C200083F3118808BD0000044B11220021013AF2
:102C3000C3E9051103F12003F9D170470C4A0020C4
:102C400013B56C46031D84E8060094E8030083E88E
:102C50000500012002B010BD73B58568019155B122
:102C60001B885B0707D4D0E900369B6B9847019A15
:102C7000C1B23046A847012002B070BDF0B58668E9
:102C800089B005460C465EB1BDF838305B070AD402
:102C9000D0E900379B6B98472246C1B23846B0470F
:102CA000012009B0F0BD0022002301F10806CDE9A2
:102CB000002300230A46ADF8083003AB1068083241
:102CC00052F8041C1C46B24203C42346F6D11068D5
:102CD00020609288A28000F0AFF90423ADF808309C
:102CE0002B68CDE90001DB6B694628469847D7E79A
:102CF000082817D909280CD00A280CD00B280CD08A
:102D00000C280CD00D280CD00E2814BF40203020E9
:102D100070470C207047102070471420704718200F
:102D2000704720207047000010B5037C044613B99B
:102D3000006804F0A5F9204610BD00000023BFF391
:102D40005B8FC360BFF35B8FBFF35B8F8360BFF3A9
:102D50005B8F7047BFF35B8F0068BFF35B8F70477B
:102D600070B505460C30FFF7F5FF044605F108067F
:102D70003046FFF7EFFFA04206D96D683046FFF7F7
:102D8000E9FF2544281A70BD3046FFF7E3FF201AFB
:102D9000F9E7000070B505464068A0B105F10C06E2
:102DA00005F10800FFF7D6FF04463046FFF7D2FFD3
:102DB000844204F1FF34304694BF6D680025FFF76C
:102DC000C9FF2C44201A70BD38B50C460546FFF7E4
:102DD000C7FFA04210D305F10800FFF7BBFF044472
:102DE0006868BFF35B8FB4FBF0F100FB1144012076
:102DF000AC60BFF35B8F38BD0020FCE72DE9F041EC
:102E0000144607460D46FFF7C5FF844228BF044617
:102E1000D4B1B84658F80C6B4046FFF79BFF3044DE
:102E2000286040467E68FFF795FF331A9C4203D81E
:102E300001206C60BDE8F081A41B6B603B682044FE
:102E4000AB60E8600220F5E72046F3E738B50C46B2
:102E50000546FFF79FFFA04210D305F10C00FFF7D6
:102E600079FF04446868BFF35B8FB4FBF0F100FBAB
:102E700011440120EC60BFF35B8F38BD0020FCE7FC
:102E80002DE9FF418846694607466C46FFF7B6FFC5
:102E9000002506B204EBC606B4420AD0626808EB0D
:102EA000050120680834FEF713FE54F8043C1D4465
:102EB000F2E729463846FFF7C9FF284604B0BDE8C7
:102EC000F0810000F8B505460C300F46FFF742FFD1
:102ED00005F1080604463046FFF73CFFA0423046A5
:102EE00088BF6C68FFF736FF201A386020B12C6865
:102EF0003046FFF72FFF2044F8BD000073B514469D
:102F000006460D46FFF72CFF8442019028BF044679
:102F1000DCB101A93046FFF7D5FF019B33B9326818
:102F2000C5E90233C5E9002401200CE09C42286079
:102F300038BF0194019884426860F5D93368241A37
:102F40000220AB60EC6002B070BD2046FBE70000E1
:102F50002DE9FF410F4669466C46FFF7CFFF00B2EF
:102F6000002604EBC005AC4209D0D4F80480B8199F
:102F700054F8081B42464644FEF7AAFDF3E73046E4
:102F800004B0BDE8F081000038B50546FFF7E0FF6A
:102F9000044601462846FFF717FF204638BD0000CB
:102FA00000B59BB0EFF3098168226846FEF790FDFB
:102FB000EFF30583044B9A6BDA6A9A6A9A6A9A6A03
:102FC0009A6A9A6A9B6AFEE700ED00E000B59BB042
:102FD000EFF3098168226846FEF77AFDEFF3058377
:102FE000044B9A6B9A6A9A6A9A6A9A6A9A6A9B6A74
:102FF000FEE700BF00ED00E000B59BB0EFF30981F4
:1030000068226846FEF764FDEFF30583034B5A6BB5
:103010009A6A9A6A9A6A9A6A9B6AFEE700ED00E0E9
:10302000FEE700000FB408B5029801F01FFFFEE7AD
:1030300002F038BC02F010BC02F00EBC2DE9F047E3
:103040000D46044600219046284640F27912FEF7CC
:1030500065FD234620220021284604F1220700F0C6
:103060003BFE231D022220212846C02600F034FE0C
:10307000631D03222221284600F02EFEA31D0322F9
:103080002521284600F028FE04F1080310222821FB
:10309000284600F021FE04F11003082238212846BA
:1030A00000F01AFE04F1110308224021284600F026
:1030B00013FE04F1120308224821284600F00CFEFA
:1030C00004F1140320225021284600F005FE04F1EB
:1030D000180340227021284600F0FEFD04F1200371
:1030E0000822B021284600F0F7FD04F12103082250
:1030F000B821284600F0F0FD314608363B4608224C
:103100002846013700F0E8FDB6F5A07FF4D100278E
:1031100004F1330A04F1320308223146284600F054
:10312000DBFD94F832304FEAC7099F4209F5A476D7
:1031300015D3B8F1000F08D1314609F24F1604F546
:1031400099730722284600F0C7FD27463B1B94F8D9
:10315000322193420CD3F01DC008BDE8F0870AEB82
:103160000703082231462846013700F0B5FDD8E7AD
:1031700007F233133146082228460836013700F09B
:10318000ABFDE3E713B504460846002120222346A1
:1031900001900160C0F8031000F09EFD231D01980E
:1031A0000222202100F098FD631D019803222221B4
:1031B00000F092FDA31D01980322252100F08CFD53
:1031C000019804F108031022282100F085FD072052
:1031D00002B010BDF8B50E46054614460021812206
:1031E0003046FEF79BFC2B4608220021304600F0BB
:1031F00073FD7CB90F246B1C07220821304600F0B8
:103200006BFD01235F1C6A78013B934204D3E01DF0
:10321000C008F8BD0824F4E7EB192146082230461F
:1032200000F05AFD08343B46ECE7000030B50A4494
:10323000084D91420DD011F8013B5840082340F34E
:103240000004013B2C4013F0FF0384EA5000F6D148
:10325000EFE730BD2083B8ED384A73B510686B4690
:1032600051686A4603C308233549364803F020FFF6
:10327000044670B9344A6B46106851686A4603C305
:10328000082332492F4803F013FF044630BB0A20BD
:1032900022E00369B3F5E01FECD8418B40F20D4208
:1032A0009142E7D12A4A024402F110018B42E1D354
:1032B000103B244900209D1AFFF7B8FF04F11801C4
:1032C00006462A460020FFF7B1FFA3689E42D1D1EF
:1032D000E3689842CED1002002B070BD0369B3F517
:1032E000E01F22D8B0F8661040F20D4291421ED184
:1032F000174A024402F15C018B421AD35C3B11492C
:1033000000209D1AFFF792FF04F1640106462A4649
:103310000020FFF78BFFA268034696420BD1E068BE
:10332000834214BF0D200020D6E70B20D4E70C20E9
:10333000D2E71020D0E70D20CEE700BF847200084E
:10334000DCFF1B00000004088D72000890FF1B00CA
:103350000800FCF72DE9F041C56915B9C161BDE868
:10336000F0814B68AC4623F06047C3F38A464FEACE
:10337000D37EC3F3807816EA230638BF3E462B4639
:103380005A68BEEBD27F22F060440AD0002A18DAD5
:10339000A40CB44217D19D420FD10D60DEE7134655
:1033A000EEE7A74207D102F08044C2F380724245A3
:1033B0000BD054B1EFE708D2EDE7CCF800100B606A
:1033C000CDE7B44201D0B442E5D81A689C46002A41
:1033D000E5D11960C3E700002DE9F047089D01F031
:1033E000070400EBD1004FF47F494FEAD50822448F
:1033F00005F00705944201D1BDE8F08704F0070706
:1034000005F0070A111B08EBD50E57453E4613F889
:103410000EC038BF5646C6F108068E4228BF0E467B
:10342000E108415C34443544B94029FA06F721FAF1
:103430000AF1FFB28CEA010147FA0AF739408CEA37
:10344000010C03F80EC0D5E780EA0120082341F201
:10345000210201B2013B4000002980B2B8BF5040B8
:1034600013F0FF03F5D1704738B50C468D18A5420F
:1034700000D138BD14F8011BFFF7E6FFF7E70000A5
:1034800002684AB1136801890360C38801339BB2A3
:103490009942C38038BF03811046704770B588B029
:1034A000044620220D4668460021FEF737FB2046E1
:1034B0000495FFF7E5FF024660B16B46054608AE8E
:1034C0001C46083503CCB44245F8080C45F8041CEA
:1034D0002346F5D1104608B070BD0000082817D962
:1034E00009280CD00A280CD00B280CD00C280CD0A2
:1034F0000D280CD00E2814BF4020302070470C201F
:103500007047102070471420704718207047202003
:1035100070470000082817D90C280CD910280CD99E
:1035200014280CD918280CD920280CD930288CBF85
:103530000F200E207047092070470A2070470B208B
:1035400070470C2070470D207047000010B54B6885
:1035500023B9CA8A63F30902CA8210BDC4681A6813
:103560001C60C360438A013B43824A60EFE700006E
:103570002DE9F84F1D46CB8A0F468146C3F309015A
:10358000924605290B4630D00020AAB207F11A0452
:103590009EB21FFA80F8042E0FD8904503F1010364
:1035A00006D30A44FB8A62F309030120FB821AE076
:1035B0001AF800600130E654EAE79045F1D2A1F133
:1035C000050B1C237C68BBFBF3F203FB12BB1FFA49
:1035D0008BF6002C45D14846FFF752FF044638B918
:1035E00078606FF00200BDE8F88F4FF00008E6E762
:1035F000002606607860ADB24FF0000B454510D94B
:103600000AEB0803221D13F8011B08F1010891556C
:10361000B1B21FFA88F81B292BD0454506F10106E7
:10362000F1D8FB8AC3F30902154465F30903BCE72B
:1036300001321C4692B22368002BF9D16B1F0B4458
:103640001C21B3FBF1F301339BB29A42D3D2BBF1FD
:10365000000FD0D14846FFF713FF20B9C4F800B0DF
:10366000BFE70122E7E7C0F800B05E4620600446ED
:10367000C1E74545D5D94846FFF702FF08B92060A4
:10368000AFE7C0F800B0002620600446B6E70000AF
:103690002DE9F04F2DED028B83B007469146BDF822
:1036A0003C50CDE90013002A00F092802DB10E9B12
:1036B000002B00F08D80072D32D807F10C00FFF7AA
:1036C000DFFE044638B96FF00204204603B0BDECBB
:1036D000028BBDE8F08F14220021FEF71FFA2A4664
:1036E0000E9904F10800FEF7F3F9681CC0B2FFF769
:1036F00011FFFFF7F3FE207499F80030013803F052
:103700001F0314FA80F063F03F0303723846009BF6
:1037100043F0004161602146FFF71CFE0124D4E71D
:103720004FF0000800F10C034FF0800A4646444673
:1037300008EE103A18EE100AFFF7A2FE83460028A2
:10374000C1D014220021FEF7E9F9C6BB019B02207B
:10375000ABF808300E9B00F1080299195BFA82F26F
:103760000130C0B2082801D0AE422AD3FFF7D2FE02
:10377000AE4208BF4FF0400AFFF7B0FE99F80020B4
:10378000411E009B02F01F0201345BFA81F142EA04
:10379000481288F0010824B24AEA020A43F00042C3
:1037A00081F808A059468BF810003846CBF8042061
:1037B0004FF0000AFFF7CEFDAE42BBD185E70020F7
:1037C000C8E711F801CB013602F801CBB6B2C7E762
:1037D0006FF0010479E70000F8B515460E4628227F
:1037E000002104461F46FEF799F9069BB5F5001F18
:1037F000A760636004F10C00079B34BF6A094FF6B1
:10380000FF722362002397B29A4205D80023036017
:1038100027826382A382F8BD0660013330462036DA
:10382000F2E7000003781BB94BB2002BC8BF017050
:1038300070470000007870472DE9F74FDDF83C90A5
:10384000804692469B46BDF830500D9E9DF838400C
:10385000BDF84070B9F1000F01D1002F51D11F2CDC
:103860004FD898F80000B0B9072F47D835F00303B8
:1038700047D13A4649464FF6FF702D02FFF7F4FD57
:1038800020F0010045EA04644004400C44EA40246E
:103890004FF6FF7321E040EA0520072F40EA046459
:1038A000F6D900254FF6FF73C5F12000A5F12002DF
:1038B0002AFA05F108350BFA00F02BFA02F201435F
:1038C00018461143C9B2FFF7BFFD402D0346EBD1A7
:1038D0003A464946FFF7C8FD034632462146404670
:1038E000CDE90097FFF7D4FE33780133DBB21F2B0D
:1038F00088BF0023337003B0BDE8F08F6FF0030082
:10390000F9E76FF00100F6E72DE9F04F85B0924638
:1039100006469B46DDF848800F9D9DF840209DF8A7
:103920004490BDF84C70B8F1000F01D1002F49D17F
:103930001F2A47D83378002B47D00C029DF8381047
:10394000072F44EA026444EAC93444EA014444EAE1
:10395000030444F0800432D900234FF6FF72C3F110
:10396000200CA3F120002AFA03F103930BFA0CFCBC
:103970002BFA00F041EA0C0101431046C9B2FFF7EF
:1039800063FD039B02460833402BE8D13A4641468B
:10399000FFF76AFD03462A4621463046CDE90087F7
:1039A000FFF776FEB9F1010F06D12B780133DBB2B8
:1039B0001F2B88BF00232B7005B0BDE8F08F4FF69A
:1039C000FF73E8E76FF00100F6E76FF00300F3E73D
:1039D000C06900B104307047C3691A68C261C26827
:1039E0001A60C360438A013B438270472DE9F0416E
:1039F000D0F8188014461D46184E4146002709B9D4
:103A0000BDE8F081D1E90223A21A65EB03039642D7
:103A100077EB03031ED283698B420DD1FFF796FD2E
:103A200083691B688361C3680B60438AC160013B83
:103A3000816943828846E2E7FFF788FD0B68C8F892
:103A40000030C3680B60438AC160013B4382D8F8F1
:103A50000010D4E788460968D1E700BF80841E00C3
:103A60002DE9F04F8BB00D4614469B46DDF8509083
:103A70008046002800F01881B9F1000F00F0148191
:103A8000531E3F2B00F21081012A03D1BBF1000F1E
:103A900040F00A810023CDE90833B8F81430B5EBC3
:103AA000C30F4FEAC30703D300200BB0BDE8F08F6C
:103AB0002B199F42D8F80C3036BF7F1B2746FFB228
:103AC0001BB9D8F81030002B7AD0272D4DD8C5F16E
:103AD000280600232946B742009308ABD8F808000F
:103AE0002CBFF6B23E46A7EB060A354432465FFAD3
:103AF0008AFAFFF771FCB8F81430282103F100535B
:103B0000053BDB000493D8F80C300393039B13B1FF
:103B1000BAF1000F2CD1D8F8100040B1BAF1000F63
:103B200005D008AB5246691A0096FFF755FC38B22B
:103B3000002FB9D066070AD00AAB624203EBD4016A
:103B400002F0070211F8083C134101F8083C082C68
:103B50003DD9102C40F2B580202C40F2B780BBF14B
:103B6000000F00F09C80082335E0BA460026C2E72B
:103B7000049BE02B28BFE02306930B44AB42059344
:103B800015D95A1B0398691A0096924508AB00F1A3
:103B9000040034BF5246D2B20792FFF71DFC079AC9
:103BA0001644AAEB020A1544F6B25FFA8AFA049B9D
:103BB000069A05999B1A0493039B1B680393A5E738
:103BC00000933A4608AB2946D8F80800ADE7BBF1A8
:103BD000000F13D00123B4EBC30F6BD0082C12D805
:103BE0009DF82030621E23FA02F2D50706D54FF069
:103BF000FF3202FA04F423438DF820309DF8203080
:103C000089F8003051E7102C12D8BDF82030621E20
:103C100023FA02F2D10706D54FF0FF3202FA04F47C
:103C20002343ADF82030BDF82030A9F800303CE740
:103C3000202C0FD80899631E21FA03F3DA0705D563
:103C40004FF0FF3202FA04F40C430894089BC9F8C1
:103C500000302AE7402C2AD0611EC4F12102A4F1D1
:103C60002103DDE9086526FA01F105FA02F225FAD9
:103C700003F311431943CB0711D50122A4F120030B
:103C8000C4F1200102FA03F322FA01F1A2400B432E
:103C9000524263EB430332432B43CDE90823DDE972
:103CA0000823C9E9002300E76FF00100FDE66FF08B
:103CB0000800FAE6082CA1D9102CB4D9202CEED893
:103CC000C4E7BBF1000FAED0022384E7BBF1000FC5
:103CD000BCD004237FE70000012A30B5144638BF6A
:103CE000012485B00025402C28BF4024012ACDE9BD
:103CF000025518D81B788DF8083063070AD004AB3A
:103D0000624203EBD40502F0070215F8083C934029
:103D100005F8083C034600912246002102A8FFF75F
:103D20005BFB05B030BD082AE4D9102A03D81B88F4
:103D3000ADF80830E1E7202A95BF1B68D3E90023DE
:103D40000293CDE90223D8E710B5CB681BB98B608D
:103D50000B618B8210BDC4681A681C60C360438A03
:103D6000013B4382CA60F0E72DE9F04F95B004466D
:103D70000D46CDE904230B681806C3F3C01147BFF5
:103D8000C3F3C03BC3F306264FF0020B0E46002BD5
:103D900080F2018213F0C04940F0FD812A7B002AA5
:103DA00000F0F981BBF1020F03D02078B04240F05F
:103DB000F581C3F30460089003F07F00069059B3C7
:103DC000C3F3074A7606069B2A4446EA0B4692F856
:103DD0000380002246EA83460023CDE90A235FEAF6
:103DE000D81346EA0A0603936AD0069B52460AA9EC
:103DF000204600935B466768B847002800F0D181F1
:103E0000A76987B9314604F10C00FFF747FB074665
:103E1000C8B96FF0020057E0C3F30F2A590608BF74
:103E20000AF0030ACEE73B699E420DD03F68002F9F
:103E3000F9D1314604F10C00FFF730FB07460028AA
:103E4000E7D0A3693B60A761FE7D08F01F03C6F3BE
:103E500084060793F01A9B1B1FFA80FC0028B8BF4A
:103E60000CF120001FFA83FCB8BF00B2002B0993AD
:103E7000B8BF0CF12003D7E90221BCBF1BB20993E4
:103E800052EA010335D0049EDFF8D4C2B21A059E6F
:103E900066EB01010026944576EB010329D395F8E2
:103EA0000DE097F81AC0E64516D1039B002B78D099
:103EB00001281EDCA948904276EB010316D338E0B6
:103EC000A76927B96FF00C0015B0BDE8F08F3B690A
:103ED0009E42B9D03F68F4E7A048904276EB0103D8
:103EE00001D30020F0E7039B002BFAD0099B0F2B96
:103EF00018DCFA7D4FEA88033946204602F00302B7
:103F000003F07C031343FB75FFF720FB6B7BBB7651
:103F1000039B3BB9FB7DC3F38402013262F386034A
:103F2000FB75CFE76A7BBB7E9A42DAD1039B002BFD
:103F300037D04FEA9813022B33D0049B1422002170
:103F40000FA8BB60059BFB60FDF7E8FD049B0CA977
:103F500020460C93059BADF846A00D932B1D8DF8C4
:103F600048B00E932B7B013BDBB2ADF84430079B8E
:103F70008DF84930089B8DF84A30069B8DF84B3000
:103F800094F8243083F001038DF84C30A3689847EF
:103F9000FB7DC3F38403013303F01F039B02FB8209
:103FA0009FE7FB7DC8F34012B2EBD31F40F0FC80CB
:103FB000C3F38403079A934240F0F98003994FEAD0
:103FC00098122B7B00294DD0D2075DD4032B40F2F1
:103FD000F180049BAE1D394604F10C00BB603246F3
:103FE000059BFB602B7B033BDBB2FFF7C1FA00288C
:103FF0000CDA39462046FFF7A9FAFB7DC3F38403A8
:10400000013303F01F039B02FB8202E7AB88DDE96B
:104010000A843B834FF6FF73C9F12000A9F1200207
:1040200028FA09F109F1080904FA00F024FA02F269
:10403000014318461143C9B2FFF706FAB9F1400F20
:104040000346E9D1B88231462A7B033AD2B2FFF760
:104050000BFAFB7DB882DA43C2F3C01262F3C713D6
:10406000FB753EE782B92E1D013B394604F10C0079
:10407000DBB23246FFF77CFA0028BADB2A7B3146F6
:10408000B88A013AD2B2E2E7F98A013BC1F30901E9
:10409000DAB204295CD8281D002307F11B069A42D6
:1040A00008D910F801CB013306F801C00131DBB2A9
:1040B0000529F4D1049993420C9138BF0433059932
:1040C0002CBF002355FA83F30D9107F11B010E91CC
:1040D000796810930F91291DFB8AADF846A0C3F3B0
:1040E00009038DF848B01A44079B8DF84930089BA6
:1040F000ADF844208DF84A30069B8DF84B3094F88B
:10410000243083F001038DF84C300023B88A7B60A3
:104110002A7B013AFFF7A8F93B8BB882834203D18F
:10412000A3680CA92046984720460CA9FFF70CFE6F
:10413000FB7DBA8AC3F38403013303F01F039B02A0
:10414000FB823B8B9A420CBF00206FF01000BBE655
:104150007B68002BAED0052006E000BF40420F0078
:1041600080841E001C3033461E68002EFAD1091AC6
:104170002E1D081D184401EB090C5FFA89F3BCF1F0
:104180001B0F97D89A4295D916F8013B09F10109FE
:1041900000F8013BEFE76FF0090095E66FF00A00C9
:1041A00092E66FF00B008FE66FF00D008CE66FF07B
:1041B0000E0089E66FF00F0086E600BFEFF309837B
:1041C000054968334A6B22F001024A6383F3098888
:1041D000002383F31188704700EF00E0302080F364
:1041E000118862B60D4B0E4AD96821F4E0610904CA
:1041F000090C0A430B49DA60D3F8FC2042F08072C4
:10420000C3F8FC20084AC2F8B01F116841F0010150
:1042100011602022DA7783F82200704700ED00E079
:104220000003FA0555CEACC5001000E0302310B5F0
:1042300083F311880E4B5B6813F4006314D0F1EE26
:10424000103AEFF309844FF08073683CE361094B47
:10425000DB6B236684F3098800F0ACFD10B1064BDC
:10426000A36110BD054BFBE783F31188F9E700BF9D
:1042700000ED00E000EF00E0470700084A070008F3
:10428000090100F16043012203F56143C9B283F8DB
:10429000001300F01F039A4043099B0003F16043A1
:1042A00003F56143C3F880211A60704713B5406B72
:1042B00000F58054D4F89C381A681178042914D178
:1042C000017A022911D11979012312898B401342F5
:1042D0000BD101A9443002F01DFAD4F89C480246E3
:1042E000019B2179206800F0F7F902B010BD0000B1
:1042F0000C3002F09FB900004FF0FF330C3002F099
:1043000099B90000443002F071BA00004FF0FF3359
:10431000443002F06BBA00000C3002F06DB90000BE
:104320004FF0FF310C3002F067B90000443002F06A
:104330003DBA00004FF0FF32443002F037BA0000BF
:104340000020704710B500F58054D4F89C381A68E6
:104350001178042917D1017A022914D1597901233E
:1043600052898B4013420ED10C3002F0FFF8024606
:1043700048B1D4F89C484FF4407361792068BDE897
:10438000104000F097B910BD406BFFF7DBBF000095
:10439000704700007FB50346114A0125042643F803
:1043A000042B0446436000F17C020E4B2946057243
:1043B00002900C3001934FF44073009602F0B2F873
:1043C000094B04F68C42294604F144000294CDE9DD
:1043D00000634FF4407302F079F904B070BD00BF80
:1043E0009872000889430008AD4200080A6830232B
:1043F00083F311880B790B3342F823004B79133385
:1044000042F823008B7913B10B3342F8230000F5F7
:104410008053C3F89C1802230372002080F3118894
:104420007047000038B5037D044613B190F84C3056
:10443000ABB90125201D022100F0FEFB04F10C00A8
:104440006FF00101257500F0E1FD04F1440084F8EE
:104450004C506FF00101BDE8384000F0D7BD38BDC9
:1044600010B501210446043000F0E6FB002323755B
:1044700084F84C3010BD000038B5044600250C30DF
:1044800002F068F804F14400257502F037F9201DA8
:1044900084F84C50012100F0CFFB2046BDE83840A5
:1044A000FFF750BF90F8803003F06003202B06D157
:1044B00090F881200023212A03D81F2A06D8002043
:1044C0007047222AFBD1C0E91D3303E0034A42674B
:1044D00007228267C3670120704700BF3422002093
:1044E00037B500F58055D5F89C381A68117804293D
:1044F0001AD1017A022917D11979012312898B4027
:10450000134211D100F14404204602F0B7F958B12A
:1045100001A9204602F0FEF8D5F89C480246019B0E
:104520002179206800F0D8F803B030BD01F10B0309
:10453000F0B550F8236085B004460D46FEB1302337
:1045400083F3118804EB8507301D082100F074FB0C
:10455000FB6806F144005B691B681BB1019002F027
:10456000E7F8019803A902F0D5F8024648B1039B89
:104570002946204600F0B0F8002383F3118805B0E7
:10458000F0BDFB685A691268002AF5D01B8A013B0E
:104590001340F1D104F18002EAE70000133138B58D
:1045A00050F82140ECB1302383F3118804F5805397
:1045B000D3F89C281368527903EB8203DB689B696C
:1045C0005D6845B10421601800F036FB294604F10E
:1045D0000C0001F0D5FF2046FFF7B4FE002383F363
:1045E000118838BD7047000001F0BCBA0123402299
:1045F000002110B5044600F8303BFDF78FFA002388
:10460000C4E9013310BD000010B53023044683F324
:1046100011882422416000210C30FDF77FFA2046EA
:1046200001F0B2FA02230020237080F3118810BD3C
:1046300070B500EB8103054650690E461446DA60FA
:1046400018B114220021FDF769FAA06918B11422EB
:104650000021FDF763FA31462846BDE8704001F0BD
:1046600077BB0000F8B58368044600F1100500F13F
:10467000300603F001130027836055F8043B7BB13B
:10468000586920B16FF001010C3000F099FC55F829
:10469000043C986920B16FF001010C3000F090FCEF
:1046A000B54245F8047CE8D12046BDE8F84001F069
:1046B000DBBB0000F0B4012500EB81044789E4680E
:1046C0008D40A4693D43458123600023A26063605F
:1046D000E360F0BC01F0F6BBF0B4012500EB81040F
:1046E0000789E4688D4064693D43058123600023A8
:1046F000A2606360E360F0BC01F07CBC2DE9F04196
:1047000002230026044600F10C0500F130074FF0AB
:1047100030080370C0F88860866055F8043BABB180
:1047200088F3118855F8043C586920B16FF00101F5
:104730000C3000F045FC55F8043C986920B16FF04E
:1047400001010C3000F03CFC86F31188BD4245F8B5
:10475000046CE2D1204684F8706001F08DFA636841
:104760001B6823B120460021BDE8F0411847BDE891
:10477000F0810000F8B50378044680F88C300523FA
:10478000037043681B680BB104219847002604F1AD
:104790000C053027303444F8286C55F8043BABB195
:1047A00087F3118855F8043C586920B16FF0010176
:1047B0000C3000F005FC55F8043C986920B16FF00E
:1047C00001010C3000F0FCFB86F31188A542E4D116
:1047D000F8BD000090F88C20436802701B680BB194
:1047E000052118477047000070B590F870300446F6
:1047F00013B1002380F8703004F18002204601F0EC
:1048000057FB63689B68B3B994F8803013F0600578
:1048100035D00021204601F061FE0021204601F044
:1048200051FE63681B6813B1062120469847062392
:1048300084F8703070BD204698470028E4D0B4F862
:104840008630A26F9A4288BFA36794F98030A56F23
:10485000002B4FF0300380F20381002D00F0F28036
:10486000092284F8702083F3118800212046D4E9BE
:104870001D23FFF731FF002383F31188DAE794F853
:10488000812003F07F0343EA022340F20232934285
:1048900000F0C58021D8B3F5807F48D00DD8012B1A
:1048A0003FD0022B00F09380002BB2D104F188029C
:1048B00062670222A267E367C1E7B3F5817F00F078
:1048C0009B80B3F5407FA4D194F88230012BA0D116
:1048D000B4F8883043F0020332E0B3F5006F4DD0F6
:1048E00017D8B3F5A06F31D0A3F5C063012B90D8D2
:1048F0006368204694F882205E6894F88310B4F8C8
:104900008430B047002884D0436863670368A36796
:104910001AE0B3F5106F36D040F6024293427FF4AE
:1049200078AF5C4B63670223A3670023C3E794F867
:104930008230012B7FF46DAFB4F8883023F002038E
:10494000A4F88830C4E91D55E56778E7B4F88030ED
:10495000B3F5A06F0ED194F88230204684F88A30E7
:1049600001F0E8F963681B6813B1012120469847FC
:10497000032323700023C4E91D339CE704F18B0358
:1049800063670123C3E72378042B10D1302383F31B
:1049900011882046FFF766FE85F3118803216368BE
:1049A00084F88B5021701B680BB12046984794F80F
:1049B0008230002BDED084F88B30042323706368B0
:1049C0001B68002BD6D0022120469847D2E794F8E6
:1049D000843020461D0603F00F010AD501F05AFA73
:1049E000012804D002287FF414AF2B4B9AE72B4BFD
:1049F00098E701F041FAF3E794F88230002B7FF456
:104A000008AF94F8843013F00F01B3D01A06204693
:104A100002D501F07BFDADE701F06CFDAAE794F84B
:104A20008230002B7FF4F5AE94F8843013F00F0140
:104A3000A0D01B06204602D501F050FD9AE701F0F8
:104A400041FD97E7142284F8702083F311882B46E8
:104A50002A4629462046FFF72DFE85F31188E9E610
:104A60005DB1152284F8702083F31188002120465F
:104A7000D4E91D23FFF71EFEFDE60B2284F870200B
:104A800083F311882B462A4629462046FFF724FE49
:104A9000E3E700BFC8720008C0720008C4720008D3
:104AA00038B590F870300446002B3ED0063BDAB2A1
:104AB0000F2A34D80F2B32D8DFE803F03731310812
:104AC000223231313131313131313737856FB0F800
:104AD00086309D4214D2C3681B8AB5FBF3F203FBF8
:104AE00012556DB9302383F311882B462A46294687
:104AF000FFF7F2FD85F311880A2384F870300EE089
:104B0000142384F87030302383F311880023204667
:104B10001A461946FFF7CEFD002383F3118838BDEE
:104B2000C36F03B198470023E7E70021204601F057
:104B3000D5FC0021204601F0C5FC63681B6813B159
:104B40000621204698470623D7E7000010B590F8C5
:104B500070300446142B29D017D8062B05D001D865
:104B60001BB110BD093B022BFBD80021204601F0F0
:104B7000B5FC0021204601F0A5FC63681B6813B159
:104B8000062120469847062319E0152BE9D10B236F
:104B900080F87030302383F3118800231A461946B9
:104BA000FFF79AFD002383F31188DAE7C3689B6956
:104BB0005B68002BD5D1C36F03B19847002384F8FD
:104BC0007030CEE730B5302484F31188064C056888
:104BD000E4680D600160C1E901420022C1E90323DC
:104BE00082F3118830BD00BF304C0020302383F3A6
:104BF000118803461A461B68984203D08B42F9D1AC
:104C00001B681360002383F311887047036B1943FB
:104C100090F824300A2B016303D1836A194205D12D
:104C200070470B2B06D1836A8B4303D10023836229
:104C300000F082B87047000070B506460D46046863
:104C4000B44200D170BDE3682B43E36015B1236922
:104C50001D4203D0D4E90101FFF7D8FF2468EFE734
:104C600008B5302383F31188FFF7E6FF00F0CCF896
:104C7000002383F3118808BD0F4A70B5D668054636
:104C8000302282F31188346B04400CD119B984F3BB
:104C90001188204670BDB0620A2000F06DF800282F
:104CA000F5DB346B2C40336B23EA040333630023BE
:104CB00083F31188EDE700BF304C002000238268A9
:104CC00080F8243083691B6899689142FBD25A6846
:104CD00003604260106058607047000000238268E3
:104CE00080F8243083691B6899689142FBD85A6820
:104CF00003604260106058607047000008B50846C5
:104D0000302383F3118891F82430032B05D0042B32
:104D10000DD02BB983F3118808BD8B6A00221A606D
:104D20004FF0FF338362FFF7C9FF0023F2E7D1E9B9
:104D3000003213605A60F3E7FFF7C0BF38B50D4B80
:104D40001C68DD6885F82400226853601A6001221F
:104D5000DC6084F82420EFF30983643B2A6A9A42DA
:104D600002D9284600F03CFE29462046BDE83840DE
:104D7000FBF7D4BC304C00200C4B30B5DD684B1C2D
:104D800087B004460FD02B46094A684600F004FA63
:104D90002046FFF7D3FF009B13B1684600F006FAE8
:104DA000A86A07B030BDFFF7C9FFF9E7304C002013
:104DB000FD4C0008044B1A68DB6890689B689842B9
:104DC00094BF002001207047304C002038B50D4BB7
:104DD0001C68D868226853601A600122DC6084F87D
:104DE0002420FFF77BFF0546EFF30983643B026A4B
:104DF0009A4201D900F0F4FD29462046BDE838402A
:104E0000FBF78CBC304C0020044B1A68DB689268BE
:104E10009B689A4201D9FFF7D9BF7047304C0020F8
:104E200030B501230E4C87B004252370002368465B
:104E3000C4E9013300F0F8F8684600F001F968466B
:104E400000F004F9013DF7D1009B06490648A36034
:104E500001F052FD0223237085F3118807B030BDA5
:104E6000E04E0020D0720008304C002008B572B629
:104E7000044B986700F0E2FC00F0B0FD024B032207
:104E80001A70FEE7304C0020E04E002000F0C4B95C
:104E9000EFF3118020B9EFF30583302282F31188FC
:104EA0007047000010B530B9EFF30584C4F308046F
:104EB00014B180F3118810BDFFF7A6FF84F31188A9
:104EC000F9E70000034A516853685B1A9842FBD81F
:104ED000704700BF001000E08B608B630023CA6145
:104EE00000F1280288610A61C1E90C3302238B8436
:104EF000012381F8263001F11003C26A4A61136070
:104F0000C36201F12C030846CB62704703460A1ABC
:104F100001338B4288BF01225521FCF7FFBD000001
:104F2000D0E90131026841F8203CA1F1A4034039E5
:104F3000CB60036941F8243C436941F8203C034BB2
:104F400041F8043CC3680248FFF7C6BF35070008B4
:104F5000304C002008B5FFF7E3FFBDE80840FFF73D
:104F6000EBBE000038B50C4BDC6804F12C05A062E8
:104F7000E06AA8420BD194F826301BB9D4E9043278
:104F800013605A600F20BDE83840FFF7D7BE0368B2
:104F9000E362FFF7D1FEEBE7304C0020302383F3D0
:104FA0001188FFF7DFBF000008B50146302383F307
:104FB00011880820FFF7E0FE002383F3118808BD65
:104FC00003682BB10022026018469962FFF7B4BE55
:104FD00070470000064BDB6839B1426818605A60C0
:104FE000136043600420FFF7C7BE4FF0FF307047E7
:104FF000304C00200368984206D01A680260506066
:1050000018469962FFF798BE7047000038B504460D
:105010000D462068844200D138BD036823605C607F
:105020008562FFF789FEF4E700234FF0FF32C0E905
:105030000233C0E9002300220023C0E904237047A3
:10504000014B5B6883607047001000E00D4A0E4B17
:105050009168C2685B6801325B1AC26082689B1A01
:10506000D0E904218360D21841F10001C0E9042194
:1050700042689342026888BF4360934238BF03602E
:10508000704700BFE04E0020001000E0036810B53C
:105090009C68A2420CD85C688A600B604C602160FE
:1050A000596099688A1A9A604FF0FF33836010BD87
:1050B000121B1B68ECE700000A2938BF0A2170B5F3
:1050C00004460D460A26601901F00EFC01F0F6FBBD
:1050D000041BA54203D8751C04462E46F3E70A2E8E
:1050E00004D90120BDE8704001F04EBC70BD000045
:1050F000F8B5144B0D460A2A4FF00A07D96103F19F
:105100001001826038BF0A224160196914460160AB
:1051100048601861A81801F0D7FB01F0CFFB431BD2
:105120000646A34206D37C1C28192746354601F0C3
:10513000DBFBF2E70A2F04D90120BDE8F84001F0BB
:1051400023BCF8BD304C0020F8B506460D4601F0F2
:10515000B5FB0F4A134653F8107F9F4206D12A46EB
:1051600001463046BDE8F840FFF7C2BFD169BB68D1
:10517000441A2C1928BF2C46A34202D92946FFF70E
:105180009BFF224631460348BDE8F840FFF77EBF4B
:10519000304C0020404C0020C0E90323002310B411
:1051A0005DF8044B4361FFF7CFBF000010B5194C09
:1051B000236998420DD08168D0E9003213605A60AB
:1051C0009A680A449A60002303604FF0FF33A3619A
:1051D00010BD0268234643F8102F5360002202607E
:1051E00022699A4203D1BDE8104001F077BB936871
:1051F00081680B44936001F061FB2269E169926868
:10520000441AA242E4D91144BDE81040091AFFF73C
:1052100053BF00BF304C00202DE9F047DFF8BC80C1
:1052200008F110072C4ED8F8105001F047FBD8F8C1
:105230001C40AA68031B9A423ED814444FF0000950
:10524000D5E90032C8F81C4013605A60C5F80090D8
:10525000D8F81030B34201D101F040FB89F3118836
:10526000D5E9033128469847302383F311886B69C9
:10527000002BD8D001F022FB6A69A0EB040982461A
:105280004A450DD2022001F07FFB0022D8F81030F1
:10529000B34208D151462846BDE8F047FFF728BF82
:1052A000121A2244F2E712EB09092946384638BFA0
:1052B0004A46FFF7EBFEB5E7D8F81030B34208D006
:1052C0001444C8F81C00211AA960BDE8F047FFF794
:1052D000F3BEBDE8F08700BF404C0020304C0020FA
:1052E00000207047FEE70000704700004FF0FF30DD
:1052F0007047000002290CD0032904D00129074877
:1053000018BF00207047032A05D8054800EBC200EB
:105310007047044870470020704700BFB073000812
:10532000442200206473000870B59AB00546084610
:10533000144601A900F0C2F801A8FCF7E7FB431CE2
:105340000022C6B25B001046C5E900342370032377
:10535000023404F8013C01ABD1B202348E4201D8D0
:105360001AB070BD13F8011B013204F8010C04F8E7
:10537000021CF1E708B5302383F311880348FFF7D7
:10538000AFF8002383F3118808BD00BFEC4E002066
:1053900090F8803003F01F02012A07D190F8812095
:1053A0000B2A03D10023C0E91D3315E003F060038D
:1053B000202B08D1B0F884302BB990F88120212A15
:1053C00003D81F2A04D8FFF76DB8222AEBD0FAE7DA
:1053D000034A426707228267C3670120704700BF04
:1053E0003B22002007B5052917D8DFE801F0191680
:1053F00003191920302383F31188104A01210190E9
:10540000FFF716F9019802210D4AFFF711F90D482F
:10541000FFF732F8002383F3118803B05DF804FB33
:10542000302383F311880748FEF7FCFFF2E73023AF
:1054300083F311880348FFF713F8EBE704730008C0
:1054400028730008EC4E002038B50C4D0C4C2A4651
:105450000C4904F10800FFF767FF05F1CA0204F1E7
:1054600010000949FFF760FF05F5CA7204F1180042
:105470000649BDE83840FFF757BF00BFC8670020A6
:1054800044220020E4720008EE720008F97200085D
:1054900070B5044608460D46FCF738FBC6B22046F8
:1054A000013403780BB9184670BD32462946FCF723
:1054B00019FB0028F3D10120F6E700002DE9F84F91
:1054C00005460C46FCF722FB2B49C6B22846FFF7DF
:1054D000DFFF2A492846FFF7DBFF08B11036F6B296
:1054E000632E0DD8DFF89080DFF89090244FDFF81E
:1054F00098A0DFF898B02E7846B92670BDE8F88FEE
:1055000029462046BDE8F84F01F040BE252E2ED199
:10551000072241462846FCF7E5FA70B9DBF800306F
:105520000735073444F8073CBBF8043024F8033C43
:105530009BF8063004F8013CDDE70822494628467E
:10554000FCF7D0FA98B9A21C0E4B1978023209095F
:10555000C95D02F8041C13F8011B01F00F0153454B
:10556000C95D02F8031CF0D118340835C3E70135D2
:1055700004F8016BBFE700BFD0730008F9720008A0
:10558000E073000800E8F11F0CE8F11FD873000871
:10559000BFF34F8F044B1A695107FCD1D3F8102188
:1055A0005207F8D1704700BF0020005208B50D4BDC
:1055B0001B78ABB9FFF7ECFF0B4BDA68D10704D5CA
:1055C0000A4A5A6002F188325A60D3F80C21D20795
:1055D00006D5064AC3F8042102F18832C3F8042133
:1055E00008BD00BF266A0020002000522301674545
:1055F00008B5114B1B78F3B9104B1A69510703D545
:10560000DA6842F04002DA60D3F81021520705D57B
:10561000D3F80C2142F04002C3F80C21FFF7B8FF89
:10562000064BDA6842F00102DA60D3F80C2142F04E
:105630000102C3F80C2108BD266A00200020005298
:105640000F289ABF00F580604004002070470000DA
:105650004FF4003070470000102070470F2808B545
:105660000BD8FFF7EDFF00F500330268013204D1DB
:1056700004308342F9D1012008BD0020FCE700007E
:105680000F2870B5054645D8FFF702FC224CFFF7FE
:105690007FFF0646FFF78AFF4FF0FF33072D636158
:1056A000C4F8143120D82361FFF772FF2B0243F0B6
:1056B0002403E360E36843F08003E36023695A074F
:1056C000FCD42846FFF764FF4FF40031FFF7B8FF22
:1056D00000F060F93046FFF78BFFFFF7E3FB284649
:1056E000BDE87040FFF7BABFC4F81031FFF750FFB4
:1056F000A5F108031B0243F02403C4F80C31D4F8CD
:105700000C3143F08003C4F80C31D4F810315B073E
:10571000FBD4D6E7002070BD002000522DE9F84FE1
:1057200040EA020305460C461746D80602D0002080
:10573000BDE8F88F27F01F07DFF8D4B0FFF736FF7A
:105740002744BC4203D10120FFF752FFF0E720229B
:105750002946204601F09CFC10B920352034F0E7A2
:105760002B4605F120021E68711CE0D104339A42D9
:10577000F9D1FFF78DFB05F17843234AB3F5801F7C
:10578000224B28BF9A4603F1040338BF9046A2F18A
:10579000080228BF9846A3F108033ABF9146DA46AB
:1057A0009946FFF7F5FEC8F80060A5EB040CD9F8A0
:1057B000002004F11C0142F00202C9F80020221F5F
:1057C000DAF8006016F00506FAD152F8043F8A4272
:1057D0004CF80230F4D1BFF34F8FFFF7D9FE4FF0F2
:1057E000FF32C8F80020D9F8002022F00202C9F8E0
:1057F0000020FFF757FB20222146284601F048FCF5
:105800000028AAD030469FE71420005210210052F1
:105810001020005210B5084C237828B11BB9FFF7AF
:10582000C5FE0123237010BD002BFCD02070BDE805
:105830001040FFF7DDBE00BF266A002038B5054DD9
:1058400000240334696855F80C0B00F0B5F8122CED
:10585000F7D138BDF473000870B5104E82B0FFF771
:1058600017FB054601F02AF8326803469042336080
:1058700037BF0B4A0A495168146836BF0131D1E974
:10588000004151600419284641F100010191FFF7E0
:1058900009FB2046019902B070BD00BF286A0020B4
:1058A000306A002070B5124E82B0FFF7F1FA05465B
:1058B00001F004F8326803469042336037BF0D4A66
:1058C0000C495168146836BF0131D1E9004151607B
:1058D0000419284641F100010191FFF7E3FA4FF462
:1058E0007A72002320460199FAF702FD02B070BDDA
:1058F000286A0020306A00200244074BD2B210B55B
:10590000904200D110BD441C00B253F8200041F871
:10591000040BE0B2F4E700BF504000580E4B30B526
:105920001C6F240405D41C6F1C671C6F44F40044D6
:105930001C670A4C02442368D2B243F4807323608C
:10594000074B904200D130BD441C51F8045B00B2BB
:1059500043F82050E0B2F4E70044025800480258EF
:105960005040005807B5012201A90020FFF7C4FFED
:10597000019803B05DF804FB13B50446FFF7F2FF8E
:10598000A04205D0012201A900200194FFF7C6FF23
:1059900002B010BD0144BFF34F8F064B884204D3C1
:1059A000BFF34F8FBFF36F8F7047C3F85C02203097
:1059B000F4E700BF00ED00E00144BFF34F8F064B5A
:1059C000884204D3BFF34F8FBFF36F8F7047C3F884
:1059D00070022030F4E700BF00ED00E070470000E7
:1059E0007047000000207047034B1B781BB1034B2E
:1059F0004AF6AA221A6070473C6A00200048005804
:105A0000034B1A681AB9034AD2F8D0241A607047B7
:105A1000386A002000400258024B4FF48032C3F82D
:105A2000D02470470040025808B5FFF7E9FF024B49
:105A30001868C0F3806008BD386A002070B5BFF3F5
:105A40004F8FBFF36F8F1A4A0021C2F85012BFF375
:105A50004F8FBFF36F8F536943F400335361BFF32C
:105A60004F8FBFF36F8FC2F88410BFF34F8FD2F800
:105A7000803043F6E074C3F3C900C3F34E335B01D7
:105A800003EA0406014646EA81750139C2F860520C
:105A9000F9D2203B13F1200FF2D1BFF34F8F53699E
:105AA00043F480335361BFF34F8FBFF36F8F70BDEB
:105AB00000ED00E0FEE700000A4B0B480B4A904265
:105AC0000BD30B4BC11EDA1C121A22F003028B42BD
:105AD00038BF00220021FCF721B853F8041B40F81E
:105AE000041BECE7A8760008806B0020806B002088
:105AF000806B00207047000070B5D0E9244300227D
:105B00004FF0FF359E6804EB42135101D3F80009B2
:105B1000002805DAD3F8000940F08040C3F80009F6
:105B2000D3F8000B002805DAD3F8000B40F08040D2
:105B3000C3F8000B013263189642C3F80859C3F842
:105B4000085BE0D24FF00113C4F81C3870BD0000B0
:105B5000890141F02001016103699B06FCD41220F8
:105B6000FFF7B0B910B5054C2046FEF73FFD044BDA
:105B7000C4F89030034BC4F8943010BD406A002044
:105B8000000004406074000870B503780546012BDE
:105B900061D1324ED0F89040B0422AD1304B4D20E6
:105BA0009A6B42F000729A631A6E42F000721A66A3
:105BB0001A6E2C4AD2F8801041F00071C2F88010A1
:105BC000D2F8801021F00071C2F880100E21D2F8B6
:105BD00080209A6B42F080629A631A6E42F0806273
:105BE0001A661B6EFEF74CFB1F4BE3601F4BC4F89D
:105BF00000380023C022B542C4F8003E226000D124
:105C0000A363D5F890603369002BFCDA01230C20E4
:105C10003361FFF757F93369DB07FCD41220FFF734
:105C200051F93369002BFCDA00262846A660FFF7FD
:105C300063FF6B68C4F81068DB68C4F81468C4F8C4
:105C40001C684BB90A4BA3614FF0FF336361A36833
:105C500043F00103A36070BD064BF4E7406A0020E7
:105C6000004502580044025800270040010020026D
:105C7000003C30C0083C30C0F8B5D0F89040054634
:105C800000214FF000662046FFF762FFD5F8941020
:105C900000234FF001128F684FF0FF30C4F8343802
:105CA000C4F81C2804EB431201339F42C2F8006978
:105CB000C2F8006BC2F80809C2F8080BF2D20B68F0
:105CC000D5F89020C5F898306362102313611669E7
:105CD00016F01006FBD11220FFF7F4F8D4F80038C4
:105CE00023F4FE63C4F80038A36943F4402343F06F
:105CF0001003A3610923C4F81038C4F814380B4BFF
:105D0000EB604FF0C043C4F8103B094BC4F8003BB4
:105D1000C4F81069C4F80039D5F8983003F11002BE
:105D200043F48013C5F89820A362F8BD3C740008C2
:105D300040800010D0F8902090F88A10D2F80038F7
:105D400023F4FE6343EA0113C2F8003870470000F1
:105D50002DE9F84300EB8103D0F890500C468046C3
:105D6000DA680FFA81F94801166806F00306731E17
:105D7000022B05EB41134FF0000194BFB604384EDF
:105D8000C3F8101B4FF0010104F1100398BF06F196
:105D9000805601FA03F3916998BF06F50046002981
:105DA0003AD0578A04F15801374349016F50D5F86A
:105DB0001C180B430021C5F81C382B180127C3F809
:105DC0001019A7405369611E9BB3138A928B9B08DD
:105DD000012A88BF5343D8F89820981842EA034311
:105DE00001F140022146C8F89800284605EB8202DE
:105DF0005360FFF7ADFE08EB8900C3681B8A43EAD6
:105E0000845348341E4364012E51D5F81C381F4377
:105E1000C5F81C78BDE8F88305EB4917D7F8001BD7
:105E200021F40041C7F8001BD5F81C1821EA030330
:105E3000C0E704F13F030B4A2846214605EB8303E4
:105E40005A60FFF785FE05EB4910D0F8003923F4BE
:105E50000043C0F80039D5F81C3823EA0707D7E714
:105E60000080001000040002D0F894201268C0F8EE
:105E70009820FFF741BE00005831D0F8903049011A
:105E80005B5813F4004004D013F4001F0CBF022031
:105E9000012070474831D0F8903049015B5813F425
:105EA000004004D013F4001F0CBF022001207047F3
:105EB00000EB8101CB68196A0B6813604B68536073
:105EC0007047000000EB810330B5DD68AA691368F4
:105ED000136119B9402B84BF402313606B8A146887
:105EE000D0F890201C4402EB4110013C09B2B4FBF5
:105EF000F3F46343033323F0030343EAC44343F05F
:105F0000C043C0F8103B2B6803F00303012B0ED1F4
:105F1000D2F8083802EB411013F4807FD0F8003B30
:105F200014BF43F0805343F00053C0F8003B02EB32
:105F30004112D2F8003B43F00443C2F8003B30BDAD
:105F4000F8B52B4D0446D5F8906006EB4013D3F816
:105F5000087B3807C3F8087B0AD5D6F81438190728
:105F600006D505EB840321462846DB685B68984725
:105F7000FA0720D5D6F81438DB071CD5A61C05EB8C
:105F800086035968C4B98B69488A5A68B2FBF0F72E
:105F900000FB172282B918681A6990420CD2121AB3
:105FA000C3E90024302383F3118811482146FFF709
:105FB00089FF84F31188F8BD012303FA04F26B8989
:105FC00023EA02036B81CB6813B121460848984746
:105FD000302383F3118805EB86056B689869416867
:105FE0000C30FEF7EDFF002383F31188E3E700BFD9
:105FF000406A002000EB81034A0170B5DD68D0F8EB
:1060000090306C692668266156BB1A444FF4002014
:10601000C2F810092A6802F00302012A0AB20ED15E
:10602000D3F8080803EB421410F4807FD4F8000979
:1060300014BF40F0805040F00050C4F8000903EB5A
:106040004212D2F8000940F00440C2F800090122CF
:10605000D3F8340802FA01F10143C3F8341870BDD3
:1060600019B9402E84BF4020206020681A442E8A2F
:106070008419013CB4FBF6F440EAC44040F00050FF
:10608000C6E700002DE9F843424D04464701D5F824
:10609000908008EB4013D3F8089919F0010FC3F86A
:1060A000089919D0D8F81038DB0715D5861C05EBF0
:1060B000860359684B6918681A6990422FD2121AE0
:1060C00000261A605E60302383F31188214628463B
:1060D000FFF790FF86F3118819F0800F1DD001267D
:1060E000D8F83438A640334217D005EB8403013486
:1060F000D5F89050D3F80CC0E4B22F44DCF814204B
:1061000005EB0434D2F800E05168714522D3D5F88C
:10611000343823EA0606C5F83468BDE8F88301235D
:1061200003FA04F22B8923EA02032B818B6813B153
:10613000214628469847302383F3118805EB8606CD
:106140000021736858690C30FEF73AFF002383F38F
:106150001188C1E7AEEB0103BCF81000834228BFF1
:106160000346D7F8180980B2B3EB800FD5D89068F2
:10617000A0F1040959F8048FC4F80080A0EB0908C5
:106180009844B8F1040FF5D818440B44906053605C
:10619000BAE700BF406A00202DE9F74FAD4CD4F8B4
:1061A00090607569B3691D4015F48057756107D01B
:1061B0002046FEF7A3FA03B0BDE8F04FFEF736B86D
:1061C000002D12DAD6F8003E9A0705D0D6F8003E28
:1061D00023F00303C6F8003ED6F804389D4823F0A8
:1061E0000103C6F80438FEF7F5FA2B0505D59948E2
:1061F000FFF782FC9748FEF7BDFAA8040CD5D6F845
:10620000083813F0060FF36823F470530CBF43F4FF
:10621000105343F4A053F360290704D56368DB6887
:106220000BB18C489847EA0200F1C380AB0240D51D
:10623000D4F890304FF000084FF001094FF0300AC9
:10624000DFF810B20093009B03EB4812D2F8003B3A
:1062500003F44023B3F5802F22D1D2F8003B002B6A
:106260001EDA628909FA08F322EA0303638108F15E
:10627000020304EB83025268D26822B141465846B9
:1062800001939047019B8AF3118804EB83035B68B9
:10629000986941680C30FEF793FE002383F3118860
:1062A00008F10108D4F894305FFA88F89B689845A3
:1062B000C9D9E8061AD5D4F890C0DCF82020C2F37A
:1062C0000A1002F00F0302F4F012B2F5802F00F072
:1062D000CF80B2F5402F09D104EB830300220CF5E7
:1062E000805CDB681B6A904240F0B6802B03D6F8D6
:1062F00018482CD5E70302D50020FFF721FEA6039E
:1063000002D50120FFF71CFE600302D50220FFF733
:1063100017FE210302D50320FFF712FEE20202D589
:106320000420FFF70DFEA30202D50520FFF708FEAB
:10633000670202D50620FFF703FE260202D50720DA
:10634000FFF7FEFDE00102D50820FFF7F9FD690324
:106350007FF531AFE20702D50020FFF793FEA307D8
:1063600002D50120FFF78EFE670702D50220FFF756
:1063700089FE260702D50320FFF784FEE50602D535
:106380000420FFF77FFEA00602D50520FFF77AFE66
:10639000610602D50620FFF775FE220602D507200A
:1063A000FFF770FEE3057FF506AF0820FFF76AFEF2
:1063B00001E7D4F890304FF000084FF001094FF09A
:1063C000300ADFF890B00093D4F894305FFA88F187
:1063D0009B6899423FF62AAF009B03EB4113D3F829
:1063E000002902F44022B2F5802F30D1D3F80029E1
:1063F000002A2CDAD3F8002942F09042C3F8002991
:10640000D3F80029002AFBDBD4F890000191FFF7B4
:106410009FFB0199228909FA01F322EA03032381F0
:106420008B1C04EB8302526892681AB158460193A0
:106430009047019B8AF3118804EB830300215B687A
:1064400058690C30FEF7BCFD002383F3118808F176
:106450000108B9E7406A0020910701D1DCF800701B
:10646000072A02F101029CBF03F8017B3F0A3AE7C9
:1064700002330CF5805C04EB83025268D2F818E01A
:10648000DEF80820DEE9001EA1EB0E0E0021884296
:106490000AD104EB830463689B699A6802449A609A
:1064A0005A6802445A6021E711F0030F01D1DCF869
:1064B00000708E4501F1010184BF02F8017B3F0AA3
:1064C000E5E700BFD0F8903003EB4111D1F8003B75
:1064D00043F40013C1F8003B70470000D0F890303F
:1064E00003EB4111D1F8003943F40013C1F800392E
:1064F00070470000D0F8903003EB4111D1F8003B19
:1065000023F40013C1F8003B70470000D0F890302E
:1065100003EB4111D1F8003923F40013C1F800391D
:106520007047000030B50433039C0172002104FB66
:106530000325C160C0E90653049B0363059BC0E9C2
:106540000000C0E90422C0E90842C0E90A1143631F
:1065500030BD00000022416AC260C0E90411C0E9F8
:106560000A226FF00101FEF751BD0000D0E90432AC
:10657000934201D1C2680AB9181D704700207047C4
:10658000036919600021C2680132C260C269134404
:1065900082699342036124BF436A0361FEF72ABD07
:1065A00038B504460D46E3683BB162690020131D0F
:1065B0001268A3621344E36207E0237A33B92946E1
:1065C0002046FEF707FD0028EDDA38BD6FF0010028
:1065D000FBE70000C368C269013BC3604369134421
:1065E00082699342436124BF436A4361002383620B
:1065F000036B03B11847704770B53023044683F32B
:106600001188866A3EB9FFF7CBFF054618B186F3BD
:106610001188284670BDA36AE26A13F8015B9342B1
:10662000A36202D32046FFF7D5FF002383F311882E
:10663000EFE700002DE9F84F04460E46174698464E
:106640004FF0300989F311880025AA46D4F828B004
:10665000BBF1000F09D141462046FFF7A1FF20B151
:106660008BF311882846BDE8F88FD4E90A12A7EB0E
:10667000050B521A934528BF9346BBF1400F1BD917
:10668000334601F1400251F8040B914243F8040BE8
:10669000F9D1A36A403640354033A362D4E90A23D6
:1066A0009A4202D32046FFF795FF8AF31188BD4234
:1066B000D8D289F31188C9E730465A46FBF708FA61
:1066C000A36A5E445D445B44A362E7E710B5029CA5
:1066D0000433017203FB0421C460C0E906130023E4
:1066E000C0E90A33039B0363049BC0E90000C0E9CF
:1066F0000422C0E90842436310BD0000026A6FF043
:106700000101C260426AC0E904220022C0E90A22F3
:10671000FEF77CBCD0E904239A4201D1C26822B9B9
:10672000184650F8043B0B6070470020704700008B
:10673000C3680021C2690133C3604369134482699D
:106740009342436124BF436A4361FEF753BC000098
:1067500038B504460D46E3683BB1236900201A1D95
:10676000A262E2691344E36207E0237A33B929465F
:106770002046FEF72FFC0028EDDA38BD6FF001004F
:10678000FBE7000003691960C268013AC260C26990
:10679000134482699342036124BF436A0361002367
:1067A0008362036B03B118477047000070B5302354
:1067B0000D460446114683F31188866A2EB9FFF709
:1067C000C7FF10B186F3118870BDA36A1D70A36A5C
:1067D000E26A01339342A36204D3E169204604399B
:1067E000FFF7D0FF002080F31188EDE72DE9F84F87
:1067F00004460D46904699464FF0300A8AF31188B8
:106800000026B346A76A4FB949462046FFF7A0FFC6
:1068100020B187F311883046BDE8F88FD4E90A0724
:106820003A1AA8EB0607974228BF1746402F1BD9F4
:1068300005F1400355F8042B9D4240F8042BF9D193
:10684000A36A40364033A362D4E90A239A4204D3B0
:10685000E16920460439FFF795FF8BF3118846451F
:10686000D9D28AF31188CDE729463A46FBF730F9A9
:10687000A36A3D443E443B44A362E5E7D0E90423D8
:106880009A4217D1C3689BB1836A8BB1043B9B1AB0
:106890000ED01360C368013BC360C3691A448369A7
:1068A0009A42026124BF436A036100238362012389
:1068B000184670470023FBE700F024B9014B586AE3
:1068C000704700BF000C0040034B002258631A6160
:1068D0000222DA60704700BF000C0040014B00222A
:1068E000DA607047000C0040014B5863704700BFEE
:1068F000000C0040FEE7000070B51F4B0025044669
:1069000086B058600E4605638163FDF767FC04F1AD
:106910002803A5606563C4E90A3304F11003C4E9E0
:1069200004334FF0FF33C4E90044C4E90635FFF7F0
:10693000C5FF2B46024604F13C012046C4E908236A
:1069400080230E4AA567FEF7C7FA7368E06003620A
:1069500001230B4A80F824303169F06800920190DD
:10696000CDE90213074BCDE90435FEF7CFFA6846AF
:10697000FEF7F0FA06B070BDE04E00207474000817
:106980006C740008F5680008024A536B18435063A2
:10699000704700BF304C00204B6843608B688360B9
:1069A000CB68C3600B6943614B6903628B694362C7
:1069B0000B6803607047000008B53A4B40F2FF7166
:1069C0003948D3F888200A43C3F88820D3F88820B0
:1069D00022F4FF6222F00702C3F88820D3F888303F
:1069E000324B1A6C0A431A649A6E0A439A66304A0A
:1069F0009B6E1146FFF7D0FF00F5806002F11C018D
:106A0000FFF7CAFF00F5806002F13801FFF7C4FF0D
:106A100000F5806002F15401FFF7BEFF00F58060D1
:106A200002F17001FFF7B8FF00F5806002F18C0100
:106A3000FFF7B2FF00F5806002F1A801FFF7ACFF9D
:106A400000F5806002F1C401FFF7A6FF00F5806049
:106A500002F1E001FFF7A0FF00F5806002F1FC0108
:106A6000FFF79AFF02F58C7100F58060FFF794FF45
:106A700000F002F90F4BD3F8902242F00102C3F864
:106A80009022D3F8942242F00102C3F89422052206
:106A9000C3F898204FF06052C3F89C20064AC3F810
:106AA000A02008BD004402580000025800450258CA
:106AB000A074000800ED00E01F00080308B500F016
:106AC000ABFAFEF7ADF90C4BDA6B42F04002DA6339
:106AD0005A6E22F040025A665B6E084B1A6842F00A
:106AE00008021A601A6842F004021A60FEF788FF72
:106AF000BDE80840FEF7A8BC00450258001802484F
:106B0000704700000E4B9A6C42F008029A641A6FAC
:106B100042F008021A670B4A1B6FD36B43F008035D
:106B2000D363C722084B9A624FF0FF32DA62002229
:106B30009A615A63DA605A6001225A611A6070479A
:106B4000004502580010005C000C0040094A08B5DE
:106B50001169D3680B40D9B29B076FEA010111613B
:106B600007D5302383F31188FEF790F9002383F3D0
:106B7000118808BD000C0040044BDA6B0243DA6355
:106B80005A6E104358665B6E704700BF004502584E
:106B9000384B4FF0FF31D3F88020C3F88010D3F882
:106BA00080200022C3F88020D3F88000D3F884002E
:106BB000C3F88410D3F88400C3F88420D3F8840089
:106BC000D86F40F0FF4040F4FF0040F4DF4040F059
:106BD0007F00D867D86F20F0FF4020F4FF0020F43A
:106BE000DF4020F07F00D867D86FD3F888006FEAC5
:106BF00040506FEA5050C3F88800D3F88800C0F3C3
:106C00000A00C3F88800D3F88800D3F89000C3F8CE
:106C10009010D3F89000C3F89020D3F89000D3F8E8
:106C20009400C3F89410D3F89400C3F89420D3F8D8
:106C30009400D3F89800C3F89810D3F89800C3F8DC
:106C40009820D3F89800D3F88C00C3F88C10D3F8B0
:106C50008C00C3F88C20D3F88C00D3F89C00C3F8C8
:106C60009C10D3F89C10C3F89C20D3F89C3000F003
:106C7000ABB900BF0044025808B50122504BC3F81D
:106C80000821504B5A6D42F002025A65DA6F42F009
:106C90000202DA670422DB6F4B4BDA605A68910418
:106CA000FCD54A4A1A6001229A60494ADA600022F9
:106CB0001A614FF440429A61434B9A699204FCD5A1
:106CC0001A6842F480721A60424B1A6F12F4407FC5
:106CD00004D04FF480321A6700221A671A6842F013
:106CE00001021A603B4B1A685007FCD500221A615A
:106CF0001A6912F03802FBD1012119604FF080416E
:106D000059605A67344ADA62344A1A611A6842F49E
:106D100080321A602F4B1A689103FCD51A6842F42E
:106D200080521A601A689204FCD52D4A2D499A6245
:106D300000225A63196301F57C01DA6301F5E771FA
:106D400099635A64284A1A64284ADA621A6842F037
:106D5000A8521A601F4B1A6802F02852B2F1285F3D
:106D6000F9D148229A614FF48862DA6140221A62AE
:106D70001F4ADA641F4A1A651F4A5A651F4A9A65F4
:106D800032231F4A1360136803F00F03022BFAD15A
:106D9000104A136943F003031361136903F03803C6
:106DA000182BFAD14FF00050FFF7E6FE4FF080406D
:106DB000FFF7E2FE4FF00040BDE80840FFF7DCBE01
:106DC00000800051004502580048025800C000F001
:106DD00004000001004402580000FF0100889008F0
:106DE0003220600063020901470E0508DD0BBF0178
:106DF00020000020000001100910E0000001011037
:106E0000002000524FF0B04208B5D2F8883003F0AD
:106E10000103C2F8883023B1044A13680BB15068EB
:106E20009847BDE80840FDF701BA00BFF86A0020A6
:106E30004FF0B04208B5D2F8883003F00203C2F830
:106E4000883023B1044A93680BB1D0689847BDE8F5
:106E50000840FDF7EBB900BFF86A00204FF0B042E0
:106E600008B5D2F8883003F00403C2F8883023B1A3
:106E7000044A13690BB150699847BDE80840FDF713
:106E8000D5B900BFF86A00204FF0B04208B5D2F87B
:106E9000883003F00803C2F8883023B1044A9369AC
:106EA0000BB1D0699847BDE80840FDF7BFB900BFF6
:106EB000F86A00204FF0B04208B5D2F8883003F0ED
:106EC0001003C2F8883023B1044A136A0BB1506A28
:106ED0009847BDE80840FDF7A9B900BFF86A00204F
:106EE0004FF0B04310B5D3F8884004F47872C3F87B
:106EF0008820A30604D5124A936A0BB1D06A98473A
:106F0000600604D50E4A136B0BB1506B98472106EF
:106F100004D50B4A936B0BB1D06B9847E20504D5AF
:106F2000074A136C0BB1506C9847A30504D5044A6B
:106F3000936C0BB1D06C9847BDE81040FDF776B963
:106F4000F86A00204FF0B04310B5D3F8884004F43D
:106F50007C42C3F88820620504D5164A136D0BB134
:106F6000506D9847230504D5124A936D0BB1D06D2F
:106F70009847E00404D50F4A136E0BB1506E984742
:106F8000A10404D50B4A936E0BB1D06E98476204EE
:106F900004D5084A136F0BB1506F9847230404D5EA
:106FA000044A936F0BB1D06F9847BDE81040FDF7CE
:106FB0003DB900BFF86A002008B5FFF7C7FDBDE87E
:106FC0000840FDF733B90000062108B50846FDF773
:106FD00057F906210720FDF753F906210820FDF790
:106FE0004FF906210920FDF74BF906210A20FDF78C
:106FF00047F906211720FDF743F906212820FDF760
:107000003FF909217A20FDF73BF907213220BDE83D
:107010000840FDF735B9000008B5FFF7B9FD00F0ED
:107020000BF8FDF7E1FAFDF7B3F9FFF769FDBDE8ED
:107030000840FFF741BC00000023054A1946013310
:10704000102BC2E9001102F10802F8D1704700BF0D
:10705000F86A00200B460146184600F003B800000D
:1070600000F00EB810B5054C13462CB10A46014687
:107070000220AFF3008010BD2046FCE700000000B6
:10708000024B0146186800F035B800BF64220020AA
:1070900010B501390244904201D1002005E0037887
:1070A00011F8014FA34201D0181B10BD0130F2E7C7
:1070B0002DE9F041A3B1C91A17780144044603F140
:1070C000FF3C8C42204601D9002009E00578BD42F2
:1070D00004F10104F5D10CEB0405D618A54201D149
:1070E000BDE8F08115F8018D16F801EDF045F5D0F9
:1070F000E7E7000037B5002944D051F8043C01907F
:10710000002BA1F10404B8BFE41800F047F81E4AB0
:107110000198136833B96360146003B0BDE8304070
:1071200000F042B8A34208D9256861198B4201BF1B
:1071300019685B6849192160EDE71A465B680BB175
:10714000A342FAD911685518A5420BD124682144ED
:107150005418A3421160E0D11C685B68536021445D
:107160001160DAE702D90C230360D6E725686119BC
:107170008B4204BF19685B68636004BF49192160D2
:107180005460CAE703B030BD786B0020034611F8A5
:10719000012B03F8012B002AF9D17047014800F0B8
:1071A00009B800BF7C6B0020014800F005B800BFA3
:1071B0007C6B00207047000070470000636F6D2EED
:1071C0006375626570696C6F742E68657265707244
:1071D0006F00000053544D333248373F3F3F005358
:1071E000544D3332483734332F37353300000000E5
:1071F00043414E464449666163653A204D65737369
:107200006167652052414D204F766572666C6F77DD
:10721000210000004261642043414E49666163657C
:1072200020696E6465782E000000000000000000F8
:10723000992300083D1C0008CD2A0008AD1C000859
:10724000E51C0008F52000085D1E0008751C0008FC
:10725000791C0008511C0008391C0008B5200008E2
:107260005D1C0008412C0008691C000889200008EA
:107270000000000000000000092C0008112C00088C
:10728000B92B000840A2E4F1646891060041A3E52F
:10729000F265699207000000000000000D4300083D
:1072A000F942000835430008214300082D43000837
:1072B0001943000805430008F14200084143000853
:1072C000000000000100000000000000633000002A
:1072D000CC7200080006002000220020B04C0020E4
:1072E000E04E00204375626550696C6F7400254262
:1072F0004F415244252D424C002553455249414CA3
:107300002500000002000000000000002D450008DC
:107310009D450008400040008C670020A0670020C9
:107320000200000000000000030000000000000058
:10733000E54500080000000010000000B4670020D0
:10734000000000000100000000000000406A002072
:1073500001010200E5530008F552000891530008AE
:1073600075530008430000006C73000809024300D5
:10737000020100C0320904000001020201000524DC
:107380000010010524010001042402020524060066
:1073900001070582030800FF09040100020A00003A
:1073A00000070501024000000705810240000000BF
:1073B00012000000B8730008120110010200004022
:1073C000AE2D115000020102030100000403090464
:1073D00025424F41524425004865726550726F0046
:1073E00030313233343536373839414243444546FB
:1073F0000000000000000020000002000200000069
:107400000001003000000000000000000000002427
:1074100000000800040000000004000000FC000060
:1074200002000000000004300080000000000000A6
:107430000000003800000100010000000000000012
:10744000E9470008A14A00084D4B000840004000F1
:10745000DC6A0020DC6A002001000000F06A0020E5
:1074600000020000001000000800000069646C6564
:10747000000000006D61696E002C043804043C08B3
:107480000C10141C202425000000000000006404DF
:107490000100040000000000000C0010283034003F
:1074A0008008802A00000000EAAEAAAA000000249A
:1074B000FFFF000000A0A000009009000A48A01AE9
:1074C00000000000AF6EFA9F000000007FBF0000C8
:1074D000AA00A00000AAAA00A60000040000000064
:1074E000F7AAAAAA00000000FFDF00000AAA000015
:1074F0000000000000000A0000000000AAAAAAAADA
:1075000000000500FFFF0000000000007700000001
:107510000000000100000000AAAAAAA900000000C3
:10752000FFFF00000000000000000000000000005D
:1075300000000000AAAAAAAA00000000FFFF0000A5
:10754000000000000000000000000000000000003B
:10755000AAAAAAAA00000000FFFF00000000000085
:10756000000000000000000000000000AAAAAAAA73
:1075700000000000FFFF000000000000000000000D
:107580000000000000000000AAAAAAAA0000000053
:10759000FFFF0000000000000000000000000000ED
:1075A00000000000AAAAAAAA00000000FFFF000035
:1075B00000000000000000000000000000000000CB
:1075C000AAAAAAAA00000000FFFF00000000000015
:1075D000000000004C8DFF7F010000000000000053
:1075E0000D04000000000000000018000000000072
:1075F000FE2A0100D2040000FF000000000000008D
:10760000D47100083F00000050040000DF71000842
:107610003F000000009600000000080096000000F7
:107620000008000004000000CC7300080000000007
:10763000000000000000000000000000000000004A
:107640000000000068220020000000000000000090
:10765000000000000000000000000000000000002A
:10766000000000000000000000000000000000001A
:10767000000000000000000000000000000000000A
:1076800000000000000000000000000000000000FA
:1076900000000000000000000000000000000000EA
:1076A0000000000000000000FFFFFFFFFFFFFFFFE2
:1076B000FFFFFFFFFFFFFFFFFFFFFFFFFFFFFFFFDA
:1076C000FFFFFFFFFFFFFFFFFFFFFFFFFFFFFFFFCA
:1076D000FFFFFFFFFFFFFFFFFFFFFFFFFFFFFFFFBA
:1076E000FFFFFFFFFFFFFFFFFFFFFFFFFFFFFFFFAA
:020000040803EF
:020000040804EE
:1000000000210030B10D0408C195060865030408FD
:10001000499506084195060845950608B30D04085C
:10002000B30D0408B30D0408B30D0408353A0B08EA
:10003000B30D0408B30D0408B30D0408B30D040890
:10004000B30D0408B30D0408B30D0408B30D040880
:10005000B30D0408B30D040845A50B0871A50B08E2
:100060009DA50B08C9A50B08F5A50B088D470B0826
:10007000B5470B08E1470B080D480B0839480B083A
:1000800061480B088D480B08E1430B08C965060859
:10009000F1650608DD6506080566060821A60B0859
:1000A000B30D040835A70B08B30D040849A70B08C6
:1000B000B30D0408B30D0408B30D0408B30D040810
:1000C000B30D0408B30D0408B30D040829600B0830
:1000D000B30D0408B30D0408B30D04080DA70B08F5
:1000E00085A60B08B30D0408B30D0408B30D04086E
:1000F000B30D0408B30D0408B30D0408B9480B0888
:10010000B30D0408F9A60B084DA70B08B30D04089E
:10011000B30D0408B30D0408B30D0408B30D0408AF
:10012000E5480B080D490B0839490B0865490B08D0
:1001300091490B08B30D0408B30D0408B30D04086E
:10014000B30D0408B30D0408B30D0408B30D04087F
:10015000B9490B08E5490B08114A0B08B30D04080F
:10016000B30D0408B30D0408B30D0408B30D04085F
:10017000B30D040825540B08B30D0408B30D04088F
:10018000B30D0408B30D040821A70B08B30D040830
:100190003D600B08B30D0408B30D0408B30D04084B
:1001A000B30D0408B30D0408B30D0408B30D04081F
:1001B000B30D0408B30D0408B30D0408B30D04080F
:1001C000B30D0408B30D0408B30D0408B30D0408FF
:1001D000B30D0408B30D0408B30D0408B30D0408EF
:1001E000B30D0408B30D0408B30D0408B30D0408DF
:1001F000B30D0408B30D0408B30D0408B30D0408CF
:10020000B30D0408B30D0408B30D0408B30D0408BE
:10021000B30D0408B30D0408B30D0408B30D0408AE
:10022000B30D0408B30D0408B30D0408B30D04089E
:10023000B30D0408B30D0408B30D040801440B0802
:10024000B30D040865450B088D450B08B9450B082F
:10025000E5450B0811460B083D460B0869460B089F
:1002600095460B08B30D0408B30D0408B30D04083C
:10027000B30D0408B30D0408B30D0408B30D04084E
:10028000B30D0408B30D0408B30D0408B30D04083E
:10029000B30D0408B30D0408B30D0408B30D04082E
:1002A000B30D0408B30D0408B30D0408B30D04081E
:1002B000B30D0408B30D0408B30D0408B30D04080E
:1002C000B30D0408B30D0408B30D0408B30D0408FE
:1002D000B30D0408B30D0408B30D0408B30D0408EE
:1002E00041210408553C0408C556040885630408E8
:1002F000A54B05086D8F05081DC10508C9C805086F
:1003000025CC0508D93F060819660608F9680608CD
:10031000FD6D0608818E06084DA40608852B080889
:1003200079CA09083DE5090815050A08D9300A08FF
:10033000D5350A0845830A080000000000000000C7
:1003400040A2E4F16468910658A9CDD000D5049587
:10035000A4E50900F180ABA000000D04FFFFFFFF42
:10036000FFFFFFFFEFF30383EFF30982EFF3088151
:10037000DFF814D02DE9FE4F684601F00DF9BDE815
:10038000FE4F8D467047000054450030F1EE101AC4
:10039000A0EC200A01607047A0EC108A704700BFF3
:1003A00081F0004102E000BF83F0004330B54FEA26
:1003B00041044FEA430594EA050F08BF90EA020F93
:1003C0001FBF54EA000C55EA020C7FEA645C7FEA26
:1003D000655C00F0E2804FEA5454D4EB5555B8BF49
:1003E0006D420CDD2C4480EA020281EA030382EABA
:1003F000000083EA010180EA020281EA0303362D4C
:1004000088BF30BD11F0004F4FEA01314FF4801C1E
:100410004CEA113102D0404261EB410113F0004F30
:100420004FEA03334CEA133302D0524263EB4303E7
:1004300094EA050F00F0A780A4F10104D5F1200E85
:100440000DDB02FA0EFC22FA05F2801841F10001E0
:1004500003FA0EF2801843FA05F359410EE0A5F1B4
:1004600020050EF1200E012A03FA0EFC28BF4CF0E5
:10047000020C43FA05F3C01851EBE37101F000459B
:1004800007D54FF0000EDCF1000C7EEB00006EEBA8
:100490000101B1F5801F1BD3B1F5001F0CD3490832
:1004A0005FEA30004FEA3C0C04F101044FEA445289
:1004B00012F5800F80F09A80BCF1004F08BF5FEA10
:1004C000500C50F1000041EB045141EA050130BDF0
:1004D0005FEA4C0C404141EB0101013C28BFB1F502
:1004E000801FE9D291F0000F04BF01460020B1FA4D
:1004F00081F308BF2033A3F10B03B3F120020CDA20
:100500000C3208DD02F1140CC2F10C0201FA0CF0FD
:1005100021FA02F10CE002F11402D8BFC2F1200C62
:1005200001FA02F120FA0CFCDCBF41EA0C01904018
:10053000E41AA2BF01EB0451294330BD6FEA040461
:100540001F3C1CDA0C340EDC04F11404C4F120024C
:1005500020FA04F001FA02F340EA030021FA04F35E
:1005600045EA030130BDC4F10C04C4F1200220FAB5
:1005700002F001FA04F340EA0300294630BD21FAF3
:1005800004F0294630BD94F0000F83F4801306BFB9
:1005900081F480110134013D4EE77FEA645C18BFAD
:1005A0007FEA655C29D094EA050F08BF90EA020F44
:1005B00005D054EA000C04BF1946104630BD91EA3C
:1005C000030F1EBF0021002030BD5FEA545C05D13F
:1005D0004000494128BF41F0004130BD14F580047E
:1005E0003CBF01F5801130BD01F0004545F0FE41F2
:1005F00041F470014FF0000030BD7FEA645C1ABF27
:10060000194610467FEA655C1CBF0B46024650EA5D
:10061000013406BF52EA033591EA030F41F4002189
:1006200030BD00BF90F0000F04BF0021704730B50F
:100630004FF4806404F132044FF000054FF00001E4
:1006400050E700BF90F0000F04BF0021704730B5A5
:100650004FF4806404F1320410F0004548BF40427A
:100660004FF000013EE700BF42004FEAE2014FEACF
:1006700031014FEA02701FBF12F07F4393F07F4FAA
:1006800081F06051704732F07F4208BF704793F0AD
:100690007F4F04BF41F40021704730B54FF46074C0
:1006A00001F0004521F000411CE700BF50EA0102C3
:1006B00008BF704730B54FF000050AE050EA01026C
:1006C00008BF704730B511F0004502D5404261EBDC
:1006D00041014FF4806404F132045FEA915C3FF41D
:1006E000D8AE4FF003025FEADC0C18BF03325FEABA
:1006F000DC0C18BF033202EBDC02C2F1200300FA6B
:1007000003FC20FA02F001FA03FE40EA0E0021FA8F
:1007100002F11444BDE600BF80F0004002E000BFDB
:1007200081F0004142001FBF5FEA410392EA030FDC
:100730007FEA226C7FEA236C6AD04FEA1262D2EB26
:100740001363C1BFD218414048404140B8BF5B422B
:10075000192B88BF704710F0004F40F4000020F0C4
:100760007F4018BF404211F0004F41F4000121F0DA
:100770007F4118BF494292EA030F3FD0A2F1010224
:1007800041FA03FC10EB0C00C3F1200301FA03F162
:1007900000F0004302D5494260EB4000B0F5000F85
:1007A00013D3B0F1807F06D340084FEA310102F144
:1007B0000102FE2A51D2B1F1004F40EBC25008BFF6
:1007C00020F0010040EA03007047490040EB0000C0
:1007D000013A28BFB0F5000FEDD2B0FA80FCACF1C1
:1007E000080CB2EB0C0200FA0CF0AABF00EBC250EE
:1007F00052421843BCBFD0401843704792F0000FDC
:1008000081F4000106BF80F400000132013BB5E72E
:100810004FEA41037FEA226C18BF7FEA236C21D0A4
:1008200092EA030F04D092F0000F08BF0846704709
:1008300090EA010F1CBF0020704712F07F4F04D1D7
:10084000400028BF40F00040704712F100723CBFEA
:1008500000F50000704700F0004343F0FE4040F414
:10086000000070477FEA226216BF08467FEA2363D2
:100870000146420206BF5FEA412390EA010F40F4BD
:10088000800070474FF0000304E000BF10F0004309
:1008900048BF40425FEA000C08BF704743F09643F0
:1008A00001464FF000001CE050EA010208BF70470B
:1008B0004FF000030AE000BF50EA010208BF704792
:1008C00011F0004302D5404261EB41015FEA010CA7
:1008D00002BF84460146002043F0B64308BFA3F19F
:1008E0008053A3F50003BCFA8CF2083AA3EBC25381
:1008F00010DB01FA02FC634400FA02FCC2F12002A0
:10090000BCF1004F20FA02F243EB020008BF20F0D6
:100910000100704702F1200201FA02FCC2F120023C
:1009200050EA4C0021FA02F243EB020008BF20EA31
:10093000DC7070477BB972B90029BEBF00204FF050
:10094000004106E008BF00281CBF6FF000414FF0D7
:10095000FF3000F02BBAADF1080C6DE904CE002990
:1009600009DB002B1ADB00F0B9F8DDF804E0DDE963
:10097000022304B07047404261EB4101002B1BDBB6
:1009800000F0ACF8DDF804E0DDE9022304B04042F9
:1009900061EB4101524263EB43037047524263EB08
:1009A000430300F09BF8DDF804E0DDE9022304B026
:1009B000404261EB41017047524263EB430300F058
:1009C0008DF8DDF804E0DDE9022304B0524263EB68
:1009D0004303704753B94AB9002908BF00281CBF18
:1009E0004FF0FF314FF0FF3000F0E0B9ADF1080CEF
:1009F0006DE904CE00F072F8DDF804E0DDE90223D1
:100A000004B07047430803F05533C01A830803F05D
:100A1000333300F03330184400EB101000F00F3087
:100A200000EB002000EB0040000E704708B50246C6
:100A30000B4643EC172BB5EEC07BF1EE10FA03D456
:100A4000BDE8084000F02AB8B1EE477B51EC170B27
:100A500000F024F8404261EB410108BD9FED0B6BB3
:100A600007EE900A9FED0B5BB7EEE77A27EE066B79
:100A7000BCEEC66BB8EE464BA4EE457BFCEEC77BE6
:100A800016EE101A17EE900A704700BF0000000023
:100A90000000F03D000000000000F0419FED0B6BF6
:100AA00041EC170B9FED0B5B27EE066BBCEEC66BA4
:100AB000B8EE464BA4EE457BFCEEC77B16EE101A53
:100AC00017EE900A704700BFAFF3008000000000EF
:100AD0000000F03D000000000000F0412DE9F0476B
:100AE000089D04468E46002B4DD18A42944669D912
:100AF000B2FA82F252B101FA02F3C2F1200120FAF5
:100B000001F10CFA02FC41EA030E94404FEA1C4842
:100B1000210CBEFBF8F61FFA8CF708FB16E341EA3E
:100B2000034306FB07F199420AD91CEB030306F1C4
:100B3000FF3080F01F81994240F21C81023E6344E5
:100B40005B1AA4B2B3FBF8F008FB103344EA034489
:100B500000FB07F7A7420AD91CEB040400F1FF339E
:100B600080F00A81A74240F207816444023840EADB
:100B70000640E41B00261DB1D4400023C5E9004314
:100B80003146BDE8F0878B4209D9002D00F0EF8097
:100B90000026C5E9000130463146BDE8F087B3FACA
:100BA00083F6002E4AD18B4202D3824200F2F980B2
:100BB000841A61EB030301209E46002DE0D0C5E9B5
:100BC000004EDDE702B9FFDEB2FA82F2002A40F001
:100BD0009280A1EB0C014FEA1C471FFA8CFE012604
:100BE000200CB1FBF7F307FB131140EA01410EFBA8
:100BF00003F0884208D91CEB010103F1FF3802D24F
:100C0000884200F2CB804346091AA4B2B1FBF7F048
:100C100007FB101144EA01440EFB00FEA64508D96B
:100C20001CEB040400F1FF3102D2A64500F2BB80A8
:100C30000846A4EB0E0440EA03409CE7C6F12007F7
:100C4000B34022FA07FC4CEA030C20FA07F401FA3D
:100C500006F31C43F9404FEA1C4900FA06F3B1FBC6
:100C6000F9F8200C1FFA8CFE09FB181140EA01412B
:100C700008FB0EF0884202FA06F20BD91CEB0101C8
:100C800008F1FF3A80F08880884240F28580A8F120
:100C900002086144091AA4B2B1FBF9F009FB101172
:100CA00044EA014100FB0EFE8E4508D91CEB010110
:100CB00000F1FF346CD28E456AD90238614440EAB3
:100CC0000840A0FB0294A1EB0E01A142C846A64633
:100CD00056D353D05DB1B3EB080261EB0E0101FABC
:100CE00007F722FA06F3F1401F43C5E90071002619
:100CF0003146BDE8F087C2F12003D8400CFA02FC6F
:100D000021FA03F3914001434FEA1C471FFA8CFE7E
:100D1000B3FBF7F007FB10360B0C43EA064300FB6E
:100D20000EF69E4204FA02F408D91CEB030300F10C
:100D3000FF382FD29E422DD9023863449B1B89B2C3
:100D4000B3FBF7F607FB163341EA034106FB0EF34C
:100D50008B4208D91CEB010106F1FF3816D28B42F9
:100D600014D9023E6144C91A46EA004638E72E46C5
:100D7000284605E70646E3E61846F8E64B45A9D2BD
:100D8000B9EB020864EB0C0E0138A3E74646EAE72C
:100D9000204694E74046D1E7D0467BE7023B6144DA
:100DA00032E7304609E76444023842E7704700BF43
:100DB00002E000F000F8FEE772B6384880F30888D9
:100DC000374880F3098837483749086040F2000007
:100DD000CCF200004EF63471CEF200010860BFF391
:100DE0004F8FBFF36F8F40F20000C0F2F0004EF65D
:100DF0008851CEF200010860BFF34F8FBFF36F8FB1
:100E00004FF00000E1EE100A4EF63C71CEF2000108
:100E10000860062080F31488BFF36F8F79F044FADE
:100E200079F0E6F978F05CFA4FF055301F491B4A2B
:100E300091423CBF41F8040BFAE71D49184A914220
:100E40003CBF41F8040BFAE71A491B4A1B4B9A4274
:100E50003EBF51F8040B42F8040BF8E70020184994
:100E6000184A91423CBF41F8040BFAE779F0FEF9C9
:100E700078F0B8FA144C154DAC4203DA54F8041B60
:100E80008847F9E701F04CF9114C124DAC4203DAF6
:100E900054F8041B8847F9E779F0E6B900210030DF
:100EA000003D00300000040808ED00E000010030C3
:100EB0000021003048DF0D08003D00305C43003069
:100EC0006043003078C90130E002040838030408A8
:100ED00038030408380304082DE9F04F2DED108A7B
:100EE000C1F80CD0D0F80CD0BDEC108ABDE8F08F62
:100EF000002383F311882846A047002077F0B2FD35
:100F0000FEE777F049FC00DFFEE7000070B54FF028
:100F1000FF0C4CF4E06C1CEA11541DBF1CEA135585
:100F200094EA0C0F95EA0C0F00F0DEF82C4481EAED
:100F3000030621EA4C5123EA4C5350EA013518BF0D
:100F400052EA033541F4801143F4801338D0A0FBFA
:100F500002CE4FF00005E1FB02E506F00042E0FBA7
:100F600003E54FF00006E1FB03569CF0000F18BFAD
:100F70004EF0010EA4F1FF04B6F5007F64F5407455
:100F800004D25FEA4E0E6D4146EB060642EAC621E8
:100F900041EA55514FEAC52040EA5E504FEACE2E55
:100FA000B4F1FD0C88BFBCF5E06F1ED8BEF1004F58
:100FB00008BF5FEA500E50F1000041EB045170BDD4
:100FC00006F0004646EA010140EA020081EA030118
:100FD000B4EB5C04C2BFD4EB0C0541EA045170BD14
:100FE00041F480114FF0000E013C00F3AB8014F18E
:100FF000360FDEBF002001F0004170BDC4F10004D7
:10100000203C35DA0C341BDC04F11404C4F1200557
:1010100000FA05F320FA04F001FA05F240EA0200B2
:1010200001F0004221F0004110EBD37021FA04F6E8
:1010300042EB06015EEA430E08BF20EAD37070BDA2
:10104000C4F10C04C4F1200500FA04F320FA05F001
:1010500001FA04F240EA020001F0004110EBD37003
:1010600041F100015EEA430E08BF20EAD37070BD73
:10107000C4F1200500FA05F24EEA020E20FA04F34C
:1010800001FA05F243EA020321FA04F001F00041FB
:1010900021FA04F220EA020000EBD3705EEA430E6C
:1010A00008BF20EAD37070BD94F0000F0FD101F09B
:1010B0000046400041EB010111F4801F08BF013CD4
:1010C000F7D041EA060195F0000F18BF704703F012
:1010D0000046520043EB030313F4801F08BF013D99
:1010E000F7D043EA0603704794EA0C0F0CEA135555
:1010F00018BF95EA0C0F0CD050EA410618BF52EA0F
:101100004306D1D181EA030101F000414FF0000014
:1011100070BD50EA410606BF1046194652EA430622
:1011200019D094EA0C0F02D150EA013613D195EA96
:101130000C0F05D152EA03361CBF104619460AD1DE
:1011400081EA030101F0004141F0FE4141F47001E8
:101150004FF0000070BD41F0FE4141F4780170BDD8
:101160004FEA410212F5001215D211D56FF47873CF
:10117000B3EB625212D94FEAC12343F0004343EA72
:10118000505311F0004F23FA02F018BF404270474D
:101190004FF00000704750EA013005D111F00040D7
:1011A00008BF6FF0004070474FF00000704700BF6D
:1011B0004FEA4102B2F1E04324BFB3F5001CDCF179
:1011C000FE5C0DD901F0004C4FEAC0024CEA5070B1
:1011D000B2F1004F40EB830008BF20F001007047E0
:1011E00011F0804F21D113F13872BCBF01F00040E3
:1011F000704741F480114FEA5252C2F11802C2F115
:10120000200C10FA0CF320FA02F018BF40F0010095
:101210004FEAC1234FEAD32303FA0CFC40EA0C0047
:1012200023FA02F34FEA4303CCE77FEA625307D184
:1012300050EA01331EBF4FF0FE4040F440007047BB
:1012400001F0004040F0FE4040F40000704700BF55
:1012500001F0FF01102A2BDB10F0070F08D010F867
:10126000013B013A8B422DD010F0070F42B3F6D16B
:10127000F0B441EA012141EA014122F007047FF084
:1012800000070023F0E80256083C85EA010586EADB
:10129000010685FA47F5A3FA87F586FA47F6A5FA17
:1012A00087F68EB9EED1F0BC01F0FF0102F0070223
:1012B00032B110F8013B013A83EA010313B1F8D1CE
:1012C0000020704701387047002D06BF35460338AF
:1012D000073815F0010F07D1013015F4807F02BFE8
:1012E000013015F4C03F0130F0BC0138704700BF39
:1012F000EC46A0E8F05F4FF000007047B0E8F05F08
:10130000E546080008BF0120704700BF10F8012B18
:1013100011F8013B012A28BF9A42F7D0D01A704732
:10132000034613F8012B002AFBD1181A0138704725
:10133000C36A13F0040F01D040687047006870471B
:10134000704700BF10B5044608462160FFF7F0FF64
:10135000E060FFF7F5FF60600023A360204610BD4A
:101360000368DB6A13F0100F0CBF012000207047E8
:1013700038B50446C5682035C560FFF7F1FF08B1F0
:101380004835E5606368DB69DB0903F00403E26864
:101390001343E36038BD00BF4FF0E023D3F8880D5E
:1013A00000F4A000B0F5A00F14BF0020012070478A
:1013B00010B50446FFF7F0FF18B1A36843F001032E
:1013C000A36010BD00F47F40B0F53E4F14BF002075
:1013D0000120704710B5044643689869FFF7B0FFD5
:1013E0000088FFF7EFFF206110BD00BF014B024AEC
:1013F0001A60704760430030ED55CEAC4FF0E023EB
:10140000D3F8000D00F47020B0F5402F14BF002079
:101410000120704703691BB14268936902339361ED
:10142000704700BF08B504220121024800F01CFAF1
:1014300008BD00BFF0240C0808B5042201210830C3
:1014400000F012FA08BD00BF08B510220121406863
:1014500000F00AFA08BD00BF08B50068202201218B
:101460000C3000F001FA08BD08B5406804220121E3
:10147000103000F0F9F908BD08B5042201210C3044
:1014800000F0F2F908BD00BF08B540680C22012148
:10149000143000F0E9F908BD08B50C2201210068FC
:1014A00000F0E2F908BD00BF38B5044610E008229C
:1014B0000121204600F0D8F925682846FFF740FFB3
:1014C000217A6268521BB2FBF1F200F0CDF90C34C4
:1014D0001CB12368B3F1FF3FE9D138BD00B587B037
:1014E000094B00931433019304238DF808304FF017
:1014F000FF330393049301238DF814306846FFF7FC
:10150000D3FF07B05DF804FB28ED00E0094B1A6833
:10151000094B9A4200D1704700B583B0074B019345
:10152000042201210DEB020000F09EF903B05DF8EA
:1015300004FB00BF60430030ED55CEACACCE55EDA2
:1015400070B5A2B00446FFF70BFF08B311A8FEF771
:1015500023FF666806F1200C01AD6036AE46DCF86C
:101560000000DCF80410DCF80820DCF80C30AEE8F1
:101570000F000CF1100C7546B445EFD163681B6E7B
:1015800021938422012101A800F06EF922B070BDE0
:1015900001A8FEF7FBFEF4E700B587B0014601A8FD
:1015A000FFF7D0FE01A8FFF7E3FE01A8FFF700FF59
:1015B00001A8FFF70FFF08E001A8FFF7C1FF24E033
:1015C000FFF7A4FF00F0FEF950BBFFF70FFF04A8E0
:1015D00000F0AAF9FFF726FF01A8FFF72DFF01A8E9
:1015E000FFF732FF01A8FFF737FF01A8FFF73CFF25
:1015F00001A8FFF741FF01A8FFF746FF01A8FFF789
:101600004BFF039B13F0010FD6D100F05BF8FFF7FF
:101610004BFFFFF7F3FE0028D2D1FFF75FFFCFE7C4
:1016200001A8FFF7F7FE07B05DF804FB37B50E4DD4
:101630002A78202A15D10D4C0D4823680D491844ED
:10164000019278F0C1F823680021019A20330948FB
:10165000297023607DF072FB03B0BDE8304078F064
:1016600091BD03B030BD00BF544500307C45003013
:10167000C0E50D0855450030014B1868704700BFA4
:10168000FCFF1B08014B0248C01A7047C0E50D085B
:1016900000001C0800487047C0E50D0807490022FB
:1016A000074B5B1A9A4201D30120704751F8040B93
:1016B000013001D10432F5E700207047C0E50D0884
:1016C00000001C085A4B2DE9F74F1F680224594BA4
:1016D00007F56A57DFF880911B781837DFF87C81AF
:1016E000554D1F44DFF878A176F07AFFA9EB080B7F
:1016F00006460EB13A2C41D9A9EB0803B3EB070C0F
:1017000024D4DFF860E1661C4C4A0C21F6B2AEEB43
:101710000200614360456FDD681801276A5062442A
:1017200007721F464260DB1B77D445490234454FA0
:10173000E4B2CA1B9A424FF00C0206FB02F266DDCD
:10174000A91801203B44AF5008724B603B2C66D86F
:101750000C2301225C432B191A724FF0FF322A51DD
:101760005A60394B1B782BB1384B1B682B60384BB8
:101770001B686B60304803B0BDE8F08F336AF069D6
:1017800053450ABF334BF31AA3EB0A0380B101930D
:1017900078F0ECF9019B58B122460C2101344A4300
:1017A0000121E4B2A8180172F169A9500D3141601C
:1017B0000C2001211F4400FB04FC5F4505EB0C02DB
:1017C00045F80C6006F13C0C1172C2F804C004EB41
:1017D000010204F10204D2B2E4B200FB02F205EB12
:1017E00002000172316AA95019444160AED23046FC
:1017F00076F006FF06467CE705EB010C4FF001088A
:1018000007446A508CF80880CCF804E08BE7AB18EA
:101810000120AF501872596098E7344696E70123CB
:1018200085F8CC324FF0FF33C5E9B13399E700BFFB
:101830007C45003054450030043D003060430030AA
:101840000000043078C90130003D00308045003090
:1018500078450030003D003000001C08C0E50D0850
:101860000021003078C901302DE9F84F284B064699
:101870000F4690461B7823B3264A0025264BA2EB41
:1018800003090EE0FFF7D2FE022F1CD0042F2BD04D
:10189000012F06D12378715D5A1C22701F4AD15442
:1018A0000135A8450DD01E4B1E4C1B682278043311
:1018B00013444B45E6D3194B4FF0FF32DA61202336
:1018C0002370BDE8F88F2378DFF850A05A1C2270EF
:1018D00032780AF80320FFF7A9FE23785A1C2270F9
:1018E00000220AF80320DBE74FF0000ADFF82CB0F3
:1018F00022783378511C23FA0AF30AF1080A21707E
:101900000BF80230FFF792FEBAF1200FF0D1C7E7D3
:10191000003D003000001C08C0E50D0855450030B2
:101920007C4500305445003070B502680446EFF342
:1019300005811F4DC9B25369D92027F007FE2B78C6
:101940003BB124681CB1204678F010F910B900238F
:101950002B7070BD2046174E78F01CF900F2145021
:1019600084421FD2204678F015F930602046124E8E
:1019700078F024F904F5E053834217D9204678F033
:101980001DF9306000230D4A13600D4A1370FFF7F4
:1019900085FE0028DBD078F0F5FB0120BDE8704023
:1019A00077F08EBFA4F214533360DFE73360E9E7CA
:1019B000003D003080450030784500307C450030E7
:1019C00054450030214B1B7870B5002B3BD0204E86
:1019D000204C33682048214D1A1D21782D1A0A44C5
:1019E000AA4205D31E4A4FF0FF31D1612022227056
:1019F0002278D2B103F120018D4205D81F2A9FBF62
:101A0000174AD3612022227020221549184477F00A
:101A1000DBFE326823780021114813442022217014
:101A200033607DF08BF978F0ADFB33689D4207D9C8
:101A30000B4920220B48CB6177F0C6FE78F0A2FB61
:101A4000002077F03DFF002070BD00BF003D00305A
:101A50007C45003054450030C0E50D0800001C08EE
:101A600055450030E0FF1B080B4B10B50446C0F88D
:101A7000183700F2FC7018F091FC04F5EF6018F0D4
:101A80008DFC064BD4F8AC06C4F8083508B103F059
:101A90005DF8204610BD00BF78980C08104C0D086A
:101AA00070B5002504462C3000F8045C04F28C5616
:101AB00018F0F2F904F1500005F092FDFF2304F54F
:101AC000EE7084F8D83103F043F804F53F7022F04B
:101AD0007BF904F54F7013F07DF80023012284F8A0
:101AE000A05304F56A7004F5A565C4E9E42327F062
:101AF000B5FD04F1180104F580600CF045F9294B9F
:101B0000C4F80835284614351CF030FFB542F9D129
:101B10001E2340F2CC60C4F8B0360023A4F8B436DB
:101B200003F012F8C4F8AC0604F5D76024F0FAFD0F
:101B300004F2FC6024F0F6FD1B4B1A6812B904F5A0
:101B4000A1621A60194B04F5E36004F532651426AE
:101B5000C4F808350AF044F9154B164818600023FC
:101B600099B2013306FB0102127C002AF8D1124B14
:101B70001980124B1980124B1A6812B1114827F0C4
:101B800023FD64224FF4FA7104F535601D6018F0EE
:101B9000CFF80D4B1A680AB10C48F0E720461C60DC
:101BA00070BD00BF104C0D0804A00030EC580C08AC
:101BB000109800302C5B0C080C980030E497003033
:101BC000B8970030F4240C08844500300F250C0829
:101BD0007FB55F4D044678F0C1FA10212B68986BF1
:101BE00003685B6898472B68C4F8700B0221186D76
:101BF00003685B689847D4F8700B03681B699847C3
:101C0000F1EE007AB4EEE70AF1EE10FA40F19B80B3
:101C1000504876F09BF9504B504E0221D3F890205B
:101C2000D2F8043843F00203C2F804382B68186D68
:101C300003685B68984740F29A422021304672F070
:101C4000C3FF80234FF480523383454B5A8378F08F
:101C500099FA0321286822F085FD036880224FF459
:101C6000E131DE6A4FF48073B047204600F05CFC3F
:101C700004F12C0678F086FA204601F069FA78F033
:101C800081FA1FF023FC19F027FA304618F034FAD5
:101C90001FF01CFC1CF09EFE1FF018FC1CF0ACFE9C
:101CA0001FF014FC2F4A062119F04AFA78F06AFA5C
:101CB0009C222D4904F580600CF044FD2B492C48F2
:101CC0004B6902930B6901934B7E00930B7ED1E924
:101CD000021224F08BFE2B68586D03685B689847EE
:101CE00010B1244824F082FE4FF47A7104F5E360C9
:101CF0000BF0D2FC94F9503053B194F828303BB932
:101D00000423314604F15000C4F88C3005F0B6FCD1
:101D100004F5EE7003F076F92B68D86C03681B6845
:101D200098472B68D86C03681B6D984704F54F7073
:101D300013F08EF804F56A7027F09EFC04B0BDE83D
:101D4000704027F087BC2B6801225B6C1A717EE71C
:101D5000C045003090A301301497013000040258B0
:101D60000010025830250C08DC490C084003040818
:101D70004B250C0872250C080148FFF729BF00BF4E
:101D8000C8450030F0B52DED028B90F8A0338BB034
:101D9000002B5DD1304E27F05DFC02463368C31A3C
:101DA000632B55D92D4B04AD03F118071868083380
:101DB00053F8041C2C46BB4203C42546F6D12848E0
:101DC0000024326013F0FCF807EE900A9FED257AAC
:101DD000254DF8EEE77A87EE878A2B780AAA234406
:101DE000013403F0070303EB4303134413F8162CE9
:101DF00007EE902A13F8172C13F8183CF8EEE77A40
:101E000067EE887AFCEEE77ACDED017A07EE902A4C
:101E10009DF80420F8EEE77A67EE887AFCEEE77A20
:101E2000CDED027A07EE903A9DF808100023F8EE07
:101E3000E77A67EE887AFCEEE77ACDED037A9DF8D3
:101E40000C0013F04BF8042CC7D12B7801332B7006
:101E50000BB0BDEC028BF0BD8845003030230C0880
:101E6000044900300000C8428C4500302DE9F341A0
:101E7000144C154E2046DFF8608078F093F8134A32
:101E800001461348121B134F01F0D2FC76F0A8FB59
:101E90000446A4B1206AE169B042019114BF251A39
:101EA000A8EB060578F07EF8019902462B463846E5
:101EB00001F0BEFC204676F0A3FB0446E9E702B041
:101EC000BDE8F08100010030002100300021003029
:101ED00090250C089A250C08003D003008B590F8B4
:101EE000383363B1002380F8383321F08BFF22F0C0
:101EF0003BF821F069FDBDE8084022F03DB808BD7F
:101F000010B5094C15F0FAFC002105222368186D64
:101F10000368DB69984723682821186D0368BDE8CA
:101F200010405B68184700BFC04500302DE9F04FF6
:101F3000002587B080460F462C4EAA46DFF8B490A5
:101F4000002FE9B201DBAF4248D1D9F8000022F0FE
:101F500009FC0446002841D003689B6B9847002881
:101F60003CD0236820461B699847B0F57A7F28BF8C
:101F70004FF47A708346BBF1010B2FD31C4BEC4618
:101F800003F1180E1868083353F8041C62467345B1
:101F900003C29446F6D1236820465B69984783B212
:101FA000FF2BE8D83388162B05D806AA1A4412F955
:101FB000182C824202D0A6F800A0DCE701339BB2C5
:101FC000172B3380D7D14046FFF79AFFD9F800305E
:101FD0000121186D03689B6B9847CCE701350236E9
:101FE0000A2DADD107B0BDE8F08F00BF8E4500309F
:101FF000AC250C08C045003030B50446D0F8700B55
:1020000097B003681B699847F1EE007AB4EEE70ACF
:10201000F1EE10FA04DD384B01221B685B6C1A717B
:1020200021F0C4FD94F92B3053B1582200216846A9
:102030007CF084FE03F042FB6A46304903F028FA44
:1020400027F008FB2E4A05461368C31AB3F57A7FBA
:102050000ED9106000212046FFF768FF1FF036FA06
:10206000002120F091FA1FF031FA042120F08CFABF
:102070000BF0ECFB234A41F288311368EB1A8B42D8
:1020800006D9016821B1156002891F4801F0D0FB13
:1020900094F91030012B0AD11C4A41F2883113689F
:1020A000EB1A8B4203D920461560FFF7DFFE184A72
:1020B0001368EB1A132B0CD904F54F70156012F04E
:1020C000DBFE1FF003FA1EF0A9FE1FF0FFF921F05E
:1020D000AFF804F580600CF03DF8204601F0E6FB17
:1020E00094F828302BB9204617B0BDE83040FFF7F0
:1020F00049BE17B030BD00BFC0450030C4250C0834
:10210000A4450030AC450030D1250C08A84500306E
:10211000B04500300148FFF76FBF00BFC845003031
:1021200038B5054B0A4601461C68236820461D68E1
:10213000024BA847002038BDC0450030B4450030F0
:1021400010B50A4C2046FFF7ABFC094A0949204666
:1021500078F004FF24F042FE074B084A1860084953
:102160000848BDE8104022F0F5BA00BFC84500306D
:10217000CC360130691A0408C04500301521040826
:10218000791D0408B44500300020704770470000F6
:102190007047000070470000704700000020704743
:1021A00000207047002070470120704770470000F2
:1021B00000207047002070470020704700207047C3
:1021C00000207047002070470020704770470000D3
:1021D00000207047C82070470120704700207047DA
:1021E00000207047704700000120704700207047B2
:1021F000012070477047000001207047022070479F
:1022000000207047002070477047000070470000B2
:102210000020704703207047014B187F704700BFB4
:10222000C84500307047000008B50B4B0A211B68F9
:10223000186D03685B6898470848FFF761FEBFF3B5
:102240004F8F0749074BCA6802F4E0621343CB6023
:10225000BFF34F8F00BFFDE7C0450030C8450030D9
:1022600000ED00E00400FA0508B51BF0E7F840F0C7
:10227000200008BD13B54FF43C70CDE9002102F0F9
:1022800059FC044648B1DDE900211FF041FD044B33
:1022900023604FF0FF33C4F8F031204602B010BD88
:1022A0002C590C0810B5044602F04AFC204610BD1B
:1022B00008B590F884308B4208D20BF0C7FA5C2244
:1022C0004FF480210BF0AEFA002008BD223150F807
:1022D0002100FAE708B590F884308B4208D20BF061
:1022E000B5FA55224FF480210BF09CFA002008BD6E
:1022F000223150F82100FAE7F0B5CA78C5B00023C2
:102300000446062A01F10C0102A8029328BF062206
:10231000ADF80C307CF0EAFC029DD4F8E8319D4227
:1023200002D91D4801F084FAD4F8F031002B31DBDA
:1023300004F5FA7703F0C2F9FC262A460023D4F804
:10234000F01103F095F803F0B9F9FC233A46D4F8FC
:10235000F01103F05FF80023324639460DF1120008
:10236000ADF80E31B5FBF6F5ADF810507CF0BEFCC3
:10237000FF23DF228321207CCDE9003204AA19F05B
:1023800083FDD4F8E821BDF810100448B2FBF6F242
:1023900001F04EFA45B0F0BDE0570C08FA570C08B2
:1023A0002DE9F043CA7897B000240646092A8846EA
:1023B00003A801F10C0128BF09228DF81440CDE9D2
:1023C00003447CF093FC9DF81030222B7CD1D6F88E
:1023D000F031013362D103F071F93D4923462246C1
:1023E00002F0E0FFA0420146C6F8F00105DA3948E4
:1023F00017B0BDE8F04301F01BBA06F5FA7936488C
:1024000001F016FA03F05AF9FC234A46D6F8F01107
:1024100003F000F8B0F1000C2EDD304D06ACD6F81C
:10242000EC710FCD0FC40FCD0FC40FCD0FC495E8C5
:102430000F0084E80F00FB434C4609EB0C0014F836
:10244000012B16AD82EA0301A04201F00F0105EB5A
:10245000810151F8401C81EA131383EA121202F041
:102460000F0205EB820252F8402C82EA1313E6D1E8
:10247000DB43C6F8EC31C5E703F020F90023D6F8BA
:10248000F0111A4602F0F4FF03F018F902230022BB
:10249000D6F8F01102F0ECFFC6F8E80198F8072032
:1024A00098F808308DF82020F0228DF821300A238A
:1024B000D6E97A01CDE90032CDE9060106AA4CF24F
:1024C0005431307C19F0E0FC17B0BDE8F08300BF58
:1024D00020580C0835580C0855580C0848230C088F
:1024E00038B58A7A05464B7A0C4643EA0223CA7A03
:1024F00053EA024307D04CF2553293420CD1BDE867
:102500003840FFF7F9BE0A7A0648C97901F090F918
:1025100021462846FFF744FF21462846BDE83840BB
:1025200020F0DCBA6C580C0813B5044615F0A6FF71
:1025300014F036FF204615F021FF18B1B4F9003031
:10254000022B0BD021F054FD14F0FCFB02230DF103
:1025500006012046ADF8063016F0DCFD02B0BDE8FD
:10256000104015F0EDBC0000BFF34F8F0549064B3E
:10257000CA6802F4E0621343CB60BFF34F8F00BF21
:10258000FDE700BF00ED00E00400FA05102213B5DE
:10259000002104468DF807207CF0D0FB054B0DF19F
:1025A000070221461B68586D03685B6B984702B0B1
:1025B00010BD00BFC04500302DE9F041ADF54A7DAA
:1025C0000D46002140F2751268AC06460AA8099132
:1025D0007CF0B4FB4FF4C472002120467CF0AEFBCB
:1025E000DFF8088127F036F84FF47A72384B09AFDC
:1025F000B0FBF2F0186093E8070084E8070002F0EF
:1026000095FA037C237402F091FA437C0DF5E17096
:1026100063740323A3742F4B5A6962619A68DB6861
:10262000A261E361FFF7B2FF40F60453D8F814202B
:102630002384002A284B1868284B3CDD0DF2D32157
:10264000CDE90032264B5022406D22F07FF9502117
:102650000DF2D3207CF0D2FF98F91E20394684F881
:102660003201013A204618BF012201F053FE98F9C9
:102670001E3080B2E97E5A1E53425341079307230E
:10268000069300230393AB7E029305F11903019394
:102690000123CDE90470009330460BA3D3E9002356
:1026A0006DF014F8011E02DC0E4824F09FF90DF5C0
:1026B0004A7DBDE8F081009350220B4B0DF2D321EF
:1026C000406D22F043F9C2E79E6AC421818A46EE3A
:1026D0004451003040030408C04500303B5D0C0805
:1026E000345D0C08515D0C08B18D0C08C8450030F4
:1026F0002DE9F04FDFF8B48097B0DFF8B490404692
:102700006DF030F80446002848D00025402205A886
:10271000244F29460495ADF854507CF00FFB94F8F3
:10272000440021F0A7FD211D8DF8540005A894F860
:1027300044207CF0DBFA23681B4E43F0004306F193
:10274000100A049394F847308DF8553026F084FF32
:10275000C71941F100037068B8B1327894F8461097
:102760001141C90711D54A4492F8F822012A0CD127
:10277000026800210393009104A9D2F810B03A46F0
:10278000D8470028039BC8BF012508365645E2D12B
:10279000002DB4D040466CF0E9FFB0E717B0BDE8BB
:1027A000F08F00BF40420F00849100305051003044
:1027B000C84500302DE9F041DC220C46CAB0054680
:1027C000002144487CF0BAFA4FF04053424A1A6064
:1027D000A38A013B9BB2C92B75D8404B0026082227
:1027E00020460093002319466DF004F8721CF3B2E2
:1027F000D1001646A28A013A934209DA03F1405306
:10280000082220461633009300236CF0F3FFEDE717
:102810004FF040531A7D0AB9E27E1A752846002609
:102820006CF0F8FE4FF0405331467D22587509A8F0
:10283000DFF8B08008AF08967CF080FA314681223C
:1028400029A87CF07BFA98F91E20394629A8013A7C
:1028500018BF012201F0B8FE98F91E3080B203962D
:102860005A1E1F4E5342534107930723CDE904706C
:1028700006932846A37E029304F1190301932823AB
:102880000093E17E332411A3D3E900236CF01EFFF3
:10289000013C14F0FF0408D0FFF72AFF3368012140
:1028A000186D03685B689847F2E70E48FFF728FB4E
:1028B00028466CF0AFFE40F0304040F4002077F046
:1028C000FDFAFFF751FE4AB0BDE8F0812641727271
:1028D000DF25D7B7040000309AAD44C5140000309E
:1028E000C0450030C84500302DE9F0410D46ADF53A
:1028F000876D064677F046FC0AA9284601F0BEFE21
:102900000446002840F0AA804FF4D0720146A6A8E1
:102910007CF014FA9DF8C020102A71D8531E0F2B9A
:102920001FD80DF1C1010DF2D9307CF0DFF922463C
:102930000DF127010DF2D93014F008FF0446002CE8
:102940005ED09DF8C0304BB39DF8303033B39DF866
:102950002720013A032A00F28180DFE802F01628DE
:10296000323B49AA0DF12701BDF82800499416F021
:1029700067F80446002843D001230DF2D93249A953
:102980000093112314F028FED9E7012B66D10E9B8A
:1029900049A920468DF8243116F092FB9DF8273086
:1029A000013B032B5AD8DFE803F01C5D6368012B61
:1029B00054D10E9B49A92046ADF8243116F0C4FB32
:1029C000ECE7012B4AD10E9B49A92046499316F00A
:1029D0000BFCE3E7022B41D10EA9204616F022FBA7
:1029E000DCE701238DF8983294F90030DA17CDE94D
:1029F000A8325C210DF2D9307CF000FE8DF8D803AE
:102A00000024DFF88C8040F26F124AA821464994D6
:102A10007CF094F998F91E2049AFA6A8013A3946EE
:102A200018BF012201F034FF98F91E3080B2E97E10
:102A30005A1E039453425341079307230693AB7ED8
:102A4000029305F1190301930B23CDE90470009360
:102A500030460DA3D3E900236CF038FE0DF5876DE9
:102A6000BDE8F08101238DF89832B4F90030BDE75C
:102A700001238DF898322368B8E702238DF8983245
:102A80002368A893B5E700BFD5A4D139F922B6A72A
:102A9000C845003007B5084968466DF07DFABDF8B5
:102AA000040064235843BDF80030B0FBF3F080B25B
:102AB00003B05DF804FB00BF5051003070B5124EFA
:102AC0000546B46A74B90C21012076F0D7FFB062D4
:102AD00008B9002070BD056084600430FAE726461E
:102AE000A46824B12368AB42F9D1201DF2E70C2180
:102AF000012076F0C3FFB0600028EAD00560B3681B
:102B00009C60B068E9E700BF5091003070B50D4699
:102B100014461E466CF07EFD50B9022E07D1012CE2
:102B200005D12EA3D3E900230120C5E9002370BD00
:102B3000282C2DD00DD8601E83B20A2B16D80A2857
:102B400014D8DFE800F02113133D291313131331B8
:102B50002D0040F24C439C422AD009D840F2264333
:102B60009C4231D040F239439C4225D00020DEE720
:102B700044F625639C422BD044F627639C42F5D152
:102B800018A3D3E90023CFE718A3D3E90023CBE7A9
:102B900018A3D3E90023C7E718A3D3E90023C3E7A9
:102BA00018A3D3E90023BFE718A3D3E90023BBE7A9
:102BB00018A3D3E90023B7E718A3D3E90023B3E7A9
:102BC00018A3D3E90023AFE718A3D3E90023ABE7A9
:102BD00018A3D3E90023A7E7AFF30080401DA1208D
:102BE00026812A0BECFD51169C2A1F639E6AC42184
:102BF000818A46EE26417272DF25D7B7F017304A38
:102C000039059E56D5A4D139F922B6A7CDD269EBA4
:102C1000C51A133B03806A5575F30087C41EDD8B0C
:102C20003CD93120DBC293A716112720011517CB01
:102C30000E03561F3A13328C7423F309F0B5044681
:102C400089B012480E4615461F466CF0E3FCD0B121
:102C500044EA0540FFF732FFA8B10D4B93F91E304F
:102C600000955A1E5342534122460693072305936B
:102C7000BDF83830CDE903731823CDE9010333469D
:102C800002486CF0C9FC09B0F0BD00BF50510030E3
:102C9000C845003010B5C4B0694601F091F8E8B9F4
:102CA000BDF800300E4CB3F5007F0FD1BDF80230F7
:102CB0009FED0C7A07EE903AF8EE677A67EE877A26
:102CC0009FED097A67EE877AC4EDE67ADDE9422363
:102CD000C4E9E42326F0AAFCC4F89C0344B010BD68
:102CE000C84500300AD7233C35FA8E3C00B5CDB03C
:102CF000694600F0DDFF30B9BDF800200DF102019A
:102D0000024804F0A7FF4DB05DF804FB1846003000
:102D10002DE9F0432DED028BB1B006460C466CF068
:102D200079FC804600286BD1237E022B1BD1E38ADD
:102D3000012B18D126F08EFC07460DF0FDFE034650
:102D40004FF4C87007F51677C74DB3FBF0F202FBDE
:102D5000103317FA83F3EB62E77E4FB9C34823F0D1
:102D600045FE85F8307031B0BDEC028BBDE8F083D4
:102D70000EA9204601F0ECFB0AA8FFF707FC9DF81E
:102D80003A400AA90DF13B0022467BF09FFF28B193
:102D9000B74823F02BFE85F83080E4E70F2C0AD8E3
:102DA000EA6A2146B348A2F5167285F83040EA6215
:102DB00023F01CFED7E79DF8381030466CF022FC5B
:102DC0009DF8382095F83210AB4823F00FFEAB4A3F
:102DD00092F90F30002BC6D095F83230A5F580401F
:102DE000013303F0010382F8D8316CF013FC0028A2
:102DF000B9D19DF83810A5F580406CF003FCB2E71E
:102E0000E38A282B00F0BA801ED8013B9AB20A2A26
:102E1000A9D80A2BA7D801A252F823F06B2F0408D7
:102E2000672D0408672D0408F53004088F2F040867
:102E3000672D0408672D0408672D0408672D040812
:102E4000BF2F0408AD2F040840F24C42934200F01B
:102E5000258178D840F22642934200F0338140F237
:102E6000394293427FF47FAFDFF8108201230EA92D
:102E7000204688F8A03301F003FA00287FF473AFEE
:102E8000074608F54F79DFED7E8A9DF83820FBB2C2
:102E90009A427FF668AF30AA484602EB830313F8E4
:102EA000864C13F8855C13F8846CE400AD00F600E2
:102EB00012F086F86428E4B205F0F805F6B237D0CF
:102EC000002835DB07EE900AFF220021B8EEE78AE2
:102ED00007EE904AF8EEE77A28EE288A67EE887ABD
:102EE000FDEEE77A17EE903A18B20DF01DFE07EEF0
:102EF000905AFF220021F8EEE77AC4B267EE887A92
:102F0000FDEEE77A17EE903A18B20DF00DFE07EEDF
:102F1000906AC5B2FF22F8EEE77A002127EE888A90
:102F2000BDEEC88A18EE103A18B20DF0FDFDC6B21B
:102F3000002332462946204611F0D0FF01231F44CA
:102F400088F83833A1E744F62562934200F0CA803E
:102F500044F6276293427FF406AF204631B0BDECC1
:102F6000028BBDE8F043FFF795BE2146304631B0F5
:102F7000BDEC028BBDE8F043FFF71EBB2146304697
:102F800031B0BDEC028BBDE8F043FFF713BC3D4808
:102F900023F02CFD3C4B0A211B68186D03685B680D
:102FA00098473648FEF7ACFFFFF7DEFA2146304679
:102FB00031B0BDEC028BBDE8F043FFF795BC0AA928
:102FC000204601F02DFB00287FF4CDAE9DF828307F
:102FD000012B0FD121F00CF813F0B4FE14F0B0FF68
:102FE00015F04CFA29492A4815F0FCF829492A48D5
:102FF00015F0F8F8DFF88480102200210EA87BF08D
:103000009DFE012398F91E2008AF00250EA8D21AB4
:1030100039468DF8403018BF01220895ADF824508C
:103020008DF8265001F014FB98F91E3080B20395FC
:10303000591E4B424B4107930723CDE90470069379
:103040003046A37E029304F1190301930A230093EF
:10305000E17E03A3D3E900236CF038FB83E600BFD5
:10306000CDD269EBC51A133B50910030785D0C0846
:10307000A35D0C08C45D0C08FB5D0C08C84500305E
:103080000AD7233C175E0C08C04500309C870C080B
:1030900018460030F85F0C08A44700300EA92046FF
:1030A00001F02AF900287FF45EAE204B9DF838101D
:1030B0001B68A1F1FF02586D5142036851411B6822
:1030C000984750E60EA9204601F076F80146002800
:1030D0007FF449AE9DF839300DF13A02144804F0FE
:1030E00041FE40E6204631B0BDEC028BBDE8F04326
:1030F000FFF7FCBD0EA9204601F0B0F900287FF4CF
:1031000032AE0C4D55E9022352EA030109D0DDE944
:103110000E01CDE9000105F1100016F00DFEC5E924
:103120000001D4E9002345E902231CE6C045003034
:10313000184600300851003010B590F818110446B8
:1031400001F054FD6423C0B203FB0044A06F10BD26
:103150002DE9F04F4FF48073484D87B00446AB80A3
:1031600026F078FA4FF47A7305A9B0FBF3F02860E3
:1031700000256388B4F902207F2B41488DF8145054
:103180009CBF404B1A7015F09BFF94F90C30012B3B
:1031900004D165683C4BEB1A5D425D4194F90D30FA
:1031A00004F10C07261D012B03D1A268364B9A426D
:1031B0000DD065B9012305A938468DF8143015F0F6
:1031C00065FF314B05A93046059315F0F5FF2F4BF0
:1031D0004FF0000ADFF8C890DFF8C880039343F28D
:1031E000B0705FFA8AFB01F0A5FC054608B122F039
:1031F0002FFD039BC9F8045043F8045B89F800B025
:10320000039317F8013B87F8EB3288F80430C8F8CD
:10321000005055B194F91E302A68012B316824D131
:10322000D2F800B02846F269D847043609F10809F7
:1032300008F10808BAF1000F14D0002314494FF424
:1032400080420193A1F12800124B0093124B6CF0C5
:10325000B3F90C4B197869B1104807B0BDE8F04FCD
:103260006CF0D0B94FF0010AB9E753682846012243
:103270009847DAE707B0BDE8F08F00BF445100304F
:10328000D64500304051003040420F00949100304C
:10329000785100300D2B0408112D040850510030D6
:1032A00084910030B091003090F869381BB100F57E
:1032B000E36009F0A3BA704770B590F9F13196B0A8
:1032C0000446002B5CD090F8F332002B58D000F568
:1032D000EE75284601F09EFCD4F8246B2846FFF7D3
:1032E0002BFF86424CD094F8F412284601F07EFC65
:1032F0006426C0B206FB004090F80D32002B3FD090
:103300002846FFF719FF94F8F412C4F8240B284656
:1033100001F06CFC2822C5B200210CA87BF00EFD48
:1033200006FB05439FED1A7A0021D3ED927A152210
:1033300003A8029167EE877ACDED097AD3ED937AEF
:1033400067EE877ACDED0A7AD3ED947A67EE877AC5
:10335000CDED0B7A7BF0F2FC0E4B02A909A893F994
:103360001E20013A18BF012200F062FD02AB80B2BC
:1033700040F2E932009004A1D1E90001FFF75EFCC0
:1033800016B070BDAFF30080F2C20B46A9D4A7E21D
:103390006F12833AC84500302DE9F04100F1500723
:1033A000ADF5227D002504460DF1220209A938461B
:1033B0000995ADF8225004F02DFC002850D0BDF83E
:1033C0002260002E4CD0DDF82480B8F1000F47D0E9
:1033D00029464FF497720AA87BF0B0FC324641466A
:1033E000ADF828600DF12A0056AEDFF8A4807BF01E
:1033F0007DFC29464FF4957257A835607BF09EFC02
:1034000098F91E2031460AA8013A18BF012200F09F
:1034100029FC94F9D83185B2591C25D0012B23DC25
:103420001948FFF74BFB98F91E3003965A1E53427A
:1034300053410122069394F9D8319A401823D2B20D
:10344000CDE9010344F625631048CDE90452009309
:103450000BA3D3E900236CF0DFF8384604F0EEFB51
:103460000DF5227DBDE8F081334644F625620095D6
:1034700003A1D1E90001FFF7E1FBEEE7AFF3008024
:103480003A13328C7423F3093A1337CE505100307B
:10349000C845003030B595B00025503005AB02AAC4
:1034A00006A90695019304AB009303AB04F08CFBD3
:1034B0001E4B069C1A68A24230D0182229460EA83C
:1034C0001C607BF03BFC4FF47A7310222946A4FB6E
:1034D000034308A80795CDE90C43029B0F93039B78
:1034E0001193049B1293059B109301238DF83830A0
:1034F0007BF024FC0E4B07A90CA893F91E20013A7F
:1035000018BF012200F0FEFB07AB80B244F6266232
:10351000009004A1D1E90001FFF790FB15B030BD88
:10352000AFF300807844F995F27A72A1AC91003043
:10353000C8450030F0B500F150050446ADF5277DD3
:10354000284605F04FF82046FFF726FF2046FFF7F4
:10355000A1FF94F87061D4F8282B04EB0613D3F87C
:10356000AC309A4200F03481C4F8283B4FF4D0725A
:1035700000213EA87BF0E2FB94F8D23133B9B023AE
:1035800003FB064393F8B930012B0CD894F8487B21
:103590004FB926F053F800220023CDE93E01CDE9D2
:1035A0004023002313E001233146284684F8483B9A
:1035B00004F0D6F8CDE93E0194F87011284604F0E5
:1035C0002BF950EA0103CDE94001EAD002238DF83E
:1035D0000831B0230A2203FB064103FB0656D1F84B
:1035E000D0009C3680FB0207CDE94407D1F8CC001F
:1035F00080FB0207CDE94607D1F8C8004243CDE978
:103600004822D1F8EC2094F870114A92726803FBBA
:1036100001434B92B2684C9293F8EA208DF8342122
:1036200093F8B92094F8D23153B9062A0DD8DFE8BF
:1036300012F007000700D200D600D800DE00E30039
:1036400000238DF83531ADF83631062303AA28461C
:103650008DF8383104F06CF838B1DDED037A67EE9F
:10366000A77ACDED507ACDED4F7A04AA94F8701177
:10367000284604F067F828B1DDED047A67EEA77AF2
:10368000CDED517A05AA94F87011284604F046F859
:1036900048B1DDED057A67EEA77ACDED547ACDED30
:1036A000537ACDED527A00265C4FDA2207A83146D4
:1036B00006967BF043FB97F91E2006A93EA8013A27
:1036C00018BF012200F06EFC06AB80B240F2274228
:1036D00000904CA1D1E90001FFF7B0FA2022314659
:1036E0003EA87BF02BFB94F87031B022DFED4C6AE2
:1036F00006A93EA802FB0343B3F8E620B3F8E8307E
:1037000007EE102A97F91E2007EE903AB8EEC77A16
:10371000013AF8EEE77A18BF012227EE267A67EE23
:10372000A67A8DED407ACDED417ACDE90666CDE9F8
:10373000086600F0C1FB06AB80B240F22542009063
:1037400032A1D1E90001FFF779FA94F87011284607
:103750004096CDE93E6604F019FC94F95E308DF890
:10376000FC003BB1284604F021FC18B9409B43F013
:10377000010340939DF8FC3043B104A9284604F0AE
:10378000DDFA18B9409B43F00203409305AA94F870
:103790007011284604F01AFC08B1059B3E9397F976
:1037A0001E20002306A93EA8013A0693ADF81C305E
:1037B00018BF01228DF81E3000F0E6FA06AB80B289
:1037C00044F62362009013A1D1E90001FFF736FA15
:1037D0000DF5277DF0BD02228DF8352133E7032258
:1037E000FAE703238DF8353140F201132BE7032369
:1037F0008DF83531022326E703238DF835314FF458
:10380000817320E75F43370F00E741CAD2BFDBC3B4
:10381000C4BDE89B697F00BBABB43CBAC84500306F
:103820000AD7233C90F950300BB1FFF783BE7047A5
:103830000FB430B5C3B07C22002146AC23A854F8A5
:10384000045B7BF07BFA0021772205A804917BF0D2
:1038500075FA23462A465A210DF1AE00039423F04F
:1038600073F8114B5A2804A993F91E2028BF5A2037
:10387000013A8DF8AD0023A818BF012200F024FE04
:1038800004AB80B243F6FF72009005A1D1E90001BC
:10389000FFF7D4F943B0BDE8304004B0704700BF33
:1038A000759D040C8EA454D6C84500302DE9F04710
:1038B0002DED028BB0B0064625F0CCFE834A0746BC
:1038C0001368C31A322B09D9814B1B7833B1814954
:1038D00010600B78013303F01F030B707E4D25F051
:1038E000A5FEEB6A98420AD9A5F58040DFF8E08191
:1038F0006BF090FE002861D0002388F80030774AF2
:103900001368FB1AB3F57A7FC0F01781176025F0B2
:10391000A3FE02460B4672486BF032FFFFF7BAF87F
:10392000462804D96F4B7048197823F05FF8FFF7E9
:10393000B1F8462804D96B4B6B48197A23F056F836
:1039400025F074FE4FF47A73684DDFF8C881B0FB40
:10395000F3F0674B28601F68786D03685B6E9847CB
:1039600098F91E201EA92881013A284618BF012275
:1039700000F082FD1EAB80B240F2551200904FA1C4
:10398000D1E90001FFF75AF998F90E40002C00F038
:10399000C9800023E4B21EA908F10E008DF878302A
:1039A00015F08EFB2A2C6AD1524C2046FFF740FFBF
:1039B000386D642103685B689847F6E725F04AFE96
:1039C00098F8003004462BB1FFF764F801464A48E6
:1039D00023F00CF80DF0B0F84FF4C873B0FBF3F21D
:1039E00002FB130304F5167095F8302010FA83F0EB
:1039F000424B1B78E8625B00DBB28DF8303052B985
:103A000043F001038DF8303095F83230013303F084
:103A1000010385F832301EA8FEF7B8FD95F8301086
:103A20001EAB0DF13100C1F110041944E4B2062CB3
:103A300028BF062422467BF059F90023012228489A
:103A4000069395F83230144402FA03F3E4B2DBB281
:103A5000049405930CAB039318230293284BCDE9F0
:103A6000002318A3D3E900236BF0D6FD011E02DA70
:103A7000244822F0BBFF002385F830303FE72B2C91
:103A800004D12148FFF7D4FE204B98474FF4FA6148
:103A90001EA820F09DFE386D4FF47A7103685B68B4
:103AA0009847786D0368DB6A9847A8B3012800F04F
:103AB000B480174831E000BFAFF30080F1C6A7C162
:103AC000D068080F401DA12026812A0BA491003048
:103AD000D43F0030A891003050910030A0910030C8
:103AE00050510030849100308A5E0C0844510030FF
:103AF000C0450030B45E0C08245E0C084051003014
:103B00009C910030595E0C08C55E0C0838ED00E051
:103B1000005F0C08C84500304848FFF789FE1EA822
:103B200020F062FE00236B7125F094FD47F23053C4
:103B3000984202D9424876F0C1F996F8283013B974
:103B40003046FFF76FFE3046FFF7B6FB3046FEF714
:103B5000C5F996F8283013B93046FFF7A5FBFEF7F4
:103B6000C7FD384C00210225374E4022374F0DA8A3
:103B70000C91ADF874107BF0E1F89FED2E8B54F8AA
:103B8000043C002B4DD014F8083C334493F8F892D1
:103B9000B9F1010F45D154F8040C4FF000088DF82D
:103BA00024900DF125028DF8258009A903688DED7B
:103BB000008BD3F808A04346D0479DF8243083B348
:103BC000414648221EA87BF0B9F854F8040C0AAA12
:103BD0000CA90368D3F814800DF12603C047002810
:103BE0001FDD9DF8740020F061FB9DF875300246E2
:103BF0000DA98DF8BC001FA88DF8BF307BF076F8BA
:103C00000C9B1EA938461E9314F8083C8DF8BD3055
:103C1000DDE90A236BF07AFFBDE70D487DE701255A
:103C2000ADE7012D04F10804F9D130B0BDEC028BF1
:103C3000BDE8F0870000000000000000D55E0C0821
:103C4000263A09B08C910030C84500305051003000
:103C5000EA5E0C08024B012283F83220704700BF55
:103C600050910030F8B50E46144605464FF4977251
:103C7000002130467BF062F87CB9214609242B46AE
:103C8000092230466BF0FAFE0122571C2B88013ABC
:103C90009A4204D3E01DC008F8BD0024F4E70822CE
:103CA0002146EB1930466BF0E9FE08343A46ECE762
:103CB000F7B5037F05460E46A3B9092400910922F2
:103CC00019466BF097FD01235F1C3288013B9A4235
:103CD0000CD80734AB8AB3EBD40F14BF01200020FB
:103CE00003B0F0BD838A00240B80ECE7F319214672
:103CF00008222846009300236BF07CFD08343B46E5
:103D0000E2E7000073B50C46142605460021324652
:103D100020467BF013F82B462046382200216BF01A
:103D2000ADFE05F108032046012238216BF0A6FE06
:103D300005F10C032046202239216BF09FFE05F18E
:103D400010032022592120466BF098FE95ED050ABC
:103D50006CF02AF90DF1060310227921ADF8060066
:103D600020466BF08BFE95ED060A6CF01DF90DF107
:103D70000603ADF806001022204689216BF07EFE76
:103D8000304602B070BD000013B50446084600215D
:103D90002022234601900160C0F803106BF06EFEF4
:103DA000231D0198012220216BF068FE019804F187
:103DB0000803172221216BF061FE072002B010BD1D
:103DC000002308222DE9F3410C46009119460546CF
:103DD0006BF010FD631C0822002604F1020800931A
:103DE0001146002328466BF005FD6378F7009E42DC
:103DF00007F1100111D304F58474002340222846F2
:103E0000009457376BF0F6FCAB8AB3EBD70F14BFB7
:103E10000120002002B0BDE8F08108EB0603082273
:103E200028460136009300236BF0E4FCDDE7000038
:103E30002DE9F74305460E4600241746A8461922E9
:103E4000002130467AF07AFFB8EC010A6CF0ACF849
:103E500021461034ADF806000DF10603102230465D
:103E60006BF00CFE302CEFD13FB92146342405F124
:103E70000C03042230466BF001FE05F110094FF0EF
:103E800000082B7B04EB0817984504D3F81DC008E5
:103E900003B0BDE8F083B9EC010A08F101086CF049
:103EA00083F80DF10603ADF80600102239463046BE
:103EB0006BF0E4FDE5E7000073B50C4610260546FF
:103EC0000021324620467AF039FF95ED000A6CF069
:103ED0006BF80DF1060332460021ADF806002046CE
:103EE0006BF0CCFD95ED010A6CF05EF80DF1060368
:103EF00032463146ADF8060020466BF0BFFD95ED29
:103F0000020A6CF051F80DF1060332462021ADF89B
:103F1000060020466BF0B2FD95ED030A6CF044F804
:103F20000DF1060332463021ADF8060020466BF055
:103F3000A5FD95ED040A6CF037F80DF10603324645
:103F40004021ADF8060020466BF098FD95ED050A7E
:103F50006CF02AF80DF1060332465021ADF8060048
:103F600020466BF08BFD95ED060A6CF01DF80DF107
:103F700006033246ADF80600602120466BF07EFD58
:103F800005F11C032046072270216BF077FD2046C7
:103F900005F11D03062277216BF070FD304602B05B
:103FA00070BD00002DE9F04F0C46054685B000219C
:103FB00091462046DE2205F1440A7AF0BFFE2B46E8
:103FC00038220021204600276BF058FD382205F1E9
:103FD0000803204611466BF051FD05F11003032242
:103FE000702120466BF04AFD05F111030822802163
:103FF00020466BF043FD05F1180325228821204659
:104000006BF03CFD05F120032522AD2120466BF02D
:1040100035FD05F128031B22D22120466BF02EFD31
:1040200005F12C031B22ED2120466BF027FD05F145
:10403000300320224FF4847120466BF01FFD05F100
:10404000340320224FF4947120466BF017FD05F1E4
:10405000380320224FF4A47120466BF00FFD05F1C8
:104060003C0306224FF4B47120466BF007FD05F1C6
:104070003D0302224FF4B77120466BF0FFFC05F1BF
:104080003E0304224FF4B87120466BF0F7FC05F1B3
:104090003F0306224FF4BA7120466BF0EFFC05F1A6
:1040A000400306224FF4BD7120466BF0E7FC4FEA57
:1040B000071895F8403008F5C0719F4208F5C8769A
:1040C000019125D395ED350A6BF06EFF0DF10E03CE
:1040D000ADF80E001022019920466BF0CFFCB9F12B
:1040E000000F08D1314608F2911605F1D8030122DC
:1040F00020466BF0C3FC05F586774FF0000A95F873
:10410000D8309A4513D3F01DC00805B0BDE8F08F34
:10411000BAEC010A01376BF047FF0DF10E03ADF861
:104120000E001022019920466BF0A8FCBFE7A7F112
:104130002C0B06F16008B146494609F120095B469F
:10414000202220460BF1040B6BF098FCC845F3D1FC
:10415000A7F11C0906F1CC0B414608F124084B4697
:104160002422204609F108096BF088FCC345F3D1ED
:1041700006F1D201B946D8364FF000083B1F06229F
:1041800020466BF07BFC17F8043C984503D30AF1FA
:10419000010AC037B3E7B9EC010A08F101086BF076
:1041A00003FF3146ADF80E000DF10E03102220463C
:1041B00010366BF063FCE6E70023F7B5047F0E468C
:1041C00000910822194605466BF014FBBCB9731C1C
:1041D0000822284600932346102411466BF00AFB60
:1041E00001235F1C7278013B9A420FD80734AB8AD7
:1041F000B3EBD40F14BF0120002003B0F0BDAB8A95
:104200000824DB00083BDB087370E9E7F31921465B
:1042100008222846009300236BF0ECFA08343B4652
:10422000DFE70000F7B50C46154600920023082290
:10423000096806466BF0DEFA21686F1C0023052230
:10424000083100973046AF1C216003356BF0D2FA7D
:1042500021680023062205313046009721606BF06B
:10426000C9FA2168002305220631304600952160F5
:104270006BF0C0FA23680533236003B0F0BD000083
:10428000F0B5002385B0057F06460C46039375BB49
:104290002B460091052229466BF0ACFA039B671C64
:1042A0000533039323789D4217D23A4603A930463B
:1042B00001350437FFF7B6FFF4E7227803A930464B
:1042C00017FB02522244FFF7ADFF2378013323701E
:1042D000B28A039BB3EBC20FEFD1039BB28A0733C1
:1042E000B2EBD30F14BF0120002005B0F0BD0427AE
:1042F00001250B70ECE700000023082213B50446EB
:10430000009119466BF076FAA08A013818BF012097
:1043100002B010BD2DE9F0470D460446002190463D
:10432000284640F279127AF009FD23462022002126
:10433000284604F122076BF0A1FB231D0222202155
:104340002846C0266BF09AFB631D032222212846D3
:104350006BF094FBA31D0322252128466BF08EFBF6
:1043600004F108031022282128466BF087FB04F192
:1043700010030822382128466BF080FB04F111035A
:104380000822402128466BF079FB04F11203082231
:10439000482128466BF072FB04F1140320225021BF
:1043A00028466BF06BFB04F118034022702128466D
:1043B0006BF064FB04F120030822B02128466BF067
:1043C0005DFB04F121030822B82128466BF056FB5F
:1043D000314608363B460822284601376BF04EFB33
:1043E000B6F5A07FF4D1002704F1330A04F13203BB
:1043F0000822314628466BF041FB94F832304FEAF0
:10440000C7099F4209F5A47615D3B8F1000F08D16A
:10441000314609F24F1604F59973072228466BF0CE
:104420002DFB27463B1B94F8322193420CD3F01D01
:10443000C008BDE8F0870AEB07030822314628468A
:1044400001376BF01BFBD8E707F233133146082224
:104450002846083601376BF011FBE3E700233822CA
:1044600013B50446009119466BF0C4F9A08A0738C9
:1044700018BF012002B010BD13B504460846002144
:104480002022234601900160C0F803106BF0F6FA79
:10449000231D0198022220216BF0F0FA631D019880
:1044A000032222216BF0EAFAA31D019803222521A1
:1044B0006BF0E4FA019804F10803102228216BF054
:1044C000DDFA072002B010BD2DE9F0410E46054689
:1044D0000021174630467B227AF030FC2B4603221F
:1044E000002130466BF0CAFA6B1C052203213046CE
:1044F0006BF0C4FA0123DC0003F101086A78013B88
:104500009A4212D83FB92146073405F12103072208
:1045100030466BF0B3FA2F467B1B95F8212093426F
:104520000CD3E01DC008BDE8F08105EB08030822AC
:10453000214630466BF0A2FA4346DCE707F122033E
:10454000214608223046083401376BF097FAE3E73A
:104550000023F7B50C46067F072200911946054651
:104560006BF048F9631C01220721009328460023C1
:104570006BF040F9B6B9A31C052208212846009328
:1045800033460D266BF036F92746A2783B1B9A423C
:104590000FD80736AB8AB3EBD60F14BF012000202B
:1045A00003B0F0BDAB8A0826DB00083BDB08A37034
:1045B000EAE7FB1C31460822284600930023083610
:1045C00001376BF017F9E0E7F8B50E4605461446DB
:1045D0000021812230467AF0B1FB2B4608220021CF
:1045E00030466BF04BFA7CB90F246B1C0722082174
:1045F00030466BF043FA01235F1C6A78013B93421B
:1046000004D3E01DC008F8BD0824F4E7EB192146E7
:10461000082230466BF032FA08343B46ECE70000E3
:1046200037B50C4600230546009108341946082288
:104630006BF0E0F8012330220821284600946BF04B
:10464000D9F8A88A073818BF012003B030BD000090
:1046500038B50C4600210546034621602046C4F8C3
:10466000031030226BF00AFA204605F108030122FC
:1046700030216BF003FA072038BD00002DE9F0432C
:10468000002385B00D4690F81C800D22009119463C
:1046900006466BF0AFF80DF10F0303220D210093D6
:1046A000304600236BF0A6F89DF80F302B72013BCB
:1046B000032B5DD8DFE803F00229343F05F1100336
:1046C0005024402210210093304601236BF092F8D1
:1046D000B8F1000F4ED105F19803214607340722A7
:1046E0000093304643466BF085F82F4695F89820A6
:1046F0007B1B9A4245D80734B38AB3EBD40F14BF5F
:104700000120002005B0BDE8F08305F11003202250
:10471000102130460093012330246BF06BF8D7E76B
:1047200005F11003082210213046009300231824BD
:104730006BF060F8CCE705F11003002705F11109D3
:10474000082200931021002330466BF053F82B7C95
:10475000FC009F4204F11804BAD209EB07030822B7
:10476000214630460093002301376BF043F8EEE713
:104770001024ADE7B38AC4EBC303DB0885F8983097
:10478000B3E707F19903214608223046009300233E
:10479000083401376BF02EF8A8E7000073B51378E2
:1047A0000C46154609688DF8073002220DF1070303
:1047B00006466BF063F92168023121602B78012BEA
:1047C00003D0022B0BD002B070BD05F108034022CC
:1047D00030466BF053F9236840332360F3E705F16B
:1047E0000803202230466BF049F923682033F4E7B0
:1047F000F7B513780C46154609688DF80730032283
:104800000DF1070306466BF039F921680331216089
:104810002B78013B032B0CD8DFE803F0020D161FA9
:1048200005F10803402230466BF028F92368403335
:10483000236003B0F0BD05F10803202230466BF081
:104840001DF923682033F3E705F1080308223046F9
:104850006BF014F923680833EAE705F1080308222E
:1048600030462F466BF00AF92368083323602A7A12
:104870007B1B9A42DDD907F10903082221683046E3
:104880006BF0FCF82368013708332360EFE7000082
:10489000F7B50D4604461646002140F2731228462D
:1048A0007AF04CFA0523224601A928460193FFF726
:1048B0009FFF019B04F1900201A905332846019353
:1048C000FFF796FF019B04F5907201A92846063375
:1048D0000193FFF763FF019B04F5987201A9284635
:1048E00006330193FFF75AFF4EB904F5A073072270
:1048F000019928466BF0C2F8019B0733019300260B
:1049000004F2411794F8403101999E4203D30731D4
:10491000C80803B0F0BDBB190822284601366BF069
:10492000ADF8019B08330193ECE7000010B5044695
:104930000846636B6BB9616359B10B689B6B984711
:1049400038B1606B04F110010368BDE81040DB680A
:104950001847002010BD000030B5837A87B00446A8
:10496000C172A3B90B4A04941268106D0268156DE8
:10497000094A02930423059206AA0193238900930E
:10498000636812E90600A84708B10123A37207B0C3
:1049900030BD00BFC0450030254B0408064B10B5A4
:1049A000C0E90031054B044602811C3040F80C3C44
:1049B00021F0B8FE204610BD745F0C0800500D08B1
:1049C00070B50E4D04460E462B798B4204D1036818
:1049D00029685B68984740B92B7BB3420DD12368A7
:1049E0002046A9685B68984738B1236800222046B2
:1049F0001B681146BDE87040184770BDB09100308B
:104A0000FFF7DEBF2DE9F0431D46837A85B00446EB
:104A10000E4691461BB9002005B0BDE8F083002387
:104A2000476B8DF80E3001238DF80F303B68D3F8BB
:104A3000088024F011FE10EB090033460DF10F023F
:104A400045EB01050DF10E01CDE900053846C047E3
:104A50000028E0D09DF80F30002BDCD024F0FCFDC6
:104A6000646B084A236882184FF0020000902046C9
:104A70001D6941F100033146A847431E5842584181
:104A8000CAE700BF80841E00254B2DE9F041044693
:104A900098B01D68286D03685B6B9847002838D074
:104AA0000126002524F0CAFD676B10F57A708DF899
:104AB0000C608DF80D504FF000033A6841F1000191
:104AC000CDE9000103A9D2F8088038460DF10D02A6
:104AD000C0470028E6D09DF80C30002BE2D04022E1
:104AE000002107A8ADF80E500695ADF85C507AF09D
:104AF00025F9606B04AA06A903685F690DF10E032E
:104B0000B8470128CED1236806A920469B6898475C
:104B1000C8E7286D012103685B689847BAE700BFC2
:104B2000C045003008B5FFF7AFFF000000487047F0
:104B3000305F0C080121884238BF084674F09EBFE0
:104B400008B174F09FBF7047FFF7F4BFFFF7F8BFDD
:104B500000214FF0FF33002210B54362044600F1FC
:104B6000300301600171F83040F8F31C00F8EF1CCD
:104B700000F8DF1CD970643343F85C2C43F8582CE0
:104B800043F8542C43F8402C43F83C2C43F8382C81
:104B900043F8342C43F8302C43F82C2C43F8282CC1
:104BA00043F8242C43F8202C43F8102C43F80C2C09
:104BB00043F8082C9842DDD1044B1A6822B9044905
:104BC00020461C6013F00EFB204610BDC091003043
:104BD000F85F0C0890F8321029B901234386117050
:104BE0008375184670470020704700004FF00000A2
:104BF0007047000049B1037D012B06D05A1C0433D5
:104C0000027540F823100120704700207047000013
:104C10007047000073B590F915500446002D49D037
:104C200090F81751002D45D090F831600025227D75
:104C3000EBB29A4207D90433013554F823000368D4
:104C40009B689847F3E724F0F1FCA36FC01AB0F516
:104C5000FA7F2CBF00230123B0F5FA7F84F83130AE
:104C60000CD2636A013309D00AF040F8616A09F096
:104C700079FE18B10AF03AF809F05AF894F9F830C8
:104C800013B1002384F8183194F83150AE4211D09A
:104C90000AF02CF84FF6FF7109F064FE50B1002DB8
:104CA00014BF0022042201920AF020F8019A032185
:104CB00009F0DCFD284602B070BD000007B58DED9F
:104CC000010A19B901A9443014F094F903B05DF850
:104CD00004FB000010B504460021383012F0AEFD90
:104CE00004F14C0104F14800BDE8104014F064BA2E
:104CF00030B403460D4600F1380407CA84E80700C3
:104D00002946184630BCFFF7E5BF000007B5343030
:104D10000DF107018DF8072014F0D2F903B05DF80A
:104D200004FB0000024690F9150058B192F81701F3
:104D300040B1114491F9F80020B192F918000338FC
:104D400018BF01207047000090F831201AB190F888
:104D50001811FFF7E7BF104670470000837D13B1BD
:104D60000021FFF7DFBF18467047000090ED070AEB
:104D7000704700002DE9F0412DED088B92B090EDC9
:104D80001B7ADFED5EAA05468DED017AB0EEC77A9B
:104D9000D0ED1C7AB4EEEA7ACDED027AF1EE10FA9B
:104DA00007D5F0EEE77AF4EEEA7AF1EE10FA00F1C8
:104DB000938005F16C060CAC09AF4FF0000830464B
:104DC0009FED4FBA0DF05AFE30460DF095FA12AB3A
:104DD0008DED0F0ACDED100A8DED111A9FED438B6D
:104DE00013E907009FED439B84E8070087E807006D
:104DF00001A80CF06DFA8DED030ACDED040A5FFAFF
:104E000088F1AB7D8B426DD92846FFF78BFF10B937
:104E100008F10108F3E796E8070084E807009DED34
:104E20000C7ADDED0D7A8DED057AB0EEC77ACDED19
:104E3000067AB4EEEA7AF1EE10FA06D5F0EEE77AE9
:104E4000F4EEEA7AF1EE10FA46D405A901A80CF0C6
:104E500089F907A8CDED080A8DED070A0CF014FAC0
:104E60002046F0EE40BA0DF009FE20460DF09CFA07
:104E700005A80CF025FA394620460DF0A9FAB7EE40
:104E8000001AFFEE000A40F601000BF0E5FD77F096
:104E900065F803A9B0EE40AA05A80CF0A7F9B7EE93
:104EA000001AFFEE000A40F602000BF0D5FD77F085
:104EB00055F8B7EECA6AB4EEC86BF1EE10FA0BDC27
:104EC000B7EEC07AB4EEC97BF1EE10FA04DCF4EE72
:104ED000CBBAF1EE10FA9BDD002012B0BDEC088BCE
:104EE000BDE8F0810120F8E7AFF300800000005139
:104EF000FB21F93F0000003652C1F03F00000034B2
:104F000000004843024690F91500B0B192F817012D
:104F100098B1D2ED117A9FED097AF4EEC77AF1EEED
:104F200010FA09D4B7EE087AF4EEC77AF1EE10FA67
:104F3000D4BF01200020704700207047ABAA2A3F51
:104F4000836C1BB10021483012F078BC7047000020
:104F5000014B1868704700BFC091003010B504467F
:104F6000006810B103685B689847204610BD0000D8
:104F700010B50446006810B103685B689847204686
:104F800010BD000030B5D0F8085185B0044615F4C6
:104F9000803520D1184B01A8184A1B68196B0B6883
:104FA0001B6898470C22019B29460DEB02000393D6
:104FB000CDE901553EF0F4FE01462046FFF71AFE0A
:104FC00003A8FFF7D5FF02A8FFF7D2FF019810B1A1
:104FD00003685B689847237D0BB1A37D4BB9064BF3
:104FE00007491B68186C03681B6805B0BDE83040B2
:104FF000184705B030BD00BFC0450030805F0C08C9
:10500000875F0C0810B590F915300446A3B1836C86
:105010000365837D8BB10C4B64211B68186D03689D
:105020005B6898472046FFF7F5FD94F8323003B9E6
:10503000A364012384F8173110BDFFF7A3FFA37DFC
:10504000002BF2D0E7E700BFC0450030804B2DE9D0
:10505000F0472DED068B93ED009AF0EE409A7D4BD4
:10506000F0EE60AA80EE097A8146D3ED006A8846A8
:105070001746F4EEC06AC0EE897AF1EE10FA80F2BB
:10508000DA80BBFE478ABDEEC88A0126B8EEC88A20
:1050900028EE098ABDEEC88AB8EEC88A6E4B93ED39
:1050A000006AB4EEE96AF1EE10FA0CD8BDEEC77AE8
:1050B0000026B0EE498AB8EEC77A99EE078ABDEEAF
:1050C000C88AB8EEC88A654B93ED00AAB4EEEAAA86
:1050D000F1EE10FA80F2B580FBFE678AFDEEE88AF9
:1050E000F8EEE88A68EE898AFDEEE88AF8EEE88A4A
:1050F0005B4B93ED007AB4EEEA7AF1EE10FA0CD83D
:10510000FDEEE77A0026F0EE498AF8EEE77AD9EE6E
:10511000278AFDEEE88AF8EEE88A78EE666A1122C0
:10512000002125254F4CC6EE897AFCEEE77A17EE72
:10513000900A0BF0E9FC38EECAAA8246232200212D
:10514000CAEE097AFCEEE77A17EE900A0BF0DCFC67
:105150007AEEE88A05FB0AFC39EEC88A0AFB055597
:10516000C8EE896A0CEB000104EB8103D3ED007AF1
:10517000431CEA1805449C4404EB850004EB820EB2
:1051800090ED007A04EB8C049EED006AD4ED005A99
:1051900036EE476A344875EEE75A00EB8103A6EE17
:1051A000867A88EE096AE6EEA57ABDEC068B37EEC4
:1051B000677AE6EE077AC9ED007AD3ED007A00EB64
:1051C0008203D3ED005A00EB850300EB8C0093EDD6
:1051D000007A90ED005A304675EEC75A234B35EEF3
:1051E000675A03EB8101A6EEA57A03EB8202E6EE95
:1051F000857A03EB850503EB8C03D2ED005A93ED22
:10520000005A37EE677AE6EE077A95ED007A75EE8A
:10521000C75AA6EEA57AC8ED007AD1ED007A35EE30
:10522000675AE6EE857A37EE677AE6EE077AC7EDDB
:10523000007ABDE8F087BDEEE68A0026B8EEC88A9F
:105240002CE7FDEECA8A0026F8EEE88A50E700BF98
:10525000D8600C08E06B0C08D86B0C08E46B0C08E9
:10526000DC6B0C08DC600C08E86B0C08E4760C08BE
:105270001FB5002302AA01A903A801930293039377
:10528000FFF7E4FE9DED010A05B05DF804FB0000A8
:1052900010B52DED028BD0ED037A96B09FED260A66
:1052A000F8EEE70AD0ED027A9FED248A05AAF8EE1F
:1052B000E77A04A960EE800A06A88DED048A07AC9F
:1052C00027EE800A8DED058A8DED068AFFF7BEFE7A
:1052D000069B242200210DA807938DED088A8DEDF1
:1052E000098A79F02BFDDFED167AB0EE480A9DEDC4
:1052F000041A0DA8DDED050A21EE271A67EEE00A73
:105300000BF092FD21460DA80BF01CFD0AAB8DEDB4
:10531000070ACDED080A8DED091A94E8070083E825
:1053200007009DED0A0ADDED0B0A9DED0C1A16B083
:10533000BDEC028B10BD00BF95BFD633000000004E
:1053400035FA8E3C2DE9F3410F460E6801250D4CD0
:1053500054F8351008460191FBF7E2FF01995FFA16
:1053600080F8304642467AF021F930B9464404EBE1
:10537000C5003E6002B0BDE8F0810135052DE7D1E2
:105380000048F7E7FC810C080B680548B3F5A06FEF
:105390003FBF1A0ADBB200EBC2000B60704700BFD0
:1053A000FC810C0830B585B0CDE9022103A9019339
:1053B000FFF7C8FF044640680168DDE901320D6867
:1053C0000399A847011E09DBFF290ADD606803680D
:1053D0005B68984779F09AFB222303604FF0FF3017
:1053E00005E00448201AC0F3C70001EB002005B017
:1053F00030BD00BFFC810C0807B5019101A9FFF782
:10540000C3FF4068019903685B68984703B05DF883
:1054100004FB00001FB5CDE9022103A90193FFF7AA
:10542000B3FF40680168DDE901328C680399A04749
:1054300004B010BD1FB5CDE9022103A90193FFF708
:10544000A3FF40680168DDE90132CC680399A047F9
:1054500004B010BD07B5019101A9FFF795FF4068A1
:10546000019903681B69984703B05DF804FB0000CD
:105470001FB5CDE9022103A90193FFF785FF40681D
:105480000168DDE901324C690399A04704B010BD01
:1054900007B5CDE9002101A9FFF754FF4068036873
:1054A000DDE900219B69984703B05DF804FB00002B
:1054B00007B5019101A9FFF745FF4068019903680D
:1054C000DB69984703B05DF804FB000007B5019164
:1054D00001A9FFF737FF4068019903681B6A9847E5
:1054E00003B05DF804FB000073B5019101A9FFF75B
:1054F00029FF05460820FFF71DFB044658B16868E0
:10550000019903685B6A98470646606030B9204697
:105510003446FFF715FB204602B070BD02482D1A35
:10552000ED102570F7E700BFFC810C0841B10A7847
:10553000044B496803EBC203586803689B6A184729
:1055400008467047FC810C0838B50C4671B10A78E2
:10555000084B496803EBC20358680368DB6A984745
:1055600005462046FFF7ECFA284638BD4FF0FF35D8
:10557000FAE700BFFC810C0807B5019101A9FFF70C
:10558000E1FE4068019903681B6B984703B05DF822
:1055900004FB000007B5019101A9FFF7D3FE4068A5
:1055A000019903685B6B984703B05DF804FB00004A
:1055B00007B5CDE9002101A9FFF7C4FE40680368E3
:1055C000DDE900219B6B984703B05DF804FB000008
:1055D000014800F0A9BB00BFFC910030014800F079
:1055E000BDB800BFFC91003007B5019101A9FFF7DC
:1055F000A9FE4068019903689B6C984703B05DF869
:1056000004FB00002DE9F34715460F4601A901935D
:105610000026FFF7B9FE013D8046F4B257FA86F93D
:10562000AC4214DAD8F804004A4601990368D3F86A
:1056300008A00123D047002802DC44B920460AE034
:105640003B570D2B03D00A2B06F10106E5D10023B1
:10565000012089F8003002B0BDE8F087054B1B68D7
:105660005B6D93F89C3013B9034800F053B80020E9
:10567000704700BFC0450030FC91003038B50024B1
:10568000054D05EBC4030134586803681B6D98474A
:10569000052CF6D138BD00BFFC810C0838B50024BC
:1056A000054D05EBC4030134586803685B6D9847EA
:1056B000052CF6D138BD00BFFC810C0800487047AE
:1056C000C4910030064B074A1A60074B074A1A601C
:1056D000074B084A1A60084B084A1A60704700BF17
:1056E000FC9100308C840C086892003068850C08AE
:1056F0000492003008850C08C891003040860C08E0
:1057000013289ABF014B18564D2070473C830C0854
:105710007047000030B585B0044640F25E320C4957
:1057200001A801251FF06EF80A4B0B4A1B68039273
:1057300004AA186D0294036812E906009B6A984750
:1057400001A825711FF080F8284605B030BD00BFC4
:1057500000970030C04500306163040807B54FF47E
:105760005572064901A81FF04DF821F001F801A873
:105770001FF06AF803B05DF804FB00BF009700302B
:105780002DE9F04F85B0254C40F6B83102A81FF046
:105790001FF823780BB920F0EBFF21F09BF80546AA
:1057A00078B901230146237003A81FF011F803A85C
:1057B0001FF01AF802A81FF017F8284605B0BDE838
:1057C000F08F0023DFF858B0237010245BF8047BBF
:1057D000EFB13E684FF41472002196F83030304635
:1057E00003F0030A0193D6E90E8979F0A7FA019B29
:1057F000796830469B0748BF4AF0100A52466CF061
:105800007BFA20B942464B4630466CF043FE013CE1
:10581000A4B2002CDAD12146C6E700BFFC960030C6
:10582000BC960030F0B5D3B00E46154601F06CFEC4
:10583000002800F0958040F241224B4968461EF056
:10584000E1FF4A4B1B7873B1FFF79AFF58B979F023
:105850005DF9052303604FF0FF3468461EF0F4FF46
:10586000204653B0F0BD79F051F900234049036060
:105870003046FBF74BFD20B13E493046FBF746FD75
:1058800078B9002300220024C5E90623C5E90A23CC
:10589000C5E90E234FF480436C81AC812C616B60B1
:1058A000DBE70AA930466CF0A3FF0128044612D1B9
:1058B000314B1F68386D03681B6C984718B17B6DBE
:1058C00093F89C3043B9FFF75BFF28B10AA9304633
:1058D0006CF08EFF04463CB179F018F90246E0B254
:1058E000FFF70EFF1060B6E7BDF832200A9B5100AB
:1058F00009942B6101F03E01BDF830300191C2F3F3
:105900004511D20A0291039203F01F020492C3F3DD
:1059100043125B0A013A503305920693CDE90744DE
:1059200014F000FA01A814F07DF99DF8342040F23B
:105930006D1312F0010FC5E90601C5E90A01C5E9B9
:105940000E0140F2FF1108BF0B464FF47A71D206E8
:1059500069814CBF43F4804343F40043A9819EE72F
:105960004FF0FF347CE700BF00970030FC9600301A
:10597000F0BD0D08817F0D08C045003013B50C4601
:1059800001F0C2FDE8B140F281220F4901A81EF0EA
:1059900039FF79F0BBF80023036020466CF0E0FF8C
:1059A000044640B179F0B2F8024620464FF0FF3489
:1059B000FFF7A6FE106001A81EF046FF204602B0C9
:1059C00010BD4FF0FF34F9E70097003013B50C46D7
:1059D00001F09AFDE8B140F28F220F4901A81EF0B4
:1059E00011FF79F093F80023036020466DF034F83E
:1059F000044640B179F08AF8024620464FF0FF3461
:105A0000FFF77EFE106001A81EF01EFF204602B0C8
:105A100010BD4FF0FF34F9E700970030F7B50E46A0
:105A200001F072FD002844D040F2A722224901A8CB
:105A30001EF0E8FE214B1B786BB1FFF7A1FE044678
:105A400048B979F063F80523036001A81EF0FCFE55
:105A5000204603B0F0BD4FF4A870FFF76BF8044682
:105A60000028F2D031466CF027FE0128054612D1FD
:105A7000134B1F68386D03681B6C984718B17B6D1A
:105A800093F89C304BB9FFF77BFE30B1314620468E
:105A90006CF012FE0546002DD7D079F037F802469B
:105AA000E8B2FFF72DFE106020460024FFF748F80B
:105AB000CBE70446CCE700BF00970030FC960030EF
:105AC000C0450030F0B5CBB00D4601F01DFD0028FB
:105AD0003ED040F2C3221F4901A81EF093FE55B9E3
:105AE00079F014F816230360002401A81EF0ACFE20
:105AF00020464BB0F0BD002302A9284685F850305F
:105B00006CF03EFE074610B99DF922303BB978F0A3
:105B1000FDFF02463846FFF7F3FD1060E4E705F1AC
:105B200050040DF12200FBF7FBFB0DF122010646AC
:105B3000024620463CF004FC9DF814302E4413F03D
:105B4000100386F8507018BF012385F84F31CCE759
:105B50000446CDE70097003037B50D4601F0D4FC80
:105B600018B34FF43972124901A81EF04BFE5DB90B
:105B700078F0CCFF162303604FF0FF3401A81EF02D
:105B800063FE204603B030BD28466CF0EFFD0446AE
:105B90002846FEF7D5FF002CF0D078F0B7FF02467C
:105BA0002046FFF7ADFD1060E6E74FF0FF34E8E771
:105BB0000097003030B585B001F0A6FC48B340F244
:105BC000F922164901A81EF01DFE154B1B7883B162
:105BD000FFF7D6FD68B94FF0FF3478F097FF052343
:105BE0002546036001A81EF02FFE2046294605B079
:105BF00030BD02AA03A90B486CF02AFE10B104467E
:105C00000025EFE7029B03985C894443E50D64029D
:105C1000E8E74FF0FF342546E7E700BF0097003084
:105C2000FC960030F0BD0D0830B585B001F06CFC7D
:105C300040B340F20F32154901A81EF0E3FD144BAA
:105C40001B7853B1FFF79CFD38B978F05FFF05234F
:105C500003604FF0FF3425460DE002AA03A90D486A
:105C60006CF0F6FD0028F4D1029BDC6A5B89023CF3
:105C70005C43E50D640201A81EF0E6FD20462946BE
:105C800005B030BD4FF0FF342546F7E700970030F0
:105C9000FC960030F0BD0D0870B5CAB00023044674
:105CA0000D4602A80292039378F036FF018A03465C
:105CB000C26801315E681B8842EA4112416980680E
:105CC000503942EA4121124A02EAC0221148ADF895
:105CD000101000EA46100243204642EA5303ADF892
:105CE000123001F011FC044678B14FF450720A49A9
:105CF00001A81EF087FD02A928466CF07FFFB0FACC
:105D000080F401A864091EF09FFD20464AB070BDD2
:105D100000F8FF07E0FF1F0000970030014820F067
:105D2000C3BC00BF0097003013B501F0EDFB044683
:105D300058B140F24B32064901A81EF063FD20F035
:105D4000C9FD044601A81EF07FFD204602B010BD2B
:105D5000009700300021014820F0B0BC00970030CF
:105D60000F2810B506D978F0D1FE0024092303606E
:105D7000204610BD044B53F82040002CF8D178F099
:105D8000C5FE09230360F3E7BC960030022810B576
:105D900005D9FFF7E5FF044638B9204610BD78F075
:105DA000B5FE092300240360F7E70468002CF4D152
:105DB00078F0ACFE09230360EFE70000F7B5044676
:105DC0001E460F46154678F0A1FE002303602046CC
:105DD00001F09AFB88B340F20E22194901A81EF087
:105DE00011FD3846FFF7D2FF044630B978F08EFE39
:105DF000182303604FF0FF3419E0022FFAD9022E66
:105E000010D103691D442A46EB1720466CF042FB73
:105E1000054658B178F07AFE02462846FFF770FC36
:105E20001060E7E7012EEED1836BEBE7A46B01A8CE
:105E30001EF00AFD204603B0F0BD4FF0FF34F9E735
:105E4000009700302DE9F3470F4616461D4601F036
:105E50005BFB00284DD040F28D12274968461EF0AA
:105E6000D1FC264B1B7833B1FFF78AFC18B978F0C8
:105E70004DFE05230EE00DB100233370002478F0B1
:105E800045FE04603846FFF781FF074620B978F0E9
:105E90003DFE0923036017E0A146B5F5805FAA46E1
:105EA00001AB314628BF4FF4805A3846CDF80490F4
:105EB00052466CF081F8804648B178F027FE0246E1
:105EC0004046FFF71DFC10604FF0FF340AE0019BD5
:105ED00043B15345CBD81C441E44A5EB030501D365
:105EE000002DDAD168461EF0AFFC204602B0BDE8B6
:105EF000F0874FF0FF34F8E700970030FC96003051
:105F00002DE9F04F85B005461E460C46174678F041
:105F1000FDFD00230360284601F0F6FA002869D051
:105F20004FF4E072354902A81EF06CFC344B1B782C
:105F300033B1FFF725FC18B978F0E8FD052307E039
:105F40002046FFF723FF804630B978F0DFFD0923B4
:105F500003604FF0FF3446E00024DFF8A8B0A2460B
:105F6000B6F5805FB14603AB394628BF4FF4805980
:105F70004046CDF80CA04A466CF0E0F801280546F2
:105F80001BD1DBF80030186D01930268126C90474A
:105F9000019B18B15A6D92F89C2072B9186D64215A
:105FA00003685B689847FFF7EBFB30B103AB4A46E9
:105FB000394640466CF0C2F80546039B4B45BBD8BA
:105FC000002BB9D03DB178F0A1FD02462846FFF77D
:105FD00097FB1060BDE74B451C441F44A6EB03062E
:105FE00001D3002EBCD102A81EF02EFC204605B025
:105FF000BDE8F08F4FF0FF34F8E700BF00970030A6
:10600000FC960030C0450030022838B5044606D959
:10601000FFF7A6FE054638B94FF0FF3412E078F0DE
:1060200075FD09230360F7E7006808B173F02AFDE6
:10603000686873F027FD044B0022284643F82420AB
:1060400073F020FD204638BDBC96003037B50D46B4
:1060500001F05AFA50B34FF4B772164901A81EF076
:10606000D1FB78F053FD002303602846FFF778FE4C
:1060700038B94FF0FF3401A81EF0E6FB204603B00C
:1060800030BD2846FFF782FE0028F2D06CF0F4F90C
:1060900004462846FFF7B8FF002CECD078F036FD18
:1060A00002462046FFF72CFB1060E2E74FF0FF347A
:1060B000E4E700BF0097003013B50C4601F024FA66
:1060C00038B34FF4F872144901A81EF09BFB78F026
:1060D0001DFD002303602046FFF742FE38B94FF054
:1060E000FF3401A81EF0B0FB204602B010BD2046D0
:1060F000FFF74CFE0028F2D06CF008F904460028A7
:10610000EFD078F003FD02462046FFF7F9FA106061
:10611000E5E74FF0FF34E7E7009700302DE9F74F50
:106120008946904601F0F0F9002800F0C48040F262
:106130002312624901A81EF065FB614B1B787BB1FD
:10614000FFF71EFB60B978F0E1FC052303604FF018
:10615000FF3401A81EF078FB204603B0BDE8F08FA5
:1061600078F0D4FC0023036008F00303022B17D05F
:10617000002B0CBF0125022518F4007F06D018F46F
:10618000806F14BF45F0080545F010050024DFF8C6
:1061900038A10134102C05D178F0B8FC172310E099
:1061A0000325E9E7022CF4DD5AF82430002BF0D166
:1061B0000121082073F062FC064630B978F0A6FC95
:1061C0000C234FF0FF3403601EE001214FF41470E4
:1061D00073F054FC074618B9304673F053FCEDE7F2
:1061E0004846FBF79DF8013073F008FC834618B968
:1061F000384673F047FCEFE7494679F0ADF9C6F849
:1062000004B04AF8246037602046FFF7A9FD18B9AA
:106210002046FFF7F9FE9AE72046FFF7B7FD07464D
:1062200030B92046FFF7F0FE78F070FC09238DE7C7
:106230005FFA85FA494652466BF05EFD0128064634
:1062400018D1204B1D68286D03681B6C984718B146
:106250006B6D93F89C3073B9286D642103685B689B
:106260009847FFF78DFA30B15246494638466BF0F1
:1062700043FD06463EB178F049FC0246F0B2FFF716
:106280003FFA1060C4E718F0080F3FF462AF3846D9
:10629000D7E904236CF0FEF8054600283FF459AF17
:1062A00078F034FC02462846FFF72AFA1060384698
:1062B0006CF0E2F8ACE74FF0FF344DE700970030A8
:1062C000FC960030C0450030BC960030F7B503792D
:1062D0000446C3B1002640F272321B4901A81EF0E9
:1062E00091FA1A482671FDF7A3FA194B32464FF47A
:1062F00000711F68786D03681B6D9847044620B9CC
:1063000001A81EF0A1FA03B0F0BD02464FF40073DD
:10631000314610486CF0BEFC0546786D4FF40072B3
:10632000214603685F6D3346B8473DB90A48FDF71B
:106330007FFA20F01DFA20F0CDFAE1E72946074860
:10634000FDF776FAF5E700BF0097003024820C08CD
:10635000C045003036820C0839820C0844820C0893
:10636000FFF7B4BF01384C289ABF024B53F8200006
:106370000020704750830C0810B50446FEF7E0FB80
:10638000204610BD10B5054C204620F0CBF9204624
:10639000034A0449BDE8104074F0E0BD00970030A6
:1063A000CC36013011570408002070474FF0FF3001
:1063B000704700004FF0FF3070470000002070472A
:1063C000002070474FF0FF30704700000020002190
:1063D0007047000000200021704700000020704737
:1063E0000120704770470000002070477047000090
:1063F000704700000329F7B506460D4617461C46B0
:1064000004D8182303FB01031A793AB978F07EFB0C
:10641000092303604FF0FF3003B0F0BDD3F818C07C
:10642000BCF1000FF2D046F21B72D968ADF8002023
:10643000C1B1182202FB0562D368906923448268C7
:10644000934227D818232246394603FB0565AB69DA
:106450001868EB68184478F049FCEB682046234440
:10646000EB60D9E7052CE4D93868B7F804E0009070
:1064700080B2DCF808309042ADF804E0D9D1BDF824
:1064800004209A42D5D9D21A60463BF0C9FF0028B1
:10649000CFD1BFE79A1A00213BF0C2FF0028D1D12B
:1064A000B8E70000032938B504D8182404FB010418
:1064B000257935B978F02AFB092303604FF0FF30C6
:1064C00038BD012B08D0022B09D003B9E260182394
:1064D00003FB0100C068F3E7E3681A44F6E778F0CD
:1064E00015FB1623E9E700002DE9F04F1F460023B6
:1064F0008A4615462DED028B8FB054688DF83430E6
:10650000ACB914870DF11B0107AA284612F052FA04
:10651000BAF80420A3B280469A4212D9013400B3DB
:1065200007AA0DF11B01284612F072FAF0E7138F4B
:106530000DF11B0128460133138707AA12F068FAF0
:106540008046BAF80630B8F1000F0AD0ABB12A8FF6
:106550009A4212D3002630460FB0BDEC028BBDE844
:10656000F08FBAF80660002EF4D12C8F12F0B4FA36
:106570008442EFD012F028F8EDE7012309AA404643
:1065800029460093102311F027F805F10803E81DB0
:10659000002208EE103A09ABD1B29B4613F9014B29
:1065A000059110F9011FA14202D101320029F3D156
:1065B0005846FAF7B5FE10F0FF03049307D1059B88
:1065C0000BF1FF3B013BDBB20593012304939AF8E7
:1065D0000130039363B19DF81B10404611F062FA3D
:1065E000DDED070A0AF060F980F00100C3B2039301
:1065F0009DF81B0010F056FE049B044603F10209AF
:10660000039B002B50FA89F214BF0646002601288E
:106610001644F6B215D96D68BAF80220063535442D
:10662000B5FBF2F102FB11555DB1854209D2451B64
:1066300038460021EDB22E442F442A46F6B278F0B7
:106640007DFB039B59469DF81B50B81C45EA03127D
:10665000049B3A705A1E059B43EA02127A70049A10
:1066600078F044FB2246414607EB090078F03EFBF8
:10667000039BB3B1013D042D13D8DFE805F01803E7
:10668000181F1F00DDED077AFDEEE77A17EE903A4E
:10669000ADF8203004EB0900224608A9384478F010
:1066A00025FB09A918EE100A78F056FF53E7DDED37
:1066B000077AFDEEE77ACDED087AEBE704EB090007
:1066C000224607A9EAE700002DE9F04F064689B007
:1066D0000F461C46154642B93C222946184678F01A
:1066E0002DFB012009B0BDE8F08F5B68934204D90F
:1066F0003C220021204678F021FB94F81990B9F152
:10670000000F1AD0D4F804A0A5EB0A08C84528BF8A
:10671000C8465FFA88FBD94508D008F11A01A9EBF1
:10672000080204F11A00214478F0EEFAA9EB0B09F3
:1067300008EB0A0384F81990636004F11A0863688F
:10674000AB421BD0A5EB030A22466B4639463046C6
:10675000FFF7CAFE90B18245D14628BF81468245E7
:1067600008D2A0EB0A030DEB09014046DAB26276CB
:1067700078F0BCFA63684B446360E0E76068431BF1
:1067800058425841AEE7000003292DE9F04F8046FA
:10679000894692461D462DED028B8BB004D81823F6
:1067A0004B43C61832795AB978F0B0F909234FF043
:1067B000FF34036020460BB0BDEC028BBDE8F08FC8
:1067C0000433C31808EE103AB3691BB178F09EF990
:1067D0001623ECE7F3880BB905B1F580F3880BB10C
:1067E000AB42F3D1182202FB098213693BB1D26894
:1067F0009342C0F0AA809B1A9D4228BF1D461823D1
:1068000003FB0983DB68052B00F2A18046F21B73B2
:10681000ADF8083012F060F93389ADF80C009842F9
:10682000D4D9C01A738980B2ADF80A001BB198425E
:1068300088BFADF80A30182303FB0983D968737940
:10684000C1F10604AC4228BF2C461BB146F21C73B2
:10685000ADF80830E4B202AB50462246194478F055
:1068600045FA18232D1B03FB0983DA682244DA60FA
:10687000A0D0A2441823012703FB0983DA685E69CC
:106880000023063A7068022F06D0316C914203D380
:1068900081424FF002075CD3C3EB031306EB830680
:1068A0007368934208D0334618EE101A4046FFF73B
:1068B0000BFF00283FF47EAF002D3FF47BAF777EC7
:1068C00027B3AF42504628BF2F46FBB23A46ED1BD6
:1068D000BA44009306F11A031946019378F006FAB8
:1068E00096F819B0009B9B4508D007F11A01019B4F
:1068F000ABEB07023144184678F006FA009BABEB8D
:10690000030B73683B4486F819B0736006F11A03F1
:1069100008EE903A7DB102AB324618EE101A4046AE
:10692000FFF7E2FDE8B9182303FB0983DA68196968
:106930003A4489B91A6118213C4401FB0988D8F806
:106940000C303B44C8F80C3034E7002557E70024EE
:1069500090E70846012396E78A4294BF1A611961BD
:10696000E9E7A842834628BFAB46A84208D9401BA6
:1069700002ABC2B2591918EE900A727678F0B6F9E5
:106980005A46504602A9A5EB0B0578F0AFF972689C
:10699000DA445F4402EB0B037360BBE710B50C46AF
:1069A00009220849204678F001FE38B994F9090017
:1069B00030B1A0F13F035842584110BD0020FCE720
:1069C0000120FAE723AD0D082DE9F84F0746894667
:1069D0001446FFF7E3FF40B978F098F802234FF030
:1069E000FF3603603046BDE8F88F04F003044FF033
:1069F000000818233A1D03FB08F54646515D00299F
:106A000000F08680032E08F10108F4D178F07EF8BA
:106A10001723E4E718234FF0000A012203FB087351
:106A2000C3F80CA0C5E9012AC3F810A0C3F818A048
:106A30009CB11020FEF77EF8044618B11022514692
:106A400078F07CF9182303FB08739C612CB93B6830
:106A5000414638465B68984765E03F21484678F0F4
:106A60006BFDDFF8D0A00446DFF8CCB0002CB9D025
:106A700094F90030002BB5D004F101092C4906220D
:106A8000484678F093FD014680B907340A22204633
:106A900079F03CFD4FF6FE7398422CD828812621D0
:106AA000204678F049FD81464C46DFE751460622F4
:106AB000484678F07BFD014650B907340A2220464B
:106AC00079F024FD4FF6FE73984214D86881E6E70A
:106AD00059460D22484678F069FD01460028E3D169
:106AE0000E340A22204679F011FD012803D800F067
:106AF00001006871D3E7182000FB0877786908B1B6
:106B0000FEF724F800232B7178F000F8162366E7CF
:106B10003D44002C7FF47EAF7820FEF715F86861C5
:106B200000287FF477AF77F0F1FF0C2357E700BF21
:106B3000E4840C08EB840C08F2840C0810B51446AD
:106B4000FFF72CFF30B977F0E1FF022303604FF02D
:106B5000FF3010BD58220021204678F0EFF811F0E8
:106B6000BBFF0C23584320610020F2E72DE9F04FD2
:106B70000025934691B015704A699368052B40F241
:106B8000B98014682068A288049080B2ADF81420FF
:106B900046F21B72904240F0AD80BDF814209A423C
:106BA00040F0A8800D22294607A80634069578F003
:106BB000C5F8BDF81220ABB29A4240F29F80277808
:106BC00007F00F063F0940F0958094F8018008F027
:106BD0000F0A4FEA181808F101030AEB03090193A1
:106BE000B9F1100F00F38680524606A90BA808F1F0
:106BF000030878F07BF8019BA11C44441A460BABB8
:106C000003EB0A0078F072F810AB0DF12C0E0DF1C9
:106C1000180C994409F8147CBEE80F00ACE80F008A
:106C2000DEF800300DF10E020DF10D010BA88CF80D
:106C300000308DF80D7010F089FD48B9012E02D199
:106C400001340135B5E7022E0CBF02340434F8E7F5
:106C5000BDF80E309DF80D1013F004031ED001296D
:106C600004D190F90070B7FA87F77F098E4217D1E7
:106C7000032E15D154F8043B03600022114611F095
:106C8000ABFC002FDDD0012364218BF800301C4BBE
:106C90001B68186D03685B689847D2E71F46E5E7F5
:106CA000012E0FD1237817B11F1E18BF01275BB229
:106CB0000134019000EE103AB8EEC00A10F096FFD1
:106CC0000198DAE7022E09D134F9023B00EE103ABE
:106CD000B8EEC00A019010F089FFF1E7032E02D14F
:106CE00054F8043BF2E7042EC7D154F8043B00EEFD
:106CF000103AEFE7002011B0BDE8F08F0120FAE76D
:106D0000C045003073B505460E460524013C14F01D
:106D1000FF040CD00DF1070231462846FFF726FF8D
:106D200018B19DF80730002BF0D102B070BD0120E2
:106D3000FBE700000329F8B504460D4604D81821E6
:106D40006943461833793BB977F0E0FE4FF0FF37DF
:106D5000092303603846F8BDB369DBB90027002377
:106D60003371182606FB0543586908B1FDF7EEFE9E
:106D700006FB054600237361B6692EB130463BF031
:106D800071FB3046FDF7DCFE1821002301FB0544B2
:106D9000A361DFE704310144FFF7B4FF0028DDD130
:106DA00077F0B4FE16234FF0FF370360D7E70000FB
:106DB000002070470020002170470000002070472D
:106DC00008B577F0A3FE1E2303604FF0FF3008BD27
:106DD000032938B504D80C2404FB0104656835B9CF
:106DE00077F094FE092303604FF0FF3038BD012B8C
:106DF00008D0022B12D063B9002A05DA77F086FE9C
:106E00001623F0E7E3681A44A3689A4294BFE2604D
:106E1000E3600C2303FB0100C068E7E7A368E360BD
:106E2000F7E7000008B577F071FE1E2303604FF00E
:106E3000FF3008BD486812F093BA00000329F8B586
:106E40000646104604D80C2202FB0166776837B963
:106E500077F05CFE092303604FF0FF30F8BDD6E900
:106E600002516C1A9C4228BF1C4634B12246394458
:106E700077F03CFFF3682344F3602046EEE7000020
:106E800000F134032DE9F341CE1A1D4B8046F71073
:106E9000B6F5467F03FB07F705D977F037FE0923E0
:106EA0000360002426E04FF4847306F1380103FBED
:106EB00007070144786B12F055FA0446D0B1796B9C
:106EC00008460191FAF72CFA019905460246204638
:106ED00078F06CFB0028E4D163572F2B0ED10135DD
:106EE00087F83901FF22611906F13A04444420462B
:106EF00078F070FB204602B0BDE8F0810446F9E767
:106F0000E1830F3E70B506460C200D46FDF712FEDC
:106F1000044670B101468660284612F0D1F9054654
:106F2000606030B9204600F003FB20462C46FDF798
:106F300007FE204670BD000012F00302F8B50446BB
:106F4000084606D077F0E2FD1E234FF0FF350360C0
:106F50000FE00C23211D03FB02F615468F5957B194
:106F6000032D02F10102F6D177F0D0FD1723ECE7F3
:106F7000E7602846F8BD06F108012144344412F0C8
:106F80009FF960600028F3D177F0C0FD0223DCE7B1
:106F900000F13403C91A0D4B10B5B1F5467F4FEA25
:106FA000E10403FB04F406D977F0B0FD0923036084
:106FB0004FF0FF3010BD4FF4847303FB0404606B8B
:106FC00072F060FD00206063F4E700BFE1830F3ED4
:106FD00013B5084601A9144612F072F938B977F0D2
:106FE00095FD022303604FF0FF3002B010BD12F098
:106FF000B7F958220021204677F0A0FE019B00201F
:107000002361F2E770B50546002308464FF484710A
:1070100005F1340601FB03F4325942B10133042B6C
:10702000F8D177F073FD17230360002007E02E19D5
:10703000328772F087FD706308B13434281970BD4F
:10704000032910B504D80C2404FB0104606830B98E
:1070500077F05CFD092303604FF0FF3010BD12F0A4
:107060007FF900206060F9E74FF0FF3070470000C3
:10707000032910B504D80C2404FB0101087930B9A8
:1070800077F044FD092303604FF0FF3010BD012B62
:107090000AD0022B11D02BB9CB689B689342D4BF86
:1070A0008B608A608868F1E78B681A44CB689B68BC
:1070B0009A4294BF8A608B60F4E777F027FD16232D
:1070C000E1E7000091F9003010B533B177F01EFD13
:1070D000002402230360204610BD4FF48270FDF7A8
:1070E00029FD04460028F6D177F010FD0C2303603B
:1070F000F1E70000032970B50646104604D80C22BB
:1071000002FB0166327932B977F000FD0923036092
:107110004FF0FF3070BDD6E9021295686C1A9C42A0
:1071200028BF1C4613682246194477F0DFFDB36878
:1071300020462344B360EDE713B50B680C460020EE
:107140000B2B0DD881F80301081D0649FF22019081
:1071500051F823103BF0F4F82368019801332360C1
:1071600002B010BD08860C08032970B504460D4610
:1071700004D80C2303FB01031A7932B977F0C6FC5B
:10718000092303604FF0FF3070BD0022DE681A71E2
:107190002EB130463BF066F93046FDF7D1FC0C21AC
:1071A000002001FB0544E060EEE70000084608B55A
:1071B00031B977F0ABFC162303604FF0FF3008BD08
:1071C000FDF7BEFC0020FAE770B50D46074E00241F
:1071D00056F8041B2846FAF799F808B960B270BD52
:1071E00001340C2CF4D14FF0FF30F8E708860C087E
:1071F0002DE9F04F12F0030485B005460E4604D089
:1072000077F084FC1E23036009E14FF00C0A031D94
:107210000AFB04F9274613F809B0BBF1000F00F090
:10722000F080032F04F10104F2D177F06FFC1723F3
:10723000E9E731462846FFF7C7FF00280BDA40464A
:107240003BF010F94046FDF77BFCC9F80CB077F035
:107250005DFC0223D7E773493046FAF757F830B997
:10726000714B41461B68586D0368DB6E98476F4948
:107270003046FAF74BF848B96B4B1B68586D0C2336
:10728000026803FB0453126FD9689047684930467F
:10729000FAF73CF848B9644B1B68586D0C23026838
:1072A00003FB0453526FD968904762493046FAF79E
:1072B0002DF848B95C4B1B68586D0C23026803FB22
:1072C0000453D26FD96890475B493046FAF71EF8ED
:1072D00050B9554B1B68586D0C23026803FB0453CF
:1072E000D2F88020D968904754493046FAF70EF812
:1072F00028B153493046FAF709F868B901204A4BDA
:107300001B6803EB8000406E30B10C23026803FB66
:107310000453526AD96890474A493046F9F7F6FF54
:1073200048B9414B1B68586D0C23026803FB04539A
:10733000926FD968904744493046F9F7E7FF08BB98
:107340000C2303FB0453D3F80C80374BD3F800A075
:10735000DAF854000368D3F8943098470190DAF8CB
:1073600054000368D3F8903098470090DAF854003E
:107370000368D3F890A0D04703464046DDE90021DA
:107380003BF07AF831493046F9F7C0FF98B9264BFF
:1073900003AA02A91B68CDE90200D86B03689B69A8
:1073A000984740B10C20039B029900FB04501A46F9
:1073B000C0683BF061F80C2606FB0456F3689A6837
:1073C000AAB91B7B002B14BF0C27022777F09EFB6A
:1073D0000760F6682EB130463BF044F83046FDF7C2
:1073E000AFFB0C20002300FB0454E36017E00023F4
:1073F000C9F80830012389F80430384605B0BDE8E3
:10740000F08FA9441020FDF795FB8046C9F80C00C9
:1074100000287FF40EAF77F079FBC0F800A04FF0A2
:10742000FF37EAE7099A0C08C0450030EC990C08D0
:10743000F9990C08DD990C081A9A0C08C0850C08FB
:10744000CF850C08DE850C0831990C083B9A0C0896
:1074500070B5044616460D4619B112B191F90030C7
:107460003BB977F053FB16234FF0FF3403602046FF
:1074700070BD58220021304677F060FC2846F9F7AD
:107480004FFF012895F9003003D12F2B04D10024A0
:10749000EDE72F2B08BF013529462046FFF794FE64
:1074A000002803DA77F032FB0223DDE70D49284696
:1074B000F9F72CFF044618B94FF400433361D6E7BF
:1074C00009492846F9F722FF044640B9074B1B68D3
:1074D000586D0368D3F8903098473061C7E7044B84
:1074E0003361D4E73B9A0C0831990C08C045003051
:1074F000A0860100486810B50C4618B172F0C2FAB7
:107500000023636010BD000008B5084B1B685A6D6E
:1075100092F89C203AB1186D03681B6C984780F074
:107520000100C0B208BD0120FCE700BFC04500302B
:1075300010B50446806818B103682146DB6C984793
:10754000204610BD2DE9F04399B0036805468846F2
:107550009B6902AA9847074620B10024204619B02B
:10756000BDE8F0830C20FDF7E5FA04460028F4D0CE
:107570008560069872F042FA064630B92046FFF759
:10758000D7FF2046FDF7DCFAE7E72B6841463A468D
:107590002846D3F800903B46C847431C014603D118
:1075A000304672F06FFAE9E72B68324601902846C0
:1075B000D3F80880069BC047069B019998422B6828
:1075C00028465B6801D09847EAE79847069BC4E9DC
:1075D0000036C3E710B103685B69184770470000C5
:1075E00038B5002504462C3040F8185C40F8145C8F
:1075F00040F8105C04F0ECFA4FF0FF3304F1400067
:10760000E3631FF08FF804F174003AF055FF0C4962
:107610002046C4F89C50C4F8A050C4F8A450C4F844
:107620006851C4F86C51C4F8705110F0DBFD054B83
:107630001A6812B1044821F0C7FF20461C6038BD0B
:107640009C870C081897003098860C08084699B15A
:10765000C81FC3B2102B0ED810280CD8DFE800F0DA
:10766000090B090B0B0B0B090B0B0B0B090B090976
:10767000090000207047012070470000F7B590F91D
:10768000023004460E46032B15D100F12A07384676
:1076900010F0CCF9054670B901230DF10701384609
:1076A0008DF8073011F0F2FC0DF10701A01C8DF8E8
:1076B000075011F0EBFC21782046FFF7C7FF30B1EF
:1076C00000220521304612F0CBFCC4F81C01002535
:1076D000B3EE0E1AF1EE040A4FF4E37094ED090ACA
:1076E000A56009F0B9F9B7EE007A238A84F86850EA
:1076F000C7EE007A013B9BB2C72B84BFC82323820D
:10770000C4ED5F7A03B0F0BD034690F8210193F811
:1077100080310BB10130C0B270470000B02303FBD1
:10772000010191F8B90010B1D1F8A8301360704789
:10773000B02303FB010191F8BA0010B1D1F8AC30CD
:1077400013607047B02310B503FB010494F8BB40ED
:1077500024B101FB0333C1180B681360204610BD30
:107760002DE9F843B02384460F4603FB0103D3F809
:10777000C82022B9D3E9340150EA01032CD0B02645
:1077800006FB07C6B6F8700000283FD0204DDFF892
:107790008490A0FB0545D6E9342313431ED0463719
:1077A0005CF8270004F012F8074621F047FF14EBBD
:1077B000090245F14904D3194FF47A7544F10004E4
:1077C000A3FB053205FB0422D6E93445001B61EB1F
:1077D0000501181842EB0101BDE8F883F06E49235A
:1077E00010EB090043F10003071945EB030421F0F6
:1077F0001DFFD6F8C8104FF47A73401AC01944F12F
:107800000004A0FB030103FB0411E5E70146E3E7E5
:1078100000840C24B0F5F790B02303FB010310B5EE
:10782000B3F87040ACB1463150F8210003F0CEFF00
:10783000094B4FF47A72A4FB0313084C091943F166
:107840004903081843F10003A0FB020102FB0311E6
:1078500010BD20462146FBE700840C24B0F5F790CC
:1078600000EBC101C1F85C21A1F860317047000054
:10787000435609B2022B0BD1038D5A0710D500EBEA
:10788000C100124BC0F85C312E23A0F86031704764
:10789000A3F11102D2B2012A05D8038DDB0710D55E
:1078A0002E230B4A05E00B2B08DC092BF8DD002307
:1078B0001A4600EBC100C0F85C21E6E70F2BF6D0BA
:1078C000EEE700EBC100034BDCE700BFAC880C081F
:1078D0006C870C08DC880C0838B500EB8105D5F8FE
:1078E0001C31FBB100EBC104B4F86021D2B11A68BD
:1078F0001846126A9047D5F81C31B4F8602119680F
:107900008242CD6828BF0246D4F85C111846A847C9
:10791000D4F85C310344C4F85C31B4F86031181A0F
:10792000A4F8600138BD00002DE9F043425C85B049
:1079300004460E46172A04D801239340834A134273
:1079400004D104EB8607D7F81C310BB9002552E0AF
:107950003825012305FB064585F8293121F066FE0F
:10796000D5F824318046C31AB3F5966F25D995F81A
:107970002831774A0133DBB2082B08BF002385F892
:1079800028313825D7F81C0105FB0645036895F812
:1079900028115B6A52F821109847D7F81C01002182
:1079A0000368DB6D9847C5F8248194F91330002BE8
:1079B0000BDD31462046FFF75BFF94F91330002BB7
:1079C00003DD31462046FFF787FFA3570B2B16D068
:1079D0000F2B25D00A2B34D14FF4CC70FDF7AAF829
:1079E000054640B1B022D7F81C31214602FB0642C1
:1079F000683201F095FB284605B0BDE8F0834FF4EE
:107A0000BC70FDF797F805460028F4D0B022D7F8EF
:107A10001C31214602FB0642683200F069FEEAE7AB
:107A20004FF4C870FDF786F805460028E3D0B02271
:107A3000D7F81C31214602FB0642683201F0BCF83F
:107A4000D9E704EBC603B3F86031002B7FF47EAFB7
:107A5000D7F81C014FF03808036808FB064908FBFB
:107A600006481B6909F595799847B0F5005F28BF6E
:107A70004FF4005085B2002D3FF468AFD7F81C01D9
:107A800003685B699847A35DC1B2013B012B0AD82B
:107A900098F828212E4B53F8223094F913208ABBF2
:107AA000B3F5164F37D2238D13F0010FA35DA3F169
:107AB000110314BF4FF461324FF4E122012B1ED8A1
:107AC00098F82801224B53F82030934217D14846AA
:107AD00002F0F2FB98B1A3574FF49E60112B0CBF3C
:107AE0004FF001084FF00208FDF724F80546002882
:107AF00081D0B022CDF8008002FB06421FE0013D9C
:107B0000ADB2B8E7B3F5E13FCDD3228D500702D433
:107B1000B3F5613FC7D14846039102F0CDFB03990D
:107B20000028C0D04FF49E60FDF704F805460028F9
:107B30003FF461AFB022002302FB06420093D7F866
:107B40001C316832214603F02FFC54E70042C0008C
:107B50004C870C08F8B504460D46B02621F066FDAA
:107B60000023074606FB05462946204686F869306D
:107B70004FF6FF73A6F89630A6F89830FFF7D4FEBC
:107B800090B1012204EB051386F8692005F1460245
:107B9000194644F82200DF654FF47A63A1F860309B
:107BA000BDE8F84003F0B6BEF8BD0000054B1B6809
:107BB0002BB1C16B4A1C02D0184606F0D3BE002080
:107BC000704700BF30970030F8B51E46D0F8183126
:107BD00004460D461746DBB1D0F81431C3B121F08D
:107BE00025FDD4F81431C01AB0F5FA7F10D2D4F8BC
:107BF00004313B60D4F808313360069BD4F80C2183
:107C00001A60079BD4F810211A60D4F814312B6045
:107C1000F8BD000010B4D0F8183153B190F900004D
:107C2000112806D11868046C184623465DF8044BE9
:107C3000184700205DF8044B70470000D0F8183159
:107C40003BB190F90020112A03D11A681846526CF2
:107C50001047704790F90030122B03D1D0F818016B
:107C6000FFF7B8BC7047000031B990F8223122B15B
:107C700043F0010380F82231704723F00103F9E754
:107C800010B40C4611461A462CB9D0F818015DF80C
:107C9000044BFFF79FBC5DF8044B704770B490F93C
:107CA0000660044613467F2E0BD00A46F1B270BC24
:107CB000FFF7E6BF172B08D0D4F8180170BCFFF708
:107CC00089BC90F90030122BF4D170BC70470000D1
:107CD00070B5CE789EB00C467122712E4FF0000127
:107CE000054601A828BF712677F028F804F10C0199
:107CF00001A8324676F0FAFF9DF806206E2A04D8D5
:107D00000DF107012846FFF7C9FF1EB070BD000046
:107D100013B5044601917AB9D0F8180160B103682F
:107D20009B69984740B1D4F8180101990368DB6951
:107D300002B0BDE81040184702B010BD10B590F970
:107D400000300C460BB9002010BDD0F8180118B94E
:107D5000002301202370F7E703681B699847002878
:107D6000F1D1F5E72DE9F0479146CA0704460F46E1
:107D70001E4605D449461A46BDE8F047FFF78EBFB8
:107D8000D0F86431002B44D0C7F34105D4F864A186
:107D90004FF0B408FF089AF8003008FB05A808F176
:107DA0000608002B40D1D4F8643140465F700123AF
:107DB000D4F8641103FA05F20B78134332460B70C2
:107DC000494676F093FFB32ED4F8643141D86A1C4B
:107DD00005EB4505C5EB05159A70D4F8643106EB43
:107DE00085059D80D4F864118A78DAB1012308787A
:107DF0009340013B984215D18A8820460631FFF70F
:107E00004DFFD4F8642100239370D4F864211370DB
:107E100008E040F2D621012071F030FEC4F8640180
:107E20000028B1D1BDE8F0879AF80120BA4209D103
:107E3000EB40DB07B7D532464946404676F046FF71
:107E40000028EFD000238AF80230D4F864211370A0
:107E5000A9E71A780F2AC5D104229A704FF4347218
:107E6000D4F864319A80BDE770B5CE78AEB00C46D8
:107E7000B622B62E4FF000010546684628BFB6264A
:107E800076F05CFF04F10C016846324676F02EFF76
:107E90009DF80130B42B06D80DF102029DF80010B8
:107EA0002846FFF75FFF2EB070BD000070B58A7ADC
:107EB00005464B7A0C4643EA0223CA7A43EA024358
:107EC0007B2B05D0E92B07D1BDE87040FFF7CCBF75
:107ED000BDE87040FFF7FCBE002695F82121F3B203
:107EE0009A420CD903F1460255F8220028B1EB560C
:107EF0001BB1036821465B6A98470136EDE770BD08
:107F0000174B10B4136049BBB0F92030002B0DDDC6
:107F100007EE903A9FED137AF8EEE77A67EE877AEC
:107F2000C2ED007A01205DF8044B7047D0F818319B
:107F300013B190F8691049B990F9000010B9002305
:107F40001360EFE7431E58425841ECE719681846A2
:107F50008C6A114623465DF8044B18470020E2E77F
:107F6000CDCCCC3D6F12833A1430704790F821315C
:107F70008B4209D9083130F91100002804DDC828E6
:107F8000A8BFC82080B27047C820704759B990F97F
:107F90002A3043B990F900302BB1D0F8180110B154
:107FA0000368DB6A184700207047000008B50346E5
:107FB00090F90E0040B1D3F8180128B103681B6B8B
:107FC000984780F00100C0B208BD000031B9D0F878
:107FD000180118B1036811469B6C184700207047C0
:107FE000B02303FB010191F8C40010B1D1F8C030F7
:107FF000136070472DE9F7431F4690F8833104461C
:108000000D46DDF8289093BBB02606FB010696F8D6
:10801000BC80B8F1000F24D0D6F88C30136001AAD0
:10802000D6F89030C9F80030FFF76AFF70B1DDED87
:10803000017A9FED107AD9F8003067EE877AFCEE6E
:10804000E77A17EE902A9B1AC9F80030B02000FB9F
:10805000054393F8BD3043B105FB00000444636859
:108060003B60404603B0BDE8F083034BF8E74FF0B8
:108070000008F6E700007A44000020417FB5B023F5
:1080800003FB010393F89430EBB105AB03AA009313
:1080900004ABFFF7AFFF80B1DFED0C7A9DED030A73
:1080A00020EE270A08F092FCFDEEC07A17EE900A47
:1080B00030B180B207B05DF804FB4FF6FF70F9E70E
:1080C00048F6A040F6E71846F4E700BF0000C842B3
:1080D0002DE9F04F2DED068B90F8C43095B0884611
:1080E000856F9FED56AA002B00F09C800A23D0EDEF
:1080F000307A6B4308EE103AB8EEC88AA7EECA8A07
:10810000BDEEC88A90F8BA30002B00F08E80D0ED1A
:108110002B9A90F8BB30002B00F08A8090ED2C9ABF
:1081200090F8B930002B00F08680D0ED2A8A866D59
:108130004FF47A7790F88231A6FB077690F8699031
:1081400023B1B9F1010F28BF4FF00109DFED3C6AFF
:10815000002190ED217AD0ED227A27EE267AD0F810
:10816000803067EEA67AC26F0493BCEEC77AB0F88F
:1081700096B0FCEEE77AB0F898A0059217EE103AA8
:108180009CB217EE903A9BB2029390F89A30039308
:10819000FFF774FF049B69EE8A9A29EE0A9A059A02
:1081A0000A930A23FCEEE99A18215D43029B68EECC
:1081B0008A8A0992ADF83630BCEEC99A039B07AAA9
:1081C000FCEEE88AADF84E008DF8393018EE103A22
:1081D00040460B95CDF83A3019EE903AADF830B0F4
:1081E000CDF83E3019EE103AADF832A0CDF842305D
:1081F00018EE903AADF83440CDF8463000238DF8B3
:108200003890ADF84A30ADF84C303423CDE9003128
:108210001E23CDE9077613F037FE15B0BDEC068BB3
:10822000BDE8F08F08EE103A6CE7DFED069A70E7D4
:108230009FED049A74E7DFED038A78E700007A4443
:108240000000C842000000002DE9F043A1B0044640
:108250000D4621F0F3F905AB0027814688460093CF
:1082600003AA04AB2946204603970497FFF7C2FEF2
:10827000A323CDF84F90CDF853808DF84C30952343
:108280008DF857508DF84D3059238DF84E3094F8B5
:1082900082313BB1B02303FB054393F86930012BD6
:1082A00000F2C080B02303FB054393F86930B02689
:1082B0008DF8583006FB0546F36ECDF85930B6F808
:1082C0007030ADF85D3096F89A308DF85F30B6F8C2
:1082D0009630ADF86030F36FCDF86230D6F880306C
:1082E000CDF86630B36FCDF86A30D6F88430CDF86B
:1082F0006E30D6F88830CDF87230D6F8A430CDF88C
:108300007630039BCDF87A30474B1B6893F82031C9
:108310005A1B534253418DF87E3006F0E7FC13A9F7
:10832000332205F0DDFD06AA294620460697079769
:1083300008970997FFF7FCF907AA294620469FED01
:108340003B6AFFF7FFF908AA29462046FFF7E6F93E
:1083500009AA29462046FFF743FE9DED067ADFED88
:10836000346AA32327EE067ADDED087A8DF82830EB
:10837000952367EE867ACDF82B90B4EEE67A8DF8E9
:1083800029305A23CDF82F808DF83350F1EE10FAB2
:108390008DF82A30B6F8983058BFB0EE667AADF84E
:1083A0003430BCEEC77A17EE103A9DED077A27EE0F
:1083B000067AADF83630B4EEE67AF1EE10FAF4EE65
:1083C000E67A58BFB0EE667AF1EE10FABCEEC77AE4
:1083D00058BFF0EE667A17EE103AFCEEE77AADF889
:1083E000383017EE903AADF83A30049B0F9396F878
:1083F000B8308DF8403004EB051304EB0514DB6D49
:10840000CDF84130B4F86030ADF84530099BCDF877
:10841000473006F06BFC23220AA905F061FD21B06C
:10842000BDE8F083012342E7189700300000C842FE
:1084300000FF7F472DE9F84F435604460D46072BB2
:108440000BD063B9B02101FB050484F869304FF605
:10845000FF73A4F89630A4F89830BDE8F88F90F830
:108460002231CB40DA07F8D400EB81090FB2D9F8FA
:1084700018311BB9BDE8F84FFFF76CBB90F913300A
:10848000002B01DDFFF728FAD9F818014FEA05188B
:1084900003689B689847834621F0C8F80646BBF1FD
:1084A000000F6DD1A044D8F85C30C31AB3F57A6FD1
:1084B000D3D94FF0B00A59460AFB054052466830FE
:1084C00076F03CFC0AFB05424FF6FF734FF47A61ED
:1084D00082F86850A2F89630A2F89830C8F85C602C
:1084E000A8F86010615D172903D83B4BCB40DB0730
:1084F0000CD4D9F8180100283ED1B023002203FB88
:108500000543C9F8182183F8692002E0012382F8A5
:10851000693004EB0712B2F86030F52B58D992F8A5
:108520006210B3F5FA6F01F1010182F8621017D2FF
:1085300092ED197A07EE903AB5EEC07AF1EE10FAA4
:1085400085BFF8EEE77ADFED256AF8EE677A67EE29
:10855000A67A84BFDFED226AE7EE267AC2ED197AA9
:108560002046FFF723FB00283FF477AF294620463B
:10857000BDE8F84FFFF768BE03685B689847BCE743
:108580004FF0B00909FB054999F8D83053B10023E1
:108590004FF47A72D9E93401F8F71CFA0023064641
:1085A00089F8D83004EB080304EB0512D96D711A71
:1085B000A2F86010B022DE6502FB054292F8692045
:1085C000012AA6D994F88221002AA2D19E65A0E7AB
:1085D000002182F86210ABE70042C0000AD7A33C3A
:1085E00048E17A3F13B5044600F140014FF485623B
:1085F00001A81CF007F900212046FFF71BFFD4F863
:10860000183113B1012384F8213101A81CF01CF9A1
:1086100002B010BD014B1868704700BF18970030BA
:10862000012070470020704770470000704700002D
:10863000014B01200B607047CDCC4C3E01207047B0
:1086400001207047012070470020704770470000EC
:1086500000207047704700000620704700487047B0
:108660000C890C087047000010B50446FCF768FA46
:10867000204610BD70B586B004460E46122201ADEC
:108680000021284676F05AFB0221642303228DF84C
:1086900004108DF806300D238DF80F1004218DF88D
:1086A000073001238DF80B208DF8101007218DF86D
:1086B000162094F866218DF812108DF80820D11834
:1086C00000228DF80D308DF8116084F86611E95C98
:1086D00001330A44122BD2B2F9D1606829468DF8D1
:1086E000152013220368DB68984706B070BD0000B0
:1086F00010B5044603F04EF80F4B002120462360CE
:108700000E4B84F866111A681B79C4F86D2184F841
:108710007131C4F8681184F86C1184F85A10FFF7AD
:10872000A9FF03212046FFF7A5FF20F07FFF6E3051
:10873000C4F86801204610BD1C890C0888230C0869
:1087400070B586B004460D461646002114226846D0
:1087500076F0F4FA0223072103228DF80030642317
:108760008DF80B1006218DF802300F238DF80720AD
:108770008DF8033001238DF80C100A218DF8142098
:1087800094F866218DF80D108DF80420D118002280
:108790008DF809308DF80F308DF80E6084F8661171
:1087A0008DF811501DF8031001330A44142BD2B276
:1087B000F8D1606869468DF8132015220368DB68DC
:1087C000984706B070BD00008B18002030B5DD79E9
:1087D0000C46002165F307009D7965F30F205D7954
:1087E00065F317401D7965F31F60DD7865F30701B8
:1087F0009D785B7865F30F2163F31741A35C63F306
:108800001F6141EC100B30BD881800238A5C10B545
:10881000C47864F307038478407864F30F2360F32B
:10882000174362F31F6300EE103A10BD8B1800204F
:1088300010B5DC7864F307009C785B7864F30F2054
:1088400063F317408B5C63F31F6010BD8B184FF010
:1088500000005B7863F307008B5C63F30F2080B24A
:10886000704700002DE9F04F2DED068B90F85D303C
:1088700083B00446402B40F0F080032500269FED96
:108880007B8B9FED7C9B9FED7DAB94F85E30AB4284
:1088900040F2DD8004EB050A05F102089AF85F70EA
:1088A0009AF86090012F33D1D4F80CB0424604F10D
:1088B0005F012046FFF7BAFFCBF80400D4F80CB0F4
:1088C000AA1D2046FFF7C2FFABF80800E3689AF83C
:1088D000672083F832209AF86830E26813F0010FBD
:1088E00014D09AF869300321DD0751700AD5E26887
:1088F00004219807517005D55907E2684CBF06233B
:1089000005235370013609EB0805BEE75770F9E7F8
:10891000022F30D104F15F01424620460191FFF75A
:1089200053FF20EE080BE36805F10A020199204687
:1089300020EE090BBDEEC00B83ED050AFFF744FFE7
:1089400020EE080BE36805F112020199204620EEA3
:10895000090BBDEEC00B83ED060AFFF735FF20EED5
:108960000A0BE368BDEEC00B83ED040AE56820F056
:108970005DFE2866C6E7082F2DD104EB080393F8A7
:108980005F30DB07BED504F15F01E768EA1C2046D3
:10899000DFED3C7A0191FFF737FFEA1D204687EDB6
:1089A000070AFFF731FF20EE270AE368204683ED30
:1089B000080A02F01FFF05F10B0201992046FFF79C
:1089C00023FFB1EE400AE368012283ED0F0AE3685A
:1089D00083F8502096E7092F10D1DFED2B7AAA1DDE
:1089E00004F15F012046FFF70FFF20EE270AE3683E
:1089F000BCEEC00A10EE102ADA8583E70C2F82D174
:108A000004F15F01AA1D2046FFF7FEFEF0EE407A5A
:108A100005F10A022046FFF7F7FEE36837EE800A09
:108A200005F11202F6EE007A204620EE270A83EDC9
:108A3000110AE768FFF7E8FE012387ED120AE268F2
:108A40001E4482F85230E26882F853305BE7052E0C
:108A50004FF0010002D0E3685870002003B0BDEC75
:108A6000068BBDE8F08F00BFAFF30080F8C1631A3A
:108A7000DCA54C4000000000D01263410000000063
:108A800000005940E02E65420000C84290F85A307C
:108A9000013B052B04D8DFE803F0101B1F233944EA
:108AA000022908D140F20123A0F85A300023A0F88F
:108AB000623180F8643100207047022380F85C1036
:108AC00080F85A3090F86431194480F86411F2E764
:108AD000032380F85D10F3E7042380F85E10EFE7CE
:108AE000B0F86231C218013382F85F109BB290F87F
:108AF0006421A0F86231114490F85E209A4280F817
:108B00006411D8D8052380F85A30D4E7062380F8BA
:108B10005F1180F85A3090F864318B42CBD1FFF767
:108B2000A1BE002380F86011EDE7000038B50446CF
:108B300020F07CFD054694F86C31042B1BD8D4F84A
:108B40006821824217D22344002220466E3593F8D2
:108B50006D11FFF7F5FD94F86C3103222046234494
:108B600093F86D11FFF7ECFD94F86C31C4F868517F
:108B7000013384F86C310025606803681B699847ED
:108B800050B1606803685B699847C1B22046FFF73F
:108B90007DFF2843C5B2EFE7284638BD0620704761
:108BA000004870476C890C087047000010B50446F7
:108BB000FBF7C6FF204610BD10B5044602F0EAFDE3
:108BC000104B2360002384F8603084F86C30C4E9D3
:108BD0001933AA2384F8713141F24423A4F8723185
:108BE000A36893F913305BB160680E2206490368ED
:108BF000DB6898476068222204490368DB6898476D
:108C0000204610BD088A0C0874890C0883890C085A
:108C100070B5B0F87921044690F87431B0F8755108
:108C20001A44D0F8811102F089FE2A2D40F0B48058
:108C3000E36804F16D06B4F87F211A81E368D4F883
:108C400081215A60E56820F0F1FC9FED817B286668
:108C50000125D4F87520D4F87930E16843EC162B5F
:108C600026EE076BBDEEC66B81ED056AD4F87D205C
:108C7000D4F88130E16843EC162B26EE077BBDEE7D
:108C8000C77B81ED067AD4F88520D4F88930E16875
:108C90009FED717B43EC162B26EE077BBDEEC77B69
:108CA00081ED047AE36883F85C50E368D4F88D20A2
:108CB0009A65E36894F8AE2083F83220D4F89530B2
:108CC00007EE903AD4F8993000EE103A20EE000A00
:108CD000A7EEA70AB7EEC00A73F016F9B7EEC00BFD
:108CE000E3689FED5F7A83ED110AE268316B91646E
:108CF000E26882F85250E26882F85350B36BE2683F
:108D000007EE903A67EE877AFCEEE77AC2ED207ABA
:108D1000E36894F8AE2083F88420D4F86D30E268DC
:108D2000C3BBD4F87130222B0FD81F2B30D8102B97
:108D300016D00F2B07D9122B03D8102B03D00423E6
:108D40000FE0142BFBD001230BE0322B02D003D811
:108D5000302BF8D1062304E0443B012BEFD9F2E796
:108D60000323537094F85A3043F0010384F85A30C7
:108D700094F85A309A07C3F3400065D5E268E16D74
:108D80005268914226D123F0030384F85A305BE005
:108D90000523E6E75570E5E7632D1DD0AE2D4ED1D6
:108DA000D4F87520DFED2F6A07EE102AE36827EE6E
:108DB000267ABCEEC77A17EE102ADA85D4F8792025
:108DC000E36807EE902A67EEA67AFCEEE77A17EEE4
:108DD000902A1A86002037E0D4F87D2004F16D0532
:108DE000D4F881302046E16843EC172BF7EEC77BBF
:108DF000C1ED077AD4F88520D4F88930E16843ECD6
:108E0000172BF7EEC77BC1ED087A02F0F3FC2A6A54
:108E10006B6AE06843EC172BF7EEC77B0122F1EE9B
:108E2000677AC0ED0F7AE36883F85020D4F8813177
:108E3000E36594F85A3043F0020384F85A3094F80A
:108E40005A0010F0010093D170BD00BFAFF3008055
:108E500000000000D01263410000000000005940F3
:108E600000007A440000C8420823054A01F00100CE
:108E7000490800B15140013BF8D10846704700BF96
:108E80002083B8EDF8B5054614465618A6420AD018
:108E900014F8010B1F0A5840C1B22846FFF7E4FF3F
:108EA00087EA0003F2E71846F8BD000038B590F8ED
:108EB0006C300446013B082B06D8DFE803F010199C
:108EC0001D26374C50586000AA2904BF012380F8A2
:108ED0006C30002380F88D3184F88E3104E0442911
:108EE00004D1022384F86C30002038BD0023F9E758
:108EF0001229FBD10323F5E7042380F8741180F8CD
:108F00006C3080F88D310023E6E7B0F88D311B2BF3
:108F1000ECD8C218013382F871119AB2A0F88D31E1
:108F200090F874319342DFD80523DBE7B0F88D3138
:108F3000FF2BDBD890F874011A1A0133224482F80F
:108F40006D109AB2A4F88D31B4F8793103449A4285
:108F5000CADB0623C6E70723C0F86D11C2E7D0F8C5
:108F60006D3103EB01210823C0F86D11BAE7D0F889
:108F70006D3103EB01410923C0F86D11B2E7D0F860
:108F80006D51002300F2711205EB016580F86C3021
:108F900090F87411C0F86D51FFF774FF04F16D0281
:108FA0000346B4F879112046FFF76CFF854204D1DF
:108FB0002046BDE83840FFF72BBEA36E0133A36601
:108FC00092E7000073B58368044693F91330F3B158
:108FD00020F02CFB94F860300546032B17D8626E06
:108FE000824214D2144AC835666852F823100846E3
:108FF0000191F8F795F9336802460199DB6830462C
:10900000984794F860306566013384F86030002535
:10901000606803681B69984750B1606803685B69C2
:109020009847C1B22046FFF741FF2843C5B2EFE79A
:10903000284602B070BD00BFF0890C0806207047BA
:1090400000487047588A0C0801207047014B0120E6
:109050000B6070470AD7A33D836F01200B607047F8
:10906000836893F9133023B1006E031F58425841AF
:109070007047012070470000836F13F4746F0CBFBA
:10908000012000207047000010B50446406E70F0CB
:10909000F9FC204610BD000010B50446FFF7F4FFB0
:1090A0002046FBF74DFD204610BD00008268436F4F
:1090B00092F90E2003F42073022A04D0A3F5207342
:1090C000584258417047B3F5207F08D0064B1B68C3
:1090D0005B6D93F89C3023B990F87C0070470120B9
:1090E00070470020704700BFC045003007B5836857
:1090F00093F913307BB1026E042A0CD0C3684FF091
:10910000030C197804230131CDE9003C90F85A3062
:109110000248FAF78DFB03B05DF804FB5C8A0C088B
:1091200010B5044602F036FB0B4B23600B4BE36695
:109130000023236784F87E3020F078FAE268012368
:10914000A066204682F88530A268128D920744BF3F
:10915000E26882F82C3010BD1C8D0C08908A0C0837
:1091600030B52DED028BB0F8843040F6AE7285B08C
:109170000446C3F30C03934200F032810AD840F650
:10918000A172934200F01D8140F6A77293423AD03B
:10919000002000E140F6BC72934200F0448141F2AD
:1091A00014729342F4D1B0F88620D0F8881002F0FF
:1091B000C5FBD4F8903007EE903AD4F8943007EE1F
:1091C000103AD4F8983000EE103AE368B4EE407AE2
:1091D000F1EE10FA37FE000AF4EE407AF1EE10FAE2
:1091E00037FE800ADFEDA27AB4EEE70AF1EE10FA5C
:1091F000C0F21581012283F85120E46872F078FFF3
:1092000084ED100AC4E7B0F88C304FF6FF7299B2C3
:10921000914205D0C2681381C368D0F888205A6093
:10922000B4F886202046D4F8881002F087FBE56861
:1092300020F0FCF9DFED8F7A2866D4F8AC3007EE29
:10924000103AB4EEE77AF1EE10FA3BDDE268012560
:1092500020465363E368D4F8B0209A63D4F8B4305E
:10926000E26807EE903AF1EE677AC2ED0F7AE368B2
:1092700083F85050E16802F0E9FAB4F8CE300A21E0
:10928000E268DFED7D6A4B43C2F88030B4F8DA2043
:10929000E36807EE102AB8EE477A27EE267A83EDC8
:1092A000117AB4F8DC20E36807EE902AF8EE677ACA
:1092B00067EEA67AC3ED127AE36883F85250E3684A
:1092C00083F85350D4F89020D4F894309FED627B0B
:1092D00043EC162BB4EEC76BF1EE10FA3CDDE168FF
:1092E0009FED5F5B43EC172B9FED5F6B27EE057BDC
:1092F00027EE067BBDEEC77B81ED057AD4F898207A
:10930000D4F89C30E16843EC172B27EE057B27EE61
:10931000067BBDEEC77B81ED067AD4F8A020D4F899
:10932000A430E16843EC172BD4F8A830B7EEC77B24
:10933000012207EE903A77EE677A9FED507A67EE5A
:10934000877AFDEEE77AC1ED047AE36883F85C2062
:10935000E368D4F8A8209A6594F8CA30FF2B1CBFA4
:10936000E26882F8323094F88E3003F00F03082B55
:1093700009D8DFE803F0051417141A1D171A1D0089
:10938000E36801225A7094F88E30012013F0400FE8
:1093900011D0E368587005B0BDEC028B30BDE368B6
:1093A0000322EFE7E3680422ECE7E3680622E9E73B
:1093B000E3680522E6E71B06EDD5E36802225A7052
:1093C000E9E7B0F88620D0F8881002F0B7FAE36831
:1093D000B4F89420DA85E368B4F896201A86D7E6C4
:1093E000B0F88620D0F8881002F0A8FAD4F89430AB
:1093F000A26F6367D4F8983082EA030111F4746FA6
:1094000009D0E16803F4746302F474621C480978BB
:109410000131FAF70DFAD4F89830A367B8E60020C6
:1094200083F85100B7E7B0F88620D0F8881002F032
:1094300085FA94F88E00E36820BB83F88400E36823
:10944000C3F88000E368C3F88C00E368C3F88800C1
:10945000E368C3F890009EE700000000006A08C1BE
:10946000F8C1631ADCA54C4000000000D012634133
:1094700000000034005043C80AD7A33B0000C84294
:10948000A08A0C0894F8902083F884204FF6FF728D
:10949000B4F8BD30934216BF0A2200235343E2685A
:1094A0009FED537BC2F88030D4F89420D4F89830E4
:1094B000E56843EC162BB4EE476BF1EE10FA00F0C2
:1094C0008780D4F89C00D4F8A01041EC160BB4EEC1
:1094D000476BF1EE10FA7BD0D4F8A400D4F8A810B2
:1094E00041EC160BB4EE476BF1EE10FA70D0B4F805
:1094F000B8004FF6FF7188426AD09FED3F6B43EC96
:10950000172B27EE067BBDEEC77B85ED237AD4F8BB
:109510009C20D4F8A030E16843EC172B27EE067BA3
:10952000BDEEC77B81ED227AD4F8A830D4F8A42010
:10953000E1689FED337B43EC162B26EE077BBDEEF7
:10954000C77B81ED247AA368188D10F002003FF4E8
:1095500022AFB4F8B83001A8D4F89C2007EE903AB6
:109560009FED297AD4F8A030F8EEE77A9FED278AAC
:10957000A7EE878A43EC172BD4F89420F7EEC76B3D
:10958000D4F8983043EC172BD4F8A420B7EEC77B5F
:10959000D4F8A830CDED016A8DED027A43EC152B9D
:1095A000F7EEC57BCDED037A09F068FAD4F8A42074
:1095B000F0EE400AD4F8A830B0EE480A204643EC5A
:1095C000172BB7EEC71BB1EE411A02F0FDFADFE52B
:1095D0000020C5F88C00E368C3F88800E368C3F88E
:1095E0009000E36883F85400D5E600BFAFF3008035
:1095F000BBBDD7D9DF7CEBBD0000000000408F4031
:109600000000000000408FC00AD7233C0000344314
:109610002DE9F84F90F87E3004460D46013B082BAB
:1096200006D8DFE803F0404B4F575B63677DB2001D
:10963000242908D1012380F87E300023A0F8883146
:109640000020BDE8F88F90F88F314FB2DFF8F0912D
:109650004FF006085E1C00F5C57B0344F6B2032EEE
:10966000B24680F88F61A8BF4FF0030A83F88A7171
:109670005246594659F8040B75F098FF78B9042EF4
:1096800006D1303F092FDBD9002384F88F31D7E78B
:10969000D6D93E2DF8D1012384F89031F4E7B8F102
:1096A0000108E5D1F0E7402903D1022384F87E3098
:1096B000C6E7522940F09A800923F7E70323A0F870
:1096C0008210F3E7B0F88210042301EB0525A0F81F
:1096D0008250EBE70523A0F88410E7E7B0F8841088
:1096E000062301EB0525A0F88450DFE70723A0F847
:1096F0008610DBE7B0F8861001EB0525ADB2AB07AD
:10970000A0F886500CBF08230023072D80F87E3078
:1097100096D8002380F87E30236F013323678FE7CC
:10972000B0F88831FF2B98BFC21803F1010398BF2E
:1097300082F888109BB2B0F88620A0F88831083AE9
:109740009342FFF67DAFB3F5807F4FD80022022110
:10975000843007F0AFFA0221024604F1860007F0D8
:10976000A9FAB4F88610024604F18800083907F017
:10977000A1FA002384F87E30B4F882308342CBD142
:109780002046BDE8F84FFFF7EBBCB0F88821FE2A71
:109790002CD8831801320A2992B283F88810A0F8D5
:1097A00088217FF44DAF8318002183F8881090F84A
:1097B00088303A2B1AD1466EC6B100F18A01053ABB
:1097C000304675F0F3FE054680B9304670F05AF920
:1097D000236E6566042B06D8DFE803F0030A0C1A33
:1097E0002800012323661FF021FFA06600235DE708
:1097F0000223F7E794F85A300133DBB2032B84F8E5
:109800005A30F0D903232366002384F85A30EAE75C
:1098100094F85A30A2680133DBB284F85A3092F9D6
:109820000C200AB1022BDED90423DBE704F00EF88A
:1098300040F261124FF4801103F0F4FFD3E700BF50
:10984000EC8C0C084068112201490368DB6818475A
:10985000CC8A0C0838B58368054693F90E303BB3C3
:10986000406F10F4007412D1EB681248197801317E
:10987000F9F7DEFFEB68104819780131F9F7D8FFE6
:109880002846FFF7DFFF85F87C40002038BDC30580
:1098900006D5EB68094819780131F9F7C9FFF4E7F3
:1098A00010F0800404D1EB68054819780131F4E721
:1098B0000120EBE7E08A0C08008B0C08218B0C08D8
:1098C0003A8B0C0810B504460548F9F7B1FF13228E
:1098D000606804490368BDE81040DB68184700BFB2
:1098E000608B0C08748B0C08F0B5044640680025AA
:1098F00085B003682E461B6998470746BD420BD0CA
:109900006068013503685B699847C1B22046FFF77C
:109910007FFE0643F6B2F1E7A36893F91320FAB18C
:10992000226E042A00F093801FF080FEE36D05464E
:10993000834215D2A36E03F5FA63834213D2E06E1D
:10994000F7F7EEFC0746606803681B6A9847B84261
:1099500006D360683A46E16E0368DB689847A566FF
:10996000304605B0F0BD94F89031002BF8D0636E0E
:109970002BBB236E042B22D8DFE803F00337444AC5
:109980006100D4E90232606804F16405127813447E
:1099900093F92220036803921B6E98473E493F4B80
:1099A000039A012808BF0B463D49284600934FF40F
:1099B00061331CF0FDFF013001D100236366606E4E
:1099C0000028CDD0F7F7ACFC0546606803681B6A39
:1099D0009847A842C4D360682A46616E0368DB6872
:1099E0009847002384F89031BAE7D4E902322D4930
:1099F00004F1640012781344012293F922301CF020
:109A0000D7FFD8E794F85A20274B53F8222009E0D3
:109A1000A36893F90C30012B0AD0022B0CD0002B39
:109A2000CDD1224A224904F164001CF0C1FFC2E7F3
:109A300094F85A201F4BE8E704232366BFE703F09E
:109A400005FF96224FF4801103F0ECFEB7E793F97F
:109A50000E30022B84D1184B1B685B6D93F89C3041
:109A60001BB1012384F87C307AE794F87C30002B1A
:109A70003FF476AF636F9B057FF572AF1FF0D6FDA5
:109A8000E36D05468342BFF46BAF05F57A7520465A
:109A9000FFF718FFE56563E78D8B0C08888B0C08D2
:109AA000958B0C08B88B0C08048D0C08118C0C08D5
:109AB000D49E0C08E08C0C08C0450030062070478E
:109AC000836893F913302BB1D0F8B804B0FA80F062
:109AD0004009704701207047004870476C8D0C08A2
:109AE00010B40022D0F8B834012101FA02F41C426B
:109AF0000AD0C1680748097850F822200131064889
:109B00005DF8044BF9F794BE0132142AEDD15DF8EB
:109B1000044B7047DC8F0C08748D0C08054B10B596
:109B200004460360D0F8E80408B1FBF709F82046C2
:109B300010BD00BFEC920C0810B50446FFF7EEFF15
:109B40002046FAF7FDFF204610BD000010B5D0F802
:109B5000E804144628B102F06FF82080003818BFDE
:109B6000012010BDD0F8E80408B102F047B87047F2
:109B700013B5044601F0C0FE94F88C3463B105F0CF
:109B8000B5F8E36805491A7804F28D430132009371
:109B900004F2AB4304F002FB02B010BD9C8D0C0834
:109BA00090F8BC34822B08D81A0613D4033B012B3F
:109BB0000ED90D4B0B6001207047FF2BF9D10A4BDA
:109BC0000B60836893F91300B0FA80F04009704786
:109BD000064BEFE7054B0B6090F8CC34013B012BB3
:109BE000E9D8034BE6E700BFAE47613E8FC2F53DC3
:109BF0000AD7233E10B586B0044601F09BFEC8B3D9
:109C000016220021684675F099F8A3238DF80030DC
:109C100095238DF801305E238DF802301FF00EFD84
:109C2000E368CDF80710CDF803001B788DF80B30F2
:109C3000B4F86A30ADF80C3094F887308DF80E30F7
:109C400094F86F308DF80F30B4F86C30ADF81030F8
:109C5000D4F8B834CDF81230B4F86E34442B04BFC5
:109C600094F88F308DF80E3005F040F816226946D2
:109C700004F036F906B010BD1FB5044601F05AFED7
:109C800068B310220021684675F058F8A3238DF8B8
:109C9000003095238DF801305F238DF802301FF0DE
:109CA000CDFCE368CDF80710CDF803001B788DF8E4
:109CB0000B3094F85A308DF80C3094F85B308DF8F6
:109CC0000D3094F85C308DF80E3094F85D308DF8DE
:109CD0000F3005F00BF81022694604F001F904B0CA
:109CE00010BD000030B591B0044601F023FE0028FD
:109CF00031D004F0FBFF05461FF0A0FCD4F8723011
:109D0000164A0E93D4F86E300D93D4F86A300C9343
:109D1000B4F860300B93D4F866300A93D4F862300C
:109D20000993B4F85E300893B4F85C30079394F864
:109D30005B30069394F85A300593E3681B780493DC
:109D4000074B0193074BCDE9020100932846064BD0
:109D5000064904F06BFC11B030BD00BFC18D0C088A
:109D6000038E0C08108E0C08B48D0C08FE8D0C08A8
:109D70002DE9F0478CB00C4601F0DCFD002847D0FF
:109D80001FF05CFC002507460E464FF0A30A4FF07B
:109D900095094FF05B08A279EBB29A4238D98DF859
:109DA000152018222168013502FB0343CDF80F105E
:109DB0001A7FB4F904108DF804A08DF805908DF881
:109DC0000680CDF80770CDF80B60ADF813108DF854
:109DD00016209968DA68CDF81710CDF81B205A695B
:109DE0001969CDF823209A69CDF81F10CDF82720E6
:109DF0005A7F8DF82B209A7FDB7F8DF82C208DF8F1
:109E00002D3004F073FF2A2201A904F069F8C2E79B
:109E10000CB0BDE8F08700002DE9F04792B00C4689
:109E200001F088FD00287CD01FF008FC5C2322682C
:109E30004FF0A3098DF806304FF0950863680027AE
:109E40004FF05D0A0D46CDF8133006462389CDF854
:109E50000B10ADF81730A37ACDF80F208DF819301C
:109E6000E37A8DF804908DF81A30237B8DF8058005
:109E70008DF81B30CDF8070004F038FF182201A937
:109E800004F02EF8E27AFBB29A424AD904EB43136B
:109E90008DF81C908DF81D8001378DF81EA0CDF82F
:109EA0001F60CDF8235019695A69CDF82710CDF8F5
:109EB0002B20DA699969CDF833201A6ACDF82F1072
:109EC000CDF8372093F824208DF83B2093F82520F7
:109ED0008DF83C2093F827208DF83D2093F8291029
:109EE00093F8282042EA0122ADF83E2093F82A2078
:109EF0008DF8402093F82B208DF8412093F82C20EA
:109F00008DF8422093F82D208DF8432093F82E30C1
:109F10008DF8443004F0EAFE292207A903F0E0FF9F
:109F2000B0E712B0BDE8F087C1F302710139C9B2E0
:109F300004299ABF014B585C00207047D48F0C084D
:109F400030B5D0F8D43473B190F8D8540020C2B2F0
:109F5000954208D953F83020441C8A4201D140B2BE
:109F600030BD2046F3E74FF0FF30F9E730B5039CF2
:109F70000A44914209D011F8015B18782844C0B214
:109F80001870257828442070F3E730BD2DE9F041A2
:109F90000446406886B01D4603688846BDF83060B8
:109FA00017461B6A984706F1080398424FF00000D5
:109FB0003AD3B5238DF813700DF10F0704228DF8F5
:109FC000103062230DF112018DF80E008DF80F0094
:109FD00020468DF811300DF10E0300978DF8128098
:109FE000ADF81460FFF7C2FF3246294620460097BD
:109FF000FFF7BCFF6068062204A90368DB68984786
:10A000006068324629460368DB6898476068012229
:10A010000DF10E010368DB6898476068012239463C
:10A020000368DB689847012006B0BDE8F0810000B6
:10A0300013B50446406803681B6A9847072806D989
:10A040000023062120461A460093FFF79FFF02B027
:10A0500010BD00001FB590F88B34052B05D9FFF714
:10A06000E7FF002005B05DF804FB02238DF80C101B
:10A070008DF80D2006210093012203ABFFF786FF28
:10A08000F0E70000F0B5044640681D4685B003685F
:10A090000F4616461B6A98470A280FD90323012248
:10A0A00006212046009303AB8DF80C708DF80D60EF
:10A0B0008DF80E50FFF76AFF05B0F0BD0020FBE7FA
:10A0C00090F8CE340133DBB280F8CE342BB990F85F
:10A0D0006D2490F87214FFF7D5BF70470A2938B580
:10A0E0000546184663D004D801290AD0022964D055
:10A0F00038BD0D29FCD1032AFAD14FF48024012365
:10A100002EE0122A35D8012AF2D9931E102BEFD84F
:10A1100001A454F823F000BF7FA104088BA1040818
:10A120005DA10408F1A0040897A10408CDA10408CA
:10A13000F1A00408F1A00408F1A00408F1A00408AB
:10A14000F1A00408F1A00408F1A00408F1A004089B
:10A15000F1A00408F1A00408A3A10408012320240D
:10A16000834239D1D5F8B83423EA0403C5F8B834AA
:10A17000BEE7202ABCD14FF400440523F0E795F850
:10A18000D24484F001030224EAE795F8D24484F033
:10A1900001030424E4E795F8D24484F00103082481
:10A1A000DEE795F8D24484F001031024D8E7092AA9
:10A1B00010D00B2A9CD18024DFE7102A01D0152A69
:10A1C00096D1AB684FF480749B7BC9E701234FF4B1
:10A1D0000054C5E74024D0E72846FFF753FFD5F8E1
:10A1E000B8342343C5F8B834012385F8D0347FE769
:10A1F0002DE9F04385B0541C9146002602AFC0F80B
:10A20000E034A40097F82830054680F8D8246A4640
:10A2100080F8E434E31DC0F8D414013CDB08C0F836
:10A22000DC644068A4B2A2EBC303884602689D4682
:10A23000126A02AB7B60904704F1090292B290422D
:10A2400018D3414603AA08EBC9097B680296494521
:10A2500004D051F8080B42F8040BF8E701348B22C4
:10A2600006212846A4B20094FFF790FE0C37BD46A5
:10A27000BDE8F0833046F9E70C23092213B5044604
:10A28000062100930A4BFFF781FE1FF0CFF994F8E7
:10A290008034C4F87C040133064884F88034E368D1
:10A2A0001978013102B0BDE81040F9F7C1BA00BF1A
:10A2B0003C930C08208E0C0810B5002308248278EB
:10A2C000082A0ED8DFE802F00B051217202B3747BB
:10A2D0004D00622902D10223837002E08370B52908
:10A2E00001D0002042E083780133F5E70323C170F9
:10A2F00083700171F5E704238370C37819440379EF
:10A30000C9B2C1701944F4E7052302790170837062
:10A31000C3780B44DBB2C37013440371E1E7062337
:10A320008370C37819440379C9B2C17019440023FA
:10A3300001714370D5E7C378027819440379C9B233
:10A34000C1701944437801710133DBB29A42437002
:10A35000C7D10723C0E7C27884708A42C1D0837016
:10A36000ADE7027983708A42A9D1012010BD0000B7
:10A37000002307B504220A210093FFF707FE03B06C
:10A380005DF804FB1FB5C368044680681978FDF7C3
:10A39000EDFD012306210822ADF80A300023ADF8B7
:10A3A00008002046ADF80C3002AB0091FFF7EEFD3F
:10A3B00004B010BDB0F86E24083201F0BFBA00003E
:10A3C00090F8BC0400F0FD00A0F180035842584111
:10A3D000704700002DE9F04F85B006460C469246C6
:10A3E00002AF9B46FFF7ECFF20B900200C37BD46BB
:10A3F000BDE8F08F3046FFF797FD00238046C7E9A0
:10A40000003300F10F0370681FFA88F523F007038B
:10A41000ADEB030D03681B6A0DF10809984705F1C0
:10A4200010039BB29842E0D37C6001233C46083580
:10A430003B70424687F801B0ADB203CC029004A84D
:10A440000391514674F052FC4B468A220621304655
:10A450000095FFF79BFDC9E72DE9F04F2DED028B2D
:10A4600090F8721495B00446052948D190F86D24EF
:10A47000012A01D000201BE090F85A30062B0CD0A6
:10A480000A2BF7D190F85B30092B33D00B2BF1D18D
:10A49000D0F8B83423F0800322E090F85B30242B0E
:10A4A0001AD00AD8092B4FF0000010D0162B1AD062
:10A4B00015B0BDEC028BBDE8F08F312B00F00282AD
:10A4C0003E2BD7D1D4F8B83423F4006308E084F8E5
:10A4D000732484F8D004EBE7D0F8B83423F4806315
:10A4E000C4F8B834C6E7D4F8B83423F48053C4F8B9
:10A4F000B834DDE7D0F8B83423F04003F0E706299C
:10A5000010D190F86D24242A00F0CC8000F28880CD
